:1000000000800020BD01000021D30000D9D20000F3
:10001000D9D20000D9D20000D9D20000D9D2000034
:10002000D9D20000D9D20000D9D2000021D30000DB
:1000300021D30000D9D20000A9F50000ADF60000E0
:1000400021D3000021D3000021D3000021D30000E0
:1000500021D3000021D3000021D3000021D30000D0
:1000600021D3000021D3000021D3000021D30000C0
:1000700021D3000021D3000021D3000021D30000B0
:1000800021D3000021D3000021D3000021D30000A0
:1000900021D3000021D3000021D3000021D3000090
:1000A000F5B3000001B4000021D3000021D300000B
:1000B00021D3000021D3000021D3000021D3000070
:1000C00021D3000021D3000021D3000021D3000060
:1000D00021D3000021D3000021D3000021D3000050
:1000E00021D3000021D3000021D3000021D3000040
:1000F00021D3000089F8000021D30000B5F90000E9
:1001000021D3000069E0000021D3000021D30000CA
:1001100021D3000021D3000021D3000021D300000F
:1001200021D3000021D3000021D3000021D30000FF
:1001300021D3000021D3000021D3000021D30000EF
:1001400021D3000021D3000021D3000021D30000DF
:1001500021D3000021D3000021D3000021D30000CF
:1001600021D3000041E3000021D3000021D300008F
:1001700021D3000021D3000021D3000021D30000AF
:1001800021D3000021D3000021D3000021D300009F
:1001900021D3000021D3000021D3000021D300008F
:1001A00021D3000021D3000021D3000021D300007F
:1001B00021D3000021D3000021D30000564B4CF284
:1001C000205210B51A804DF628121A8000BF00BFC9
:1001D0000DF0AAF8514B4FF010621A60504A9A6025
:1001E000504ADA60504A136813F4807304D14F49BF
:1001F0000B604FF4A85313604D4B1A78110703D5C9
:100200001A7842F008021A704A4B4B492A221A7097
:100210004A4A4B4B8B4204D252F8040F43F8040B6A
:10022000F8E7484B484900228B4202D243F8042B9E
:10023000FAE74649464A002352F8230041F82300D2
:1002400001336F2BF8D1434B434A802103F8011B44
:100250009342FBD1414B3D4A1A60414B8A221A70AE
:10026000A3F5805324225A70A0221A709A7992071B
:10027000FCD59A79D406FCD43A4A937903F00C035E
:10028000082B384BF9D103221A7140225A719A79FE
:100290009006FCD5334A9179324B4906FBD5324A58
:1002A000324911600221516020221A709A7902F0BD
:1002B0000C020C2AFAD12E4B2E4A1A602E4B2F4AD2
:1002C0001A6000225A60072243F8042C2C4AC3F813
:1002D0000C2D62B60DF090FD144B1B68DA0705D5A6
:1002E00028480DF05DFB284B284A1A60284B1B78E4
:1002F0005B0609D5244C254B22689A4204D121483B
:100300000DF04EFB0023236010F05CFE0DF012F8A0
:100310000FF040FAFEE700BF0E2005403080044099
:10032000823F04000100002B10D0034014D0034092
:1003300002D0074000E007403C9DFF1FC846010077
:100340004088FF1F3C9DFF1FC0A3FF1F0082FF1FAF
:100350000000000000E400E05FE400E008ED00E0E1
:100360000050064000400640448004400000030165
:1003700004800440C010050014E000E0FF76010096
:1003800000002020DF0AE95C1CE00340A5C3945A6A
:1003900000F00740FFFFFFFFFFFFFFFFFFFFFFFF32
:1003A000FFFFFFFFFFFFFFFFFFFFFFFFFFFFFFFF5D
:1003B000FFFFFFFFFFFFFFFFFFFFFFFFFFFFFFFF4D
:1003C000FFFFFFFFFFFFFFFFFFFFFFFFFFFFFFFF3D
:1003D000FFFFFFFFFFFFFFFFFFFFFFFFFFFFFFFF2D
:1003E000FFFFFFFFFFFFFFFFFFFFFFFFFFFFFFFF1D
:1003F000FFFFFFFFFFFFFFFFFFFFFFFFFFFFFFFF0D
:10040000FFFFFFFFFFFFFFFFFFFFFFFFDEF9FFFF23
:1004100010B5054C237833B9044B13B10448AFF33E
:1004200000800123237010BD3C9DFF1F00000000D1
:10043000CC460100084B10B51BB108490848AFF382
:1004400000800848036803B910BD074B002BFBD0A0
:10045000BDE81040184700BF00000000409DFF1F8E
:10046000CC4601003C9DFF1F0000000070B44C68AA
:10047000A04220D901230133DBB21CB2A60051F8FF
:10048000244084421D46F6D3A04211D005F1804598
:10049000013D965951F8251052F82530401AF21AAC
:1004A00000FB02F0641AB0FBF4F4E01870BC704773
:1004B000905970BC704704260125E5E700280CDA46
:1004C000064A434282FB0320DA17C2EB600000EBCE
:1004D0004000A3EB8000C0F10C007047ABAAAA2A31
:1004E000684B1B880C2B12D8DFE803F01E29333D24
:1004F0001148525C66707A12070063490B68984293
:1005000078D90B6C9842C0F0A580604B186C70478E
:100510005D490B68984240F28E800B6C9842C0F0A7
:1005200096805B4B186C704757490B6898427FD98F
:100530000B6C9842C0F08880564B186C704752493B
:100540000B68984271D90B6C98427AD3524B186C55
:1005500070474D490B68984264D90B6C98426DD333
:100560004E4B186C704748490B68984257D90B6C32
:100570009842C0F084804A4B186C704742490B681F
:10058000984249D90B6C984276D3464B186C704709
:100590003D490B6898423CD90B6C984269D3424B59
:1005A000186C704738490B6898422FD90B6C9842E9
:1005B0005CD33E4B186C704733490B68984222D984
:1005C0000B6C98424FD33A4B186C70472E490B680E
:1005D000984215D90B6C984242D3364B186C704731
:1005E00029490B68984208D90B6C984235D3324B95
:1005F000186C7047254B186870472F4B1868704768
:100600002C4B186870472A4B18687047274B18689E
:100610007047254B18687047224B18687047204B6D
:10062000186870471D4B186870471B4B1868704757
:10063000184B18687047164B18687047174AFFF731
:1006400015BF154AFFF712BF124AFFF70FBF104A36
:10065000FFF70CBF0D4AFFF709BF174AFFF706BFA8
:10066000144AFFF703BF124AFFF700BF0F4AFFF714
:10067000FDBE0D4AFFF7FABE0A4AFFF7F7BE084A69
:10068000FFF7F4BEA49EFF1F988AFF1F848BFF1FF5
:10069000408BFF1F488DFF1F3889FF1F048DFF1FF0
:1006A000C08CFF1FA08DFF1F7C89FF1FC089FF1F0B
:1006B000048AFF1F648CFF1FFC8BFF1F38B5284A7C
:1006C000284B14881D68AC4247DA274A274B10682C
:1006D0001B88421F191BAB42A8BF2B469142A3EBBC
:1006E0000403C3BF043843430131534393FBF1F187
:1006F00005310A200DF066F91D4A1E4B14881B684F
:10070000A34205DC00210920BDE838400DF05AB9AC
:1007100019491A4A0D881068AB42A5EB0401A0F1F3
:100720000502A8BF2B4691420CDD1B1B043800FBC1
:1007300003F30131092093FBF1F1BDE838400531A5
:100740000DF040B91B1B02FB03F3092093FBF1F1F1
:10075000BDE8384005310DF035B90021C9E700BFCB
:100760001A9EFF1FE09EFF1FF88DFF1FF49EFF1FC4
:10077000E89DFF1F689DFF1FD49EFF1F8C8DFF1FEC
:100780002DE9F04F8FB002AD0024E1B26E480AF0BF
:10079000A5FE01340C2C45F8040BF6D16B4B6C4CC8
:1007A000B3F800E00A9B00227345227014DB089B1B
:1007B0009E4500F3B480069B664A9E4503DD137890
:1007C000002B40F0BC80049B9E4540F3AE804FF070
:1007D000020C84F800C009E0069B5E4A9E45CCBF2F
:1007E0004FF0060C4FF0050C84F800C00C9F039EE0
:1007F0000598079982F800C0BE45D4BF002701279D
:10080000B645D4BF002601268645099ADFF87081D7
:100810000B9B0D9DDFF86CA1DFF86C918AF80060EE
:10082000D4BF002001208E45D4BF0021012188F8CB
:10083000001096454849DFF854B1484E89F8000049
:10084000D4BF002201229E45D4BF002301230A7099
:10085000AE45434A8BF80070D4BF00250125012026
:10086000137035700DF06CFC3E4B3F4A1D681188CB
:100870003E4BA842D4BF002201220B291A7001D995
:100880000C2901D0A84246DC00230193384B9AF88A
:1008900000E01F7899F800C098F800209BF800301D
:1008A0002D49DFF8ECA091F800902D49367891F8A9
:1008B00000802478A7EB4E07CCEB070CA2EB82025A
:1008C000C3EB83776244C3EB8703134403EB490311
:1008D000BAF80020274FDFF8BCE0B7F800C0264F79
:1008E000434403EB8606033A0C2313FB046602EB36
:1008F000420206EB8202019BCEF800606244A842ED
:10090000A2F10C021A44C8BF1C4B3A60C8BF1E704B
:100910000FB0BDE8F08FA1F10C030193B6E74FF0E3
:10092000040C84F800C00B4A60E7029B9E45C6BFDA
:100930004FF0010C84F800C04FF0000C56E74FF068
:10094000030C84F800C051E7149EFF1FFC9EFF1F9C
:10095000489EFF1F549EFF1FDD9EFF1F399FFF1FF4
:10096000389FFF1F548CFF1FD69EFF1F949DFF1FB3
:10097000BC8CFF1FA89DFF1F009FFF1FFE9EFF1F37
:10098000359FFF1FCC9EFF1F349FFF1F369FFF1F09
:10099000BE9EFF1FF49DFF1F30B50E4C85B0012396
:1009A00020463C2202210BF0C7FF20460BF054FFEB
:1009B00001250022402180232046019100930295C9
:1009C0001146054B0BF054FA204605B0BDE8304007
:1009D0000CF0E4B80C9FFF1FC438010010B500EB09
:1009E000C000821DD2B293B284B09C1E981C3D23DD
:1009F00003918DE81900392102480BF09DF904B0EC
:100A000010BD00BF0C9FFF1F70B50E4C84B01225A7
:100A10000422012306460390029320468DE8240019
:100A2000142310210BF088F9062209230293039660
:100A3000019520460092142310210BF07DF904B09B
:100A400070BD00BF0C9FFF1F10B50C4C81B220463B
:100A50000BF054FC204602210BF04AFC20462122D8
:100A60005A210BF041FC064B204619880EF08AFEF5
:100A70002046BDE810400EF035BE00BF0C9FFF1FA2
:100A8000B88CFF1F10B50C4C81B220460BF036FC21
:100A9000204602210BF02CFC204621225A210BF08B
:100AA00023FC064B204619880EF06CFE2046BDE85C
:100AB00010400EF017BE00BF0C9FFF1F948AFF1F4F
:100AC00010B50C4C81B220460BF018FC20460221D8
:100AD0000BF00EFC2046212253210BF005FC064BA7
:100AE000204619880EF04EFE2046BDE810400EF05C
:100AF000F9BD00BF0C9FFF1FBA8CFF1F38B50C4615
:100B00000546C9B20CF0C0FB210A681CBDE838409C
:100B10000CF0BABB38B505460CF09CFB4FF0000456
:100B200060F30704681C0CF095FB60F30F24A0B27F
:100B300038BD00BF38B50F4D2B78013B01381B0283
:100B4000C4B203F47063200443F4404343F00C0345
:100B500000F4FE0018430EF0C5F82868013860F074
:100B60003F00C0B20DF05AFA2046BDE838400DF003
:100B700055BA00BF009EFF1F38B5104D2B78013BC2
:100B80001B0203F47063044643F41043000443F073
:100B9000090300F4FE0018430EF0A4F82868013899
:100BA00060F06F00C0B20DF039FA20460DF036FA51
:100BB0000020BDE838400DF031BA00BF009EFF1F95
:100BC00038B50E4D2B78013B1B0203F470630446CD
:100BD00043F45043000443F00D0300F4FE001843B7
:100BE0000EF080F82868013860F02F00C0B20DF0D8
:100BF00015FA2046BDE838400DF010BA009EFF1FE0
:100C000010B504464FF440600DF0B8F90DF010FA3D
:100C10002CB1102C044BA8BF10241C6010BD024B3B
:100C200001241C6010BD00BF009EFF1F10B50446CC
:100C300041F0E0000DF0F2F904F07F000DF0EEF964
:100C4000C4F3C610BDE810400DF0E8B938B5114D39
:100C50002B78A0F50052013B1B0202F30D0202F5B6
:100C6000005203F47063044643F46043100443F0FD
:100C70000E0300F4FE005204184302F0FE4210433B
:100C80000EF030F8296801392046C9B2BDE8384075
:100C9000FFF7CCBF009EFF1F2DE9F04F172087B054
:100CA0000DF04EFADFF86093C9F8000016200DF041
:100CB00047FAB84BB84A1B8810600C2B00F04F82E3
:100CC0000023B64C0F2023700DF03AFAB44A237873
:100CD000128801921146B34A054652F821404BB1A1
:100CE00020460FF0B3FE4FF07C510FF003FF10F0E1
:100CF000DDF80446AC4BDFF814831B88D8F800A05D
:100D0000AA4A013B554552F823B050DAA84BA94EE8
:100D10001B88012B00F0D581A74BA84A30680093AF
:100D20001F4604920FF092FE4FF07C510FF0E2FE4E
:100D3000A34902900988039120460FF087FE049A88
:100D400003993F6852F821100FF0D4FE01460020AD
:100D50000FF0C6FD10F0AAF8CBEB070BAB45CAEBC2
:100D60000B015A46B8BF2A46CAEB02028842BABFF4
:100D700000FB02220131424392FBF1F0DFF890A226
:100D80000FF064FE4FF07C510FF0B4FE02990FF0AB
:100D9000A9FD10F08BF830608A4A1288013A032AC4
:100DA0006AD8DFE812F0EB00D3005300DF00DFF871
:100DB00060A2DAF80020954238DD7D4B05921B8851
:100DC0007C4E012B00F0AC817B4B00931F463068BA
:100DD0007A4B04930FF03AFE4FF07C510FF08AFEED
:100DE000774902900988039120460FF02FFE03995E
:100DF000049B3F6853F821100FF07CFE10F056F86A
:100E0000059ABB44C2EB0B01AB45A8BFAB46884279
:100E1000C2EB0B0B80F2AD8100FB0BBB01319BFBE6
:100E2000F1F00FF013FE4FF07C51ADE7614E624BD5
:100E3000306800931F460FF009FE4FF07C510FF011
:100E400059FE10F033F83F683060A5E738460FF0E0
:100E5000FDFD5D490FF04EFE834628460FF0F6FD7E
:100E60005A490FF047FE014658460FF03BFD10F07F
:100E70001DF8009B074618605549564A0888128895
:100E8000D9F80010544DC0EB070EC3199142C8F8B1
:100E900000E0CAF80030B5F800E080F2DC80002500
:100EA000C2EB0E0C3C4B64451F6880F2C880631C8B
:100EB000974205FB03F50CF1010C95FBFCF5C0F224
:100EC0006681BE45A8BFBE46C2EB0E0E03FB0EF404
:100ED00094FBFCF4914200F39D80BA42C0F29A80E8
:100EE0003E4C20680FF0B2FD3D490FF003FE3D4936
:100EF0000FF0F8FC0FF0DAFFA0F5FF531C3B082BB6
:100F000098BF4FF400503368184400282060C0F2A6
:100F10009480B0F5804F80F2A580334B1B781BB1D5
:100F2000B0F5005F40F0A680304D2B78002B40F0EC
:100F3000A9802F4D20682B68284C984203D0FFF7DA
:100F400085FE23682B6007B0BDE8F08F38460FF0B0
:100F50007DFD28490FF0CEFD834628460FF076FD33
:100F600025497EE738460FF071FD1D490FF0C2FD9F
:100F7000834628460FF06AFD204972E738460FF095
:100F800065FD1F490FF0B6FD834628460FF05EFD54
:100F90001C4966E7D69EFF1F089FFF1F659DFF1F28
:100FA000D09DFF1F088BFF1FB88CFF1FC88BFF1F32
:100FB000FA9DFF1F849DFF1FC89EFF1F6C8AFF1FA5
:100FC000BC9DFF1F948AFF1FCDCC4C3FCDCC4C3E27
:100FD000BA8CFF1F309EFF1FB89DFF1F988DFF1F0B
:100FE0009A99193FCDCC4C45E89EFF1F159EFF1FD7
:100FF0003489FF1F6666663FCDCCCC3DCDCCCC3E60
:101000003333733FCDCC4C3DCC9DFF1FE49DFF1F80
:10101000409EFF1F019B002B3FF462AF2B1B002B58
:10102000B8BF5B42092B34DC33685A4C4FF4005094
:10103000184400282060BFF66CAF002214E09742ED
:1010400005FB04F5B8BF002395FBFCF580F2968004
:1010500093FBFCF43EE77145D4BFC2EB0105C2EB44
:101060000E051DE743F6FF724B4B22601B78002BE9
:101070003FF45AAF00210D200CF034FE474B012203
:101080001A7056E701210D200CF02CFE00232B7066
:101090004FE705F500500130001B0FF0D7FC404929
:1010A0003C4C0FF027FD054620680FF0CFFC3D4972
:1010B0000FF020FD014628460FF014FC0FF0F6FE5D
:1010C00021E7394B00931F463068384B04930FF0EB
:1010D000BDFC4FF07C510FF00DFD354A0290128897
:1010E000039220460FF0B2FC039A049B3F6853F82A
:1010F00022100FF0FFFC0FF0D9FECBEB070BAB4536
:10110000CAEB0B02B8BFAB46CAEB0B0B8242C6BFA1
:1011100000FB0BBB013200FB0BFB9BFBF2F02DE64F
:10112000224B0493204B306800931F460FF08EFC37
:101130004FF07C510FF0DEFC1D49029009880391AD
:1011400020460FF083FC049B03993F6853F821105D
:101150000FF0D0FC014600200FF0C2FB4EE601204C
:101160000CF0EEFF134B1B689842D4BF0023012301
:10117000A7E500FB0BFB9BFBF1F052E67745D4BFE4
:10118000C2EB0703C2EB0E0304FB03F360E79646D2
:101190009AE600BF988DFF1FE89EFF1F159EFF1F58
:1011A000CDCCCC3E9A99193FC89EFF1F6C8AFF1F79
:1011B000BC9DFF1F548CFF1F38B5054642F0B000A0
:1011C0000C460CF02BFF28460CF028FFE0B2BDE8DF
:1011D00038400CF023BF00BF70B50F4D2B78013B9A
:1011E0001B0203F47063044643F4304308062204F0
:1011F00000F0FE4043F00B03034302F4FE001843EB
:101200000E460DF06FFD2A68013A3146E0B2D2B2C7
:10121000BDE87040FFF7D0BF009EFF1F10B50C4C1B
:10122000236843B90B4B1B88022B0CD00A4A0023BE
:101230001370236010BD00210520FFF7CDFF054B83
:101240001B88022BF2D100214120FFF7C5FFEDE7FB
:10125000F09EFF1F249EFF1FEA9DFF1F08B564211B
:101260000720FFF7B9FF7F210B20BDE80840FFF7FB
:10127000B3BF00BF10B500217B20FFF7ADFF0024F6
:10128000E0B2FFF779FC013402200CF067FD802CFE
:10129000F6D110BD30B58DB06D460024E1B23448B2
:1012A0000AF01CF901340C2C45F8040BF6D1314B33
:1012B0000A9A1B889A4216DA009A934213DD029A20
:1012C000934210DD049A93420DDD2B4A2B4B11887B
:1012D0001B882B4A0B4412685B10934238DB294A67
:1012E0001268934201DB0DB030BD274B00241C7007
:1012F000FFF7C0FF21460D200CF0F4FC32200CF06B
:101300002DFD01210D200CF0EDFC32200CF026FD0E
:1013100021460D200CF0E6FC32200CF01FFD0121CF
:101320000D200CF0DFFC32200CF018FD21460D20C2
:101330000CF0D8FC32200CF011FD0D2001210CF036
:10134000D1FC4FF42F700DB0BDE830400CF006BD5D
:101350000D4B002101240D201C700CF0C3FC322029
:101360000CF0FCFC0D2021460CF0BCFC3220EAE71E
:10137000149EFF1FFC9EFF1FB89DFF1F309EFF1F86
:10138000CC9DFF1F089FFF1FA49DFF1F294A2A4BCA
:1013900010881B68294A2A491288834270B52DDBC0
:1013A0009342A8BF134698420B60C8BF002327DDB5
:1013B000101AB0F5804FAABF9B03C3EB83330130F3
:1013C00093FBF0F0FFF78CF81E4E3368C0F3C615A0
:1013D0009D42044606D01C4B1B882BBB1B4B1B8815
:1013E000F3B935601A4D2B689C4206D0164B1B880A
:1013F0005A1F032A0BD92C6070BD70BD03460860CC
:101400009A42D4BFC0EB0203C0EB0303D0E7114AFA
:10141000D05C04F07F012030FFF7DEFE2C6070BD51
:101420002846FFF7CDFBDCE70A4A2946D05CFFF7E8
:10143000D3FED3E71A9EFF1FB89EFF1FF49EFF1F27
:10144000E09EFF1FD89DFF1F9C9EFF1F169EFF1F43
:10145000A09DFF1FA88CFF1F2DE9F0417B4C7C4D08
:1014600020680FF0F3FA7B490FF044FB064610208A
:101470000CF066FE0FF0EAFA77490FF03BFB3146BD
:101480000FF030FA0FF012FD2B882060002B3FD0B8
:10149000724F3A8890423BDB01467148067836B974
:1014A0004FF0010E042B80F800E000F0B380012B18
:1014B0006AD0022B00F0BC80032B36D1694B1B880D
:1014C000092B32D023683C88674AA342128853DB39
:1014D0009342D4BFC4EB0303C4EB0203141B7E2C62
:1014E000DFF88881D5BFC3EB8313C3EBC3135B0065
:1014F000013493FBF4F4D8F800300134A34203D054
:1015000021464A20FFF768FEC8F80040BDE8F08198
:10151000534A117849B10024012B147016D0022BC4
:101520001FD0032B03D0042B28D0BDE8F0814D4BF6
:101530001B88092BF9D04D4D2B68002BF5D0214687
:101540004A20FFF749FE2C60BDE8F081474D2A682C
:10155000002AEAD018462146FFF73EFE2C60BDE87F
:10156000F081424D2B68002BDFD021460420FFF78D
:1015700033FE2C60BDE8F0810023AFE72146402018
:10158000BDE8F041FFF728BE374B1B888B42D4BF24
:10159000C2EB0306C2EB01069A1ADFF8D0807E2A5E
:1015A000D8BFC6EB8616D8F80030C6BFC6EBC61645
:1015B0000132760096FBF2F60136B34203D0314693
:1015C0000120FFF709FE2B88C8F80060022B7FF48A
:1015D00073AF23683E88244AB34212882CDA002372
:1015E000961B7E2EDFF88480D5BFC3EB8313C3EB3D
:1015F000C3135B00013693FBF6F6D8F800300136D2
:10160000B34220D031460420FFF7E6FD2B88C8F80E
:10161000006051E77F214020FFF7DEFD2B88012B82
:10162000D4D121683A88104B91421B88B4DBADE7D6
:101630000D4A236812883E889A42D4BFC6EB020343
:10164000C6EB0303CCE70223E1E700BFC09DFF1F09
:10165000C89DFF1F9A99193FCDCCCC3E8E9DFF1F90
:10166000E49EFF1F9C9EFF1F529EFF1F2C9EFF1F8C
:1016700038B5114A114B14881B68114AA3421288CD
:1016800013DA0023141B0F4D7F2CCABFDB01C3EB01
:10169000C313013493FBF4F42B68A34203D0214617
:1016A0000520FFF799FD2C6038BD9342D4BFC4EBF1
:1016B0000303C4EB0203E5E7E89DFF1F689DFF1FDE
:1016C000D49EFF1FF09EFF1F10B5174B1B78DBB198
:1016D00015200BF0DBFC154B1860154A12887AB107
:1016E00014491B68098899420ADC134C23781BB9FA
:1016F000022A13D001232370BDE81040FFF7B8BFC2
:101700000D4B1B7833B910BD11200CF019FD074BA0
:101710001860E2E7BDE81040FFF780BD7F2141205F
:10172000FFF75AFDE6E700BF1C9EFF1F689DFF1FE5
:10173000249EFF1FE89DFF1FEA9DFF1F38B5054649
:1017400042F090000C460CF069FC28460CF066FC58
:10175000E0B2BDE838400CF061BC00BF70B50F4D81
:101760002B78013B1B0203F47063044643F41043DF
:1017700000040A0600F4FE0043F00903034302F0EC
:10178000FE4018430E460DF0ADFA2A68013A314684
:101790002046D2B2BDE87040FFF7D0BF009EFF1FC9
:1017A00008B50BF00FFD084809F030FE00230121B9
:1017B0004FF07E5205480AF021F804210448BDE8A4
:1017C00008400BF031B800BF149EFF1F749EFF1F2E
:1017D0000C9FFF1F00B5244B1A7883B0012105230D
:1017E00002B3002201910093114620480AF0B8F993
:1017F0001F4B1A7802B305230122019200930022A5
:101800000A211A480AF0ACF91A4B1A7802BB0523D0
:10181000012101910093142114480AF023FA03B026
:101820005DF804FB01910093114610480AF01AFA82
:101830000F4B1A78002ADED1052301210191009374
:101840000A210A480AF00EFA0A4B1A78002ADED05A
:1018500005230122019200930022142103480AF07B
:101860007FF903B05DF804FBDD9EFF1F0C9FFF1F97
:10187000389FFF1F399FFF1F2DE9F04FC54D2B7873
:10188000A3F10A02022A83B040F22281C24EA3F1E0
:101890001402022A3CD8DFF83083C04AD8F800E0AE
:1018A0001268BF499645D1F8009080F20E82C2EBD3
:1018B000090CBCF15A0F4FF00004BA4F40F31282EA
:1018C000D7F800A05B2052450CF1010100FB04F4A5
:1018D00094FBF1F404F11C0440F3E882002292FB33
:1018E000F1F11C31A14200F0158209B20023262239
:1018F000AD480AF02BFF21B201232622AA480AF0A4
:1019000025FFA9480BF04AF9D8F800202B783A6057
:10191000A3F11E02022A00F28B80A44FDFF8ACA2D2
:101920003968DAF80030DFF8A8929942D9F8002037
:1019300080F25A81D01A5A284FF00004DFF89482BE
:1019400040F35E81D8F800104FF05B0E8B420EFB27
:1019500004F400F1010E94FBFEF404F11C0400F306
:10196000B9829142A8BF1146C3EB010C5B2101FB78
:101970000CF191FBFEF11C31A14200F0548109B23F
:101980000023262288480AF0E1FE21B20123262204
:1019900085480AF0DBFEDAF80030DFF83CA2D9F81F
:1019A0000020DAF8001099424FF0010CA2EB03007E
:1019B000C0F244819142D4BFC3EB0104C3EB0204E3
:1019C0005A28DFF8189240F34081D9F800B000F1AE
:1019D000010E5B454FF05B0000FB04F494FBFEF44A
:1019E00004F11C0400F378825A45A8BF5A46D21A63
:1019F0005B2000FB02F090FBFEF01C30A04200F0E8
:101A0000398101B20023262267480AF09FFE21B2E5
:101A10000123262264480AF099FE63480BF0BEF8C1
:101A2000DAF800103A682B78C8F80020C9F80010DE
:101A3000A3F12802022A42D8DFF8A4815C4AD8F830
:101A400000E012685B499645D1F800C080F21A8127
:101A5000C2EB0C015A294FF00004574F40F31E818E
:101A600038684FF05B09824201F1010109FB04F47F
:101A700094FBF1F404F11C0400F316828445A8BF22
:101A80008446C2EB0C0C5B2000FB0CF090FBF1F1E8
:101A90001C31A14200F0158109B2002326224248E0
:101AA0000AF054FE21B2012326223F480AF04EFEDE
:101AB0003D480BF073F8D8F800202B783A603C3B97
:101AC000012B40F23A810023337003B0BDE8F08F60
:101AD0003A4ADFF810811668D8F800E0384AB6456F
:101AE000126834DA911B5A294FF00004354F38DD63
:101AF00038684FF05B0C864201F101010CFB04F4E5
:101B000094FBF1F404F11C0400F3E8819042A8BFB7
:101B10001046861B5B2000FB06F090FBF1F11C31A8
:101B2000A14230D009B2002326221F481A4E0AF0E3
:101B30000DFE21B2012326221B480AF007FE1A4897
:101B40000BF02CF8D8F800202B783A609FE6911B18
:101B50009645D4BFC6EB0E04C6EB02045A29194FB2
:101B6000C6DCD7F800C05A20664500FB04F494FB9D
:101B7000F1F404F11C0440F3BC81002292FBF1F16A
:101B80001C31A142CED1044E3278002A40F0D380DD
:101B90007246DAE7109EFF1F679DFF1F688AFF1FCE
:101BA000E48DFF1F609EFF1F0C9FFF1FCC9DFF1F3A
:101BB000FC8DFF1F5C8AFF1F809DFF1F3C9EFF1F47
:101BC000588AFF1FD89EFF1F689DFF1FE88DFF1FCB
:101BD0003C8BFF1FD49DFF1F089FFF1F3C9FFF1FD3
:101BE000C09DFF1FB89EFF1FD01A9142D4BFC3EB08
:101BF0000104C3EB02045A28DFF824833FF7A2AEA6
:101C0000D8F800E05A21734501FB04F494FBF0F48A
:101C100004F11C0440F36481002191FBF0F11C31BC
:101C2000A1427FF4ACAE3478002C77D1DFF8F4A277
:101C3000DAF800109942A446BFF6BCAE5A284FF01D
:101C40000004DFF8E4923FF7C0AED9F800E04FF0AF
:101C50005A0B73450BFB04F494FBF0F404F11C04E1
:101C600040F319814FF0000B9BFBF0F01C30A042B9
:101C70007FF4C7AE3378002B56D1BCF1000F3FF490
:101C8000D1AECAE6C2EB0C01E645D4BFC2EB0E04EE
:101C9000C2EB0C045A299B4F3FF7E2AED7F80090F5
:101CA0005A204A4500FB04F494FBF1F404F11C04AF
:101CB00040F30781002292FBF1F11C31A1427FF435
:101CC000EBAE327872BB7246F8E6C2EB090CCE4539
:101CD000D4BFC2EB0E04C2EB0904BCF15A0F8A4F09
:101CE0003FF7EEAD39685A208A4200FB04F494FBBA
:101CF000FCF404F11C0400F3E2804945A8BF494606
:101D0000891A5A2000FB01F090FBFCF11C31A14222
:101D10007FF4EBAD32781AB97246F8E509B235E6D0
:101D200009B2E9E509B2BEE601B2012326227748ED
:101D30000AF00CFD71E609B2FCE6262200248DE8CB
:101D4000140076231C217148714D724F09F03AFF3F
:101D50001DE08242D4BFC3EB0201C3EB0001D31AE2
:101D60004FF05A0E73454FF05B00CABF41430EFB64
:101D700001F1013391FBF3F303F11C0101231C4436
:101D8000262209B261480AF0E1FC0C2C09D0E1B22C
:101D9000614809F0A3FB2B683A688342D9DD002132
:101DA000DDE7DFF888815D4C01200CF0C9F9D8F837
:101DB00000C023683A682968CCEB030E8B1A9E4555
:101DC000CCEB00005BDD03FB00000EF1010390FB98
:101DD000F3F3134499424EDC9A42D4BFC1EB0203A1
:101DE000C1EB0303521A5A2ACABF5B215A2101329E
:101DF00001FB03F393FBF2F202F11C0109B2012390
:101E0000262242480AF0A2FC00200CF099F9D8F8EA
:101E100000E03A68296824688B1ACEEB04049C42DF
:101E2000CEEB000031DD03FB0000631C90FBF3F3FD
:101E30001344994221DC9A42D4BFC1EB0203C1EBA7
:101E40000303521A5A2ACABF5B215A21013201FBED
:101E500003F393FBF2F202F11C0109B201232622E3
:101E60002A480AF073FC29480AF098FE00233370D0
:101E700003B0BDE8F08F0023B4E70023E1E703FBE4
:101E800000F393FBFEF31344A4E703FB00F393FB7F
:101E9000F4F31344CDE77245D4BFC3EB0203C3EBA5
:101EA0000E030BFB03FBDFE69446EAE5D145D4BF06
:101EB000C2EB0902C2EB0A0200FB02F20FE5114677
:101EC0001EE7CC45D4BFC2EB0C02C2EB090200FBFB
:101ED00002F2F0E6194647E51A4688E5304618E66C
:101EE0007245D4BFC3EB020EC3EB0E0E01FB0EF125
:101EF00093E66245D4BFC6EB0202C6EB0C0200FBC0
:101F000002F23BE6809DFF1F609EFF1F0C9FFF1F9C
:101F1000F48DFF1F408CFF1F149EFF1F5C8CFF1F62
:101F2000D49DFF1F089FFF1F3C9FFF1F608AFF1F5C
:101F300008B581B217480AF0E1F9022115480AF004
:101F4000D7F921225A2113480AF0CEF9124B114831
:101F500019880DF017FC0F480DF0C4FB0F4B1978D2
:101F600091B90C480AF0CAF901210A480AF0C0F9EF
:101F70003322742107480AF0B7F9012208490548BD
:101F8000BDE808400DF09ABB012102480AF0B6F9FD
:101F9000EAE700BF0C9FFF1F649EFF1FEA9EFF1F22
:101FA0001836010010B5154C012120460AF0A6F99B
:101FB000204601210AF09CF9204600220F210AF058
:101FC00093F9204602220E490DF078FB2046342278
:101FD00055210AF089F9204602220A490DF06EFBCC
:101FE0002046052208490DF069FB20460DF07AFBDA
:101FF0002046BDE810400AF0D1BD00BF0C9FFF1F76
:102000000036010004360100083601002DE9F84FC2
:102010000C200BF007F80C200BF0D2FDDD4914204A
:102020000BF0DEFD022103200BF070FE02210420E4
:102030000BF06CFE022105200BF068FE0221062049
:102040000BF064FE01210A200BF060FE0121092043
:102050000BF05CFE01210D200BF058FE0121282021
:102060000BF054FE012114200BF050FE02210B2036
:102070000BF04CFE01210C200BF048FE00210C203F
:102080000BF030FE0020FEF745FD172840F25C8281
:1020900004200BF02DFE002800F050820020FEF7F7
:1020A00039FD1F2800F08C821F210020FEF726FD3D
:1020B0000C210E20FEF722FD01211020FEF71EFD4F
:1020C00002211220FEF71AFD00211420FEF716FD52
:1020D00000211620FEF712FD02211820FEF70EFD4A
:1020E00001211A20FEF70AFD02211C20FEF706FD41
:1020F00004211E20FEF702FD14212020FEF7FEFC25
:1021000001212620FEF7FAFC03212820FEF7F6FC29
:1021100004212C20FEF7F2FC0F212E20FEF7EEFC0E
:1021200000213020FEF7EAFC0C213220FEF7E6FC0D
:1021300000213420FEF7E2FC00213620FEF7DEFC11
:1021400000213820FEF7DAFC00213A20FEF7D6FC09
:1021500000213C20FEF7D2FC00213E20FEF7CEFC01
:1021600000214020FEF7CAFC00214220FEF7C6FCF9
:102170001F214420FEF7C2FC13214620FEF7BEFCBF
:102180000E214820FEF7BAFC11214A20FEF7B6FCCA
:102190000A214C20FEF7B2FC00214E20FEF7AEFCD7
:1021A00006215020FEF7AAFC02215220FEF7A6FCD1
:1021B0000F215420FEF7A2FC00215620FEF79EFCC2
:1021C0000220FEF7A7FC744B744C18800420FEF725
:1021D000A1FC734BDFF8408218800620FEF79AFCC2
:1021E000704BDFF838A218800820FEF793FC6E4B86
:1021F0006E4E18800A20FEF78DFC6D4B6D4D1880D9
:102200000C20FEF787FC6C4B18800E20FEF782FC3A
:102210006A4B18801020FEF77DFC20801220FEF70C
:1022200079FC674B18801420FEF774FC654B18800E
:102230001620FEF76FFC644B18801820FEF76AFC2E
:10224000624B18801A20FEF765FC614B18801C2039
:10225000FEF760FC5F4B18801E20FEF75BFC5E4BB8
:1022600018802020FEF756FC5C4B18802220FEF7D9
:1022700051FC5B4B18802420FEF74CFC594B188016
:102280002620FEF747FC584B81462820A3F80090F3
:10229000FEF740FC554B18802A20FEF73BFC544BC0
:1022A00007462C201F80FEF735FC524B18802E204D
:1022B000FEF730FC504B18803020FEF72BFC4F4BC4
:1022C00018803220FEF726FC4D4B18803420FEF794
:1022D00021FCA8F800003620FEF71CFCA8F802003C
:1022E0003820FEF717FCA8F804003A20FEF712FC8D
:1022F000A8F806003C20FEF70DFCA8F808003E20D8
:10230000FEF708FCA8F80A004020FEF703FCA8F836
:102310000C004220FEF7FEFB3A4B80464420A3F817
:102320000080FEF7F7FB384BA0F1180246201A6038
:10233000FEF7F0FBA0F118034820CAF80030FEF7C2
:10234000E9FBA0F118034A20CAF80430FEF7E2FBCB
:10235000A0F118034C20CAF80830FEF7DBFBA0F10F
:1023600018034E20CAF80C30FEF7D4FB274B188018
:102370005020FEF7CFFB264B18805220FEF7CAFBF9
:10238000244B18805420FEF7C5FB30805620FEF702
:10239000C1FB45E0001B37461A9EFF1F649EFF1FCE
:1023A000F49EFF1FE89DFF1FD49EFF1FBA8CFF1FE6
:1023B000309EFF1FF29DFF1FB89DFF1FA89DFF1FAE
:1023C0009C9EFF1F169EFF1F5C9DFF1F249EFF1FEC
:1023D000D09DFF1FC89DFF1FBC9DFF1FE69EFF1FD6
:1023E0008E9DFF1F529EFF1F709EFF1FBE9EFF1FF0
:1023F000FC9EFF1FA49EFF1FC49EFF1FA69DFF1FE4
:10240000D69EFF1FF69EFF1F048BFF1FC69DFF1F5A
:10241000B88CFF1F948AFF1F709DFF1F448CFF1F05
:10242000B34ADFF838E3B349D2F800A0B24BB34A5D
:10243000DEF800B0D1F800C0D3F800E01168B04A6F
:10244000B04B85F80090CCEB0B0CCEEB0A0E82FB68
:102450000CBAD3F80090AC4BE2444FEAEC7CCCEBE6
:10246000AA1CDFF8FCA21880A84BCAF800C082FBA7
:102470000EAC1868A64BF4444FEAEE7ECEEBAC1ED1
:10248000DFF8E0C21B68CCF800E0C1EB090982FB71
:1024900009CEC01ACE44DFF8D0C29E4B9E491B68BD
:1024A00009684FEAE979C9EBAE1ECCF800E082FB7F
:1024B00000EC8444C017C1EB030EC0EBAC10DFF896
:1024C000ACC282FB0E92CCF8000072449348DFF855
:1024D000A0C24FEAEE7E5FFA88F8CEEBA21202604D
:1024E00008F002098E4A8CF8009008F0040C82F87B
:1024F00000C0DFF880E28B488B4A08F008088EF8AD
:10250000008000681268C91A121A9142A7EB0303EF
:102510000EDD02FB0333013193FBF1F30344834AE5
:10252000834813605A2109F015F8002855D1FEE7B9
:1025300002FB03F292FBF1F30344F0E706200BF0F9
:10254000D7FB00287FF4AAAD1F210020FEF7D6FAA2
:102550004FF4AF610220FEF7D1FA04204FF47A6104
:10256000FEF7CCFA0B200BF0C3FB002800F0B5807F
:1025700040F628210620FEF7C1FA40F6E441082083
:10258000FEF7BCFA4FF4AF610A20FEF7B7FA40F647
:10259000FC010C20FEF7B2FA4FF496612220FEF700
:1025A000ADFA4FF416612420FEF7A8FA7D212A2007
:1025B000FEF7A4FA0020FEF7ADFA1F287FF474ADF1
:1025C00004200BF095FB00287FF4FAAD06200BF0F9
:1025D0008FFB00283FF468ADF2E5564A5648126872
:1025E0000023012109F028F9FEF7D6F90B200BF0A2
:1025F0007FFB524B011E0CBF012200221A7002D138
:1026000011200BF083FBDFF83C814D4F0023C8F80D
:1026100000303B604FF001090F200BF091FD3B684B
:10262000DFF81CA103440E203B600AF02FFDD8F810
:10263000003009F0010103440D20C8F8003009F111
:1026400001090BF04FFBFA200BF088FBB9F1050FE5
:10265000E2D1DAF80030D8F80020318839483A4E13
:10266000002BB8BF0333002AB8BF03329B103B6076
:102670009210364F02605A1A0D200B44002133602D
:102680003A600BF02FFBFA200BF068FB01210D20C4
:102690000BF028FBFA200BF061FB00210D200BF062
:1026A00021FBFFF77FFC40F2DC500BF057FB284B7F
:1026B000012604201E600BF01BFB10B9254B28706F
:1026C0001E702378244A18461370FEF799FA0121E8
:1026D0000D20BDE8F84F0BF005BB4FF496610620C6
:1026E000FEF70CFA4FF4FA610820FEF707FA49E703
:1026F000E48DFF1F3C9EFF1F688AFF1FE88DFF1FB0
:10270000C94216B23C8BFF1FFA9DFF1F5C8AFF1F58
:10271000FC8DFF1F408CFF1FF48DFF1FDC9DFF1FF2
:10272000189EFF1F608AFF1F5C8CFF1F548CFF1FC9
:10273000149EFF1F4C8AFF1F749EFF1F1C9EFF1FCD
:10274000C89EFF1F6C9DFF1F409EFF1FE49DFF1F43
:10275000D09EFF1F959DFF1F399EFF1F588AFF1FA8
:10276000A89EFF1FC09EFF1FAC9EFF1F589EFF1F0D
:10277000BE9DFF1FEA9EFF1F70B5194C82B0342624
:102780000023012520460193009640230B223F2180
:1027900009F0E6F940230B222046009601953F21DF
:1027A00009F060FA2946204609F0A8FD294620468E
:1027B00009F09EFD20460F22442109F095FD0922D3
:1027C000084920460CF07AFF20460CF08BFF064BA0
:1027D00020461D7002B0BDE870400AF0DFB900BFAE
:1027E0000C9FFF1F10360100049FFF1F70B5194C8E
:1027F00082B0342600230125204601930096402311
:102800000B223F2109F0ACF940230B222046009611
:1028100001953F2109F026FA2946204609F06EFD70
:102820002946204609F064FD20460F22512109F077
:102830005BFD0522084920460CF040FF20460CF0C5
:1028400051FF2846FEF700F9204602B0BDE870406F
:102850000AF0A4B90C9FFF1F1C36010070B5194C7B
:1028600082B03426002301252046019300964023A0
:102870000B223F2109F074F940230B2220460096D9
:1028800001953F2109F0EEF92946204609F036FD71
:102890002946204609F02CFD20460F22442109F04C
:1028A00023FD0922084920460CF008FF20460CF0C1
:1028B00019FF2846FFF73CFB204602B0BDE87040F8
:1028C0000AF06CB90C9FFF1F2436010070B5194C3B
:1028D00082B0342600230125204601930096402330
:1028E0000B223F2109F03CF940230B2220460096A1
:1028F00001953F2109F0B6F92946204609F0FEFC72
:102900002946204609F0F4FC20460F22512109F007
:10291000EBFC0522084920460CF0D0FE20460CF0C6
:10292000E1FE2846FEF7AEF8204602B0BDE8704052
:102930000AF034B90C9FFF1F1C36010070B5194C0A
:1029400082B03426002301252046019300964023BF
:102950000B223F2109F004F940230B222046009668
:1029600001953F2109F07EF92946204609F0C6FC71
:102970002946204609F0BCFC20460F22512109F0CF
:10298000B3FC0522084920460CF098FE20460CF0C6
:10299000A9FE2846FEF794F8204602B0BDE8704034
:1029A0000AF0FCB80C9FFF1F1C36010010B581B265
:1029B000124C134809F0A2FC0221114809F098FCBE
:1029C000238821226BB94F210D4809F08DFC032289
:1029D0000C490B480CF072FE0948BDE810400CF0A1
:1029E00081BE5A21064809F07FFC218804480CF07A
:1029F000C9FE0348BDE810400CF074BEA69DFF1F41
:102A00000C9FFF1F3036010070B5194C82B0342680
:102A10000023012520460193009640230B223F21ED
:102A200009F09EF840230B222046009601953F2195
:102A300009F018F92946204609F060FC294620468D
:102A400009F056FC20460F22482109F04DFC0822CF
:102A5000084920460CF032FE20460CF043FE284682
:102A6000FFF7A4FF204602B0BDE870400AF096B818
:102A70000C9FFF1F3436010010B581B21748184C67
:102A800009F03CFC0221154809F032FC21224C21BE
:102A9000124809F029FC23884BB9032211490F4839
:102AA0000CF00CFE0D48BDE810400CF01BBE0222DD
:102AB0000D490A480CF002FE08480CF013FE2122D2
:102AC0006521064809F010FC218804480CF05AFEE4
:102AD0000248BDE810400CF005BE00BF0C9FFF1F70
:102AE000D09DFF1F303601004036010070B5194CF3
:102AF00082B034260023012520460193009640230E
:102B00000B223F2109F02CF840230B22204600968F
:102B100001953F2109F0A6F82946204609F0EEFB71
:102B20002946204609F0E4FB20460F22442109F003
:102B3000DBFB0922084920460CF0C0FD20460CF0C2
:102B4000D1FD2846FFF798FF204602B0BDE870404F
:102B50000AF024B80C9FFF1F4436010010B581B263
:102B6000124C134809F0CAFB0221114809F0C0FBBE
:102B7000238821226BB94F210D4809F0B5FB0322B0
:102B80000C490B480CF09AFD0948BDE810400CF0C8
:102B9000A9BD5A21064809F0A7FB218804480CF07A
:102BA000F1FD0348BDE810400CF09CBDBC9DFF1F2B
:102BB0000C9FFF1F3036010070B5194C82B03426CF
:102BC0000023012520460193009640230B223F213C
:102BD00008F0C6FF40230B222046009601953F21B6
:102BE00009F040F82946204609F088FB294620468E
:102BF00009F07EFB20460F22512109F075FB0522CA
:102C0000084920460CF05AFD20460CF06BFD284682
:102C1000FFF7A4FF204602B0BDE8704009F0BEBF38
:102C20000C9FFF1F1C36010008B581B2104809F047
:102C300065FB02210E4809F05BFB4F2121220C4865
:102C400009F052FB0B4B198849B903220A4908487D
:102C50000CF034FD0648BDE808400CF043BD0448C4
:102C60000CF090FD0248BDE808400CF03BBD00BFF1
:102C70000C9FFF1F5C9DFF1F5036010070B5194C63
:102C800082B034260023012520460193009640237C
:102C90000B223F2108F064FF40230B2220460096C0
:102CA00001953F2108F0DEFF2946204609F026FB6A
:102CB0002946204609F01CFB20460F22472109F037
:102CC00013FB0822084920460CF0F8FC20460CF0C3
:102CD00009FD2846FFF7A8FF204602B0BDE8704076
:102CE00009F05CBF0C9FFF1F5436010010B50C4665
:102CF00081B2194809F002FB0221174809F0F8FADD
:102D000021225021144809F0EFFA002C4FF0010263
:102D100014DB124910480CF0D1FC0F480CF0E2FC17
:102D20005D2121220C4809F0DFFA21460A480CF007
:102D300029FD0948BDE810400CF0D4BC08490648FC
:102D40000CF0BCFC04480CF0CDFC5D2121220248B3
:102D500009F0CAFA6142E9E70C9FFF1F60360100E3
:102D6000643601000CB42DE9F04184B00AAC06468B
:102D7000294814F8045B884609F06EFD01212648B5
:102D800009F0B6FA0121244809F0B8FA00221146E8
:102D9000214809F0A9FA30460EF0D2FE314602462B
:102DA0001D480CF08BFC1C480CF09CFC09220123F4
:102DB0008DE80C0000217F23174808F003FF0394DF
:102DC000EDB16F1EFFB2013704EB87070C25043409
:102DD00054F8046C104803942AB2002109F084FAD4
:102DE00030460EF0ADFE314602460B480CF066FC54
:102DF00009480CF077FC0935BC42ADB2E7D140463A
:102E00000121FDF7EBFD044809F0C8FE04B0BDE860
:102E1000F04102B0704700BF0C9FFF1F30B52B4D33
:102E20000FCD8DB006AC0FC495E8030044F8040B39
:102E3000232021800AF02AF940F6B833984212DCA8
:102E4000234B40F6F50219889B78ADF82510904287
:102E50008DF827300EDC1F4B1A889B78ADF829209F
:102E60008DF82B301EE01C4B1A889B78ADF825207E
:102E70008DF82730194A00EB400000EB001382FB6D
:102E80000320DB17C3EB60200DF0E0FD14490DF0CB
:102E900031FE0DF12903012203210AF0A9FA56237C
:102EA0008DF82C300F4B10481978104D104C114AEA
:102EB000114B04900192009306A8039502940F4BC6
:102EC0000622FFF74FFF0DB030BD00BFB436010042
:102ED000683601006C360100B0360100976A3E2B5F
:102EE000CDCCCC3D3289FF1F803601008C360100ED
:102EF00098360100A0360100A836010074360100A2
:102F000030B50A4B0A4D19780A4C0B480B4A0C4B4A
:102F100087B002900192009304950394094B0A48EC
:102F20000622FFF71FFF07B030BD00BF948DFF1FC3
:102F3000E8360100F4360100003701000C370100CB
:102F400018370100CC360100D836010010B586B024
:102F5000084C094809490A4A0A4B03900291019218
:102F600000930494084B09480622FF21FFF7FAFE5C
:102F700006B010BD34360100403701004C37010067
:102F80005436010054370100243701003037010066
:102F900010B586B0084C094809490A4A0A4B039003
:102FA0000291019200930494084B09480622FF21E4
:102FB000FFF7D8FE06B010BD783701008437010056
:102FC0009037010098370100443601006037010056
:102FD0006C37010000B585B008480949094A0A4B19
:102FE00003900291019200930848094B0522FF21AA
:102FF000FFF7B8FE05B05DF804FB00BFAC37010079
:10300000B8370100C0370100C83701009037010010
:10301000A437010010B581B22048214C09F06EF9A7
:1030200002211E4809F064F9212250211B4809F0B1
:103030005BF923880B2B4FF0010218DC1949174864
:103040000CF03CFB15480CF04DFB21225D21134890
:1030500009F04AF9218811480C390029B8BF4942C2
:103060000CF090FB0D48BDE810400CF03BBB0E4946
:103070000A480CF023FB09480CF034FB21225D21A7
:10308000064809F031F9218804480C390CF07AFB24
:103090000248BDE810400CF025BB00BF0C9FFF1F8D
:1030A000A89DFF1F643601006036010070B5194C01
:1030B00082B0342600230125204601930096402348
:1030C0000B223F2108F04CFD40230B2220460096A6
:1030D00001953F2108F0C6FD2946204609F00EF96A
:1030E0002946204609F004F920460F22442109F020
:1030F000FBF80922084920460CF0E0FA20460CF0C3
:10310000F1FA2846FFF786FF204602B0BDE870407E
:1031100009F044BD0C9FFF1F7436010010B581B249
:103120002048214C09F0EAF802211E4809F0E0F895
:10313000212250211B4809F0D7F82388022B4FF099
:10314000010218DC194917480CF0B8FA15480CF0C0
:10315000C9FA21225D21134809F0C6F821881148D7
:1031600003390029B8BF49420CF00CFB0D48BDE8FB
:1031700010400CF0B7BA0E490A480CF09FFA094803
:103180000CF0B0FA21225D21064809F0ADF8218843
:10319000044803390CF0F6FA0248BDE810400CF080
:1031A000A1BA00BF0C9FFF1FBE9EFF1F6436010027
:1031B0006036010070B5194C82B034260023012519
:1031C00020460193009640230B223F2108F0C8FCC3
:1031D00040230B222046009601953F2108F042FD36
:1031E0002946204609F08AF82946204609F080F849
:1031F00020460F224D2109F077F806220849204683
:103200000CF05CFA20460CF06DFA2846FFF786FFBA
:10321000204602B0BDE8704009F0C0BC0C9FFF1F03
:10322000A836010000B5324B1B78013B85B0052B59
:103230000AD8DFE803F00C21364B54032D492E4BFE
:103240005A20012208701A7005B05DF804FB0123B2
:103250002A4A194618461370FDF7C0FB284809F0A2
:103260009DFC284A284B12680192019A1A60FFF7C8
:103270001DFF05B05DF804FB0123244A1946022016
:103280001370FDF7ABFB1E4809F088FC1D4A1E4B6E
:1032900012680292029A1A60FFF78CFF05B05DF87F
:1032A00004FB01231A4A194603201370FDF796FB0D
:1032B000134809F073FC134A134B12680392039AE4
:1032C0001A60FFF7CBFA05B05DF804FB09490A4B19
:1032D0000A20012208701A7005B05DF804FB054948
:1032E000054B5020012208701A7005B05DF804FBF0
:1032F0003289FF1F109EFF1F588CFF1FB29EFF1FB9
:103300000C9FFF1F489FFF1F449EFF1FB09DFF1F84
:10331000F19DFF1F08B581B20D4808F0EFFF0221B3
:103320000B4808F0E5FF21224F21094808F0DCFF97
:10333000084B1B88032243B9074905480CF0BEF926
:103340000348BDE808400CF0CDB90449F5E700BFDB
:103350000C9FFF1FC69DFF1FD4370100D03701000F
:1033600070B5194C82B03426002301252046019304
:10337000009640230B223F2108F0F2FB40230B2252
:103380002046009601953F2108F06CFC2946204616
:1033900008F0B4FF2946204608F0AAFF20460F2275
:1033A000442108F0A1FF0922084920460CF086F9C3
:1033B00020460CF097F92846FFF7ACFF204602B0F4
:1033C000BDE8704009F0EABB0C9FFF1FD837010031
:1033D00000B5444B1B78013B87B0052B16D8DFE8BE
:1033E00003F0182D42576C0301233F4A194606206B
:1033F0001370FDF7F3FA3D4809F0D0FB3C4A3D4B12
:1034000012680592059A1A60FFF7AAFF07B05DF8E7
:1034100004FB0123384A194618461370FDF7DEFAFB
:10342000324809F0BBFB324A324B12680092009AD4
:103430001A60FFF7A1F907B05DF804FB01232F4ADA
:10344000194602201370FDF7C9FA284809F0A6FBB7
:10345000274A284B12680192019A1A60FFF78CF9EB
:1034600007B05DF804FB254B0222012103201A70EE
:10347000FDF7B4FA1D4809F091FB1D4A1D4B126877
:103480000292029A1A60FFF777F907B05DF804FB21
:103490001A4B0322012104201A70FDF79FFA1348EA
:1034A00009F07CFB124A134B12680392039A1A60CC
:1034B000FFF762F907B05DF804FB104B042201210D
:1034C00005201A70FDF78AFA084809F067FB084AD8
:1034D000084B12680492049A1A60FFF74DF907B07E
:1034E0005DF804FB948DFF1F5C9EFF1F0C9FFF1F68
:1034F000489FFF1F449EFF1F499EFF1FEC9EFF1F1A
:1035000008B581B20D4808F0F9FE02210B4808F019
:10351000EFFE21224F21094808F0E6FE084B1B88E8
:103520004BB90849032205480CF0C8F80348BDE828
:1035300008400CF0D7B802220349F4E70C9FFF1FA4
:10354000169EFF1F30360100E437010070B5194C9C
:1035500082B03426002301252046019300964023A3
:103560000B223F2108F0FCFA40230B222046009654
:1035700001953F2108F076FB2946204608F0BEFE63
:103580002946204608F0B4FE20460F22442108F0C8
:10359000ABFE0922084920460CF090F820460CF0BA
:1035A000A1F82846FFF7ACFF204602B0BDE8704006
:1035B00009F0F4BA0C9FFF1F5437010008B581B21F
:1035C0000D4808F09BFE02210B4808F091FE2122D5
:1035D0004F21094808F088FE084B1B88032243B19D
:1035E000074905480CF06AF80348BDE808400CF0AC
:1035F00079B80449F5E700BF0C9FFF1FFA9DFF1F34
:10360000EC370100E837010070B5194C82B0342660
:103610000023012520460193009640230B223F21E1
:1036200008F09EFA40230B222046009601953F2188
:1036300008F018FB2946204608F060FE294620467F
:1036400008F056FE20460F22442108F04DFE0922C4
:10365000084920460CF032F820460CF043F8284682
:10366000FFF7ACFF204602B0BDE8704009F096BA03
:103670000C9FFF1FAC37010000B53A4B1B78013B94
:1036800087B0042B16D8DFE803F0182D425703004B
:103690000123354A194605201370FDF79FF9334879
:1036A00009F07CFA324A334B12680592059A1A6087
:1036B000FFF7AAFF07B05DF804FB01232E4A194665
:1036C00018461370FDF78AF9284809F067FA284A66
:1036D000284B12680192019A1A60FFF76DFA07B041
:1036E0005DF804FB0123254A194602201370FDF7FB
:1036F00075F91E4809F052FA1D4A1E4B12680292D3
:10370000029A1A60FFF772F807B05DF804FB012314
:103710001B4A194603201370FDF760F9134809F09E
:103720003DFA134A134B12680392039A1A60FFF78B
:10373000CDF807B05DF804FB0123124A19460420B6
:103740001370FDF74BF9094809F028FA084A094BAC
:1037500012680492049A1A60FFF7F0F807B05DF857
:1037600004FB00BF488AFF1FE99EFF1F0C9FFF1F3D
:10377000489FFF1F449EFF1F389EFF1F049EFF1F90
:10378000E09DFF1FE89EFF1F08B581B2154808F0B5
:10379000B5FD0221134808F0ABFD4F21212211484D
:1037A00008F0A2FD104B198849B9104903220D48B1
:1037B0000BF084FF0B48BDE808400BF093BF0948AD
:1037C0000BF0E0FF07480BF08DFF28226921054828
:1037D00008F08AFD0121034808F08AFD022204490D
:1037E000E5E700BF0C9FFF1FC49EFF1F303601009E
:1037F000F037010070B5194C82B034260023012542
:1038000020460193009640230B223F2108F0A8F99F
:1038100040230B222046009601953F2108F022FA12
:103820002946204608F06AFD2946204608F060FD3A
:1038300020460F22452108F057FD0922084920465D
:103840000BF03CFF20460BF04DFF2846FFF79CFF96
:10385000204602B0BDE8704009F0A0B90C9FFF1FE0
:103860004037010008B581B2154808F047FD022134
:10387000134808F03DFD4F212122114808F034FD86
:10388000104B198849B9104903220D480BF016FF57
:103890000B48BDE808400BF025BF09480BF072FF4C
:1038A00007480BF01FFF28226921054808F01CFD7E
:1038B0000121034808F01CFD02220449E5E700BF8E
:1038C0000C9FFF1FE69EFF1F30360100F0370100FE
:1038D00070B5194C82B0342600230125204601938F
:1038E000009640230B223F2108F03AF940230B2297
:1038F0002046009601953F2108F0B4F9294620465C
:1039000008F0FCFC2946204608F0F2FC20460F2275
:10391000472108F0E9FC0822084920460BF0CEFEBA
:1039200020460BF0DFFE2846FFF79CFF204602B042
:10393000BDE8704009F032B90C9FFF1F84370100C9
:1039400030B5544883B008F087FF0121514808F092
:10395000CFFC01214F4808F0D1FC022219214D482B
:1039600008F0C2FC0B224C494A480BF0A7FE49481C
:103970000BF0B8FE14220021464808F0B5FC0322E3
:10398000464944480BF09AFE424801240BF0AAFE37
:1039900011228DE81400782319213E4808F012F90D
:1039A000132519231946009512223A48019408F06C
:1039B00009F978231946009512223648019408F037
:1039C00001F91D228DE8140078231921314808F0EF
:1039D000F9F81C251923194600951B222D4801943E
:1039E00008F0F0F87823194600951B222948019425
:1039F00008F0E8F823220021264808F075FC03228D
:103A0000274924480BF05AFE22480BF06BFE28256C
:103A10001923194624221F480194009508F0D2F872
:103A2000782319462422019400951A4808F0CAF810
:103A30001C4A1D4B11681B681C4A5B1A5C2B1288C0
:103A40001DDC511A5C2202FB01F292FBF3F31B33E3
:103A5000174A1048136001241BB21A2219468DE838
:103A60001400142208F0AEF8124B20461C70FCF72C
:103A7000CBFF084803B0BDE8304009F08FB8521AB8
:103A800002EB4202C2EB4212234492FBF3F31B33DC
:103A9000DEE700BF0C9FFF1FF43701000038010074
:103AA00004380100F48DFF1F408CFF1FFC9EFF1F98
:103AB000609DFF1F949EFF1FF0B58548854E864D83
:103AC00083B008F0C9FE0121814808F011FC0121F2
:103AD0007F4808F013FC022219217D4808F004FCFD
:103AE00010227E497A480BF0E9FD79480BF0FAFD87
:103AF00014220021764808F0F7FB03227849744825
:103B00000BF0DCFD724801240BF0ECFD11228DE876
:103B10001400782319216E4808F054F8132719234C
:103B20001946009712226A48019408F04BF878234E
:103B30001946009712226648019408F043F81D22A6
:103B40008DE8140078231921614808F03BF81C2700
:103B50001923194600971B225D48019408F032F89A
:103B60007823194600971B225948019408F02AF837
:103B700023220021564808F0B7FB03225949544834
:103B80000BF09CFD52480BF0ADFD28271923194678
:103B9000009724224E48019408F014F8782319461F
:103BA000009724224A48019408F00CF832220021A0
:103BB000474808F099FB03224B4945480BF07EFD2E
:103BC00043480BF08FFD2F228DE814007823192134
:103BD0003F4807F0F7FF3127192319460097302295
:103BE0003B48019407F0EEFF7823194600973022F6
:103BF0003748019407F0E6FF3C228DE81400782353
:103C00001921334807F0DEFF3B27192319463A22D2
:103C10002F480194009707F0D5FF782319463A22E0
:103C2000019400972A4807F0CDFF31682B682F4A8E
:103C30005B1A5C2B128839DD521A02EB4202C2EB8E
:103C40004212234492FBF3F31B33294A20481360AA
:103C500001241BB21A2219468DE81400142207F021
:103C6000B1FF31682B682348234A04705B1A5C2B30
:103C7000128823DC511A5C2202FB01F292FBF3F35F
:103C80001B331E4A1248136001241BB23922194605
:103C90008DE81400322207F095FF2046FCF7B4FEB1
:103CA0000B4803B0BDE8F04008F078BF511A5C2221
:103CB00002FB01F292FBF3F31B33C6E7521A02EB4D
:103CC0004202C2EB4212234492FBF3F31B33D8E7C8
:103CD0000C9FFF1FFC8DFF1F5C8AFF1F083801002F
:103CE00000380100043801001C3801008E9DFF1FC0
:103CF000609DFF1F949EFF1F529EFF1FB49EFF1FDB
:103D0000F0B58548854E864D83B008F0A5FD0121AC
:103D1000814808F0EDFA01217F4808F0EFFA02220D
:103D200019217D4808F0E0FA0A227E497A480BF012
:103D3000C5FC79480BF0D6FC14220021764808F027
:103D4000D3FA0322784974480BF0B8FC7248012476
:103D50000BF0C8FC11228DE81400782319216E485D
:103D600007F030FF132719231946009712226A48DB
:103D7000019407F027FF782319460097122266481E
:103D8000019407F01FFF1D228DE8140078231921EC
:103D9000614807F017FF1C271923194600971B22BB
:103DA0005D48019407F00EFF7823194600971B2207
:103DB0005948019407F006FF23220021564808F0D5
:103DC00093FA0322594954480BF078FC52480BF0FF
:103DD00089FC282719231946009724224E4801946C
:103DE00007F0F0FE78231946009724224A480194F0
:103DF00007F0E8FE32220021474808F075FA032256
:103E00004B4945480BF05AFC43480BF06BFC2F2202
:103E10008DE81400782319213F4807F0D3FE31279D
:103E200019231946009730223B48019407F0CAFE37
:103E300078231946009730223748019407F0C2FED4
:103E40003C228DE8140078231921334807F0BAFE8C
:103E50003B27192319463A222F480194009707F06F
:103E6000B1FE782319463A22019400972A4807F0B8
:103E7000A9FE31682B682F4A5B1A5C2B128839DD4A
:103E8000521A02EB4202C2EB4212234492FBF3F3BA
:103E90001B33294A2048136001241BB21A221946F9
:103EA0008DE81400142207F08DFE31682B6823483A
:103EB000234A04705B1A5C2B128823DC511A5C22A3
:103EC00002FB01F292FBF3F31B331E4A124813600C
:103ED00001241BB2392219468DE81400322207F062
:103EE00071FE2046FCF790FD0B4803B0BDE8F040A2
:103EF00008F054BE511A5C2202FB01F292FBF3F36C
:103F00001B33C6E7521A02EB4202C2EB42122344B1
:103F100092FBF3F31B33D8E70C9FFF1F688AFF1F48
:103F2000E48DFF1F20380100003801000438010033
:103F30001C380100E89DFF1F609DFF1F949EFF1F1E
:103F4000D49EFF1FB49EFF1FF0B58548854E864D59
:103F500083B008F081FC0121814808F0C9F90121F2
:103F60007F4808F0CBF9022219217D4808F0BCF9FE
:103F700006227E497A480BF0A1FB79480BF0B2FB90
:103F800014220021764808F0AFF9032278497448DA
:103F90000BF094FB724801240BF0A4FB11228DE876
:103FA0001400782319216E4807F00CFE13271923FB
:103FB0001946009712226A48019407F003FE7823FD
:103FC0001946009712226648019407F0FBFD1D2256
:103FD0008DE8140078231921614807F0F3FD1C27B0
:103FE0001923194600971B225D48019407F0EAFD4A
:103FF0007823194600971B225948019407F0E2FDE7
:1040000023220021564808F06FF9032259495448E9
:104010000BF054FB52480BF065FB28271923194677
:10402000009724224E48019407F0CCFD78231946CE
:10403000009724224A48019407F0C4FD322200214F
:10404000474808F051F903224B4945480BF036FB2D
:1040500043480BF047FB2F228DE8140078231921E9
:104060003F4807F0AFFD312719231946009730224A
:104070003B48019407F0A6FD7823194600973022AB
:104080003748019407F09EFD3C228DE81400782308
:104090001921334807F096FD3B27192319463A2288
:1040A0002F480194009707F08DFD782319463A2296
:1040B000019400972A4807F085FD31682B682F4A44
:1040C0005B1A5C2B128839DD521A02EB4202C2EBFA
:1040D0004212234492FBF3F31B33294A2048136016
:1040E00001241BB21A2219468DE81400142207F08D
:1040F00069FD31682B682348234A04705B1A5C2BE6
:10410000128823DC511A5C2202FB01F292FBF3F3CA
:104110001B331E4A1248136001241BB23922194670
:104120008DE81400322207F04DFD2046FCF76CFCB0
:104130000B4803B0BDE8F04008F030BD511A5C22D6
:1041400002FB01F292FBF3F31B33C6E7521A02EBB8
:104150004202C2EB4212234492FBF3F31B33D8E733
:104160000C9FFF1F3C9EFF1F588AFF1F2C38010029
:1041700000380100043801001C3801001A9EFF1F9E
:10418000609DFF1F949EFF1FF49EFF1FB49EFF1FA4
:10419000F0B58548854E864D83B008F05DFB012162
:1041A000814808F0A5F801217F4808F0A7F802220D
:1041B00019217D4808F098F80A227E497A480BF0C8
:1041C0007DFA79480BF08EFA14220021764808F027
:1041D0008BF80322784974480BF070FA7248012476
:1041E0000BF080FA11228DE81400782319216E4813
:1041F00007F0E8FC132719231946009712226A4892
:10420000019407F0DFFC78231946009712226648D4
:10421000019407F0D7FC1D228DE8140078231921A2
:10422000614807F0CFFC1C271923194600971B2271
:104230005D48019407F0C6FC7823194600971B22BD
:104240005948019407F0BEFC23220021564808F08B
:104250004BF80322594954480BF030FA52480BF0FE
:1042600041FA282719231946009724224E48019421
:1042700007F0A8FC78231946009724224A480194A5
:1042800007F0A0FC32220021474808F02DF8032255
:104290004B4945480BF012FA43480BF023FA2F2202
:1042A0008DE81400782319213F4807F08BFC312753
:1042B00019231946009730223B48019407F082FCED
:1042C00078231946009730223748019407F07AFC8A
:1042D0003C228DE8140078231921334807F072FC42
:1042E0003B27192319463A222F480194009707F0DB
:1042F00069FC782319463A22019400972A4807F06E
:1043000061FC31682B682F4A5B1A5C2B128839DDFF
:10431000521A02EB4202C2EB4212234492FBF3F325
:104320001B33294A2048136001241BB21A22194664
:104330008DE81400142207F045FC31682B682348EF
:10434000234A04705B1A5C2B128823DC511A5C220E
:1043500002FB01F292FBF3F31B331E4A1248136077
:1043600001241BB2392219468DE81400322207F0CD
:1043700029FC2046FCF748FB0B4803B0BDE8F040A1
:1043800008F00CBC511A5C2202FB01F292FBF3F321
:104390001B33C6E7521A02EB4202C2EB421223441D
:1043A00092FBF3F31B33D8E70C9FFF1FE88DFF1F31
:1043B0003C8BFF1F34380100003801000438010035
:1043C0001C380100309EFF1F609DFF1F949EFF1F41
:1043D000B89DFF1FB49EFF1F10B581B219481A4C3B
:1043E00007F08CFF0221174807F082FF4F2121229E
:1043F000144807F079FF21880B2910D90C2917D010
:10440000012212490F480BF059F921880D480C3947
:104410000BF0B8F90B48BDE810400BF063B90C394C
:1044200008480BF0AFF90748BDE810400BF05AB947
:104430000322074903480BF041F90248BDE8104048
:104440000BF050B90C9FFF1FD69EFF1F6036010076
:104450004038010070B5194C82B034260023012584
:1044600020460193009640230B223F2107F078FB62
:1044700040230B222046009601953F2107F0F2FBD6
:104480002946204607F03AFF2946204607F030FF2C
:1044900020460F22442107F027FF09220849204621
:1044A0000BF00CF920460BF01DF92846FFF794FF9E
:1044B000204602B0BDE8704008F070BB0C9FFF1FA3
:1044C0007837010008B581B20F4807F017FF0221C5
:1044D0000D4807F00DFF21224F210B4807F004FF84
:1044E0000A4B1A88012A0CD0022A0EBF0849094932
:1044F000032205480BF0E2F80348BDE808400BF042
:10450000F1B802220449F4E70C9FFF1F249EFF1F0D
:104510004438010030360100E437010070B5194C11
:1045200082B03426002301252046019300964023C3
:104530000B223F2107F014FB40230B22204600965C
:1045400001953F2107F08EFB2946204607F0D6FE55
:104550002946204607F0CCFE20460F22472107F0CF
:10456000C3FE0822084920460BF0A8F820460BF0AD
:10457000B9F82846FFF7A6FF204602B0BDE8704014
:1045800008F00CBB0C9FFF1F6037010008B581B21B
:10459000224807F0B3FE0221204807F0A9FE21229D
:1045A0004F211E4807F0A0FE1D4B1B88042B33D85B
:1045B000DFE803F0121A222A0300212253211748B0
:1045C00007F092FE1749022214480BF077F81348BF
:1045D000BDE808400BF086B821224F210F4807F0B4
:1045E00083FE03221049EFE7212253210B4807F0F5
:1045F0007BFE02220D49E7E721225321074807F0FD
:1046000073FE02220A49DFE721225321034807F003
:104610006BFE02220749D7E708BD00BF0C9FFF1FB2
:10462000C89DFF1F54380100303601004838010092
:104630004C3801005038010070B5194C82B0342656
:104640000023012520460193009640230B223F21A1
:1046500007F086FA40230B222046009601953F2161
:1046600007F000FB2946204607F048FE2946204671
:1046700007F03EFE20460F22442107F035FE0922B6
:10468000084920460BF01AF820460BF02BF8284674
:10469000FFF77CFF204602B0BDE8704008F07EBA0C
:1046A0000C9FFF1F9837010000B53E4B1B78013B64
:1046B00087B0052B16D8DFE803F0182D42576003AA
:1046C0000123394A194606201370FCF787F9374849
:1046D00008F064FA364A374B12680592059A1A6058
:1046E000FFF7B8FE07B05DF804FB0123324A194614
:1046F00018461370FCF772F92C4808F04FFA2C4A50
:104700002C4B12680192019A1A60FFF707FF07B05D
:104710005DF804FB0123294A194602201370FCF7B7
:104720005DF9224808F03AFA214A224B12680292B7
:10473000029A1A60FEF7DAF907B05DF804FB01236C
:104740001F4A194603201370FCF748F9174808F070
:1047500025FA174A174B12680392039A1A60FFF75B
:104760006BFF07B05DF804FB1649174B6E20012262
:1047700008701A7007B05DF804FB0123134A19464C
:1047800005201370FCF72AF9084808F007FA084AD0
:10479000084B12680492049A1A60FFF799F807B060
:1047A0005DF804FB548AFF1F969DFF1F0C9FFF1F9F
:1047B000489FFF1F449EFF1F509EFF1F589DFF1FD5
:1047C000649DFF1F109EFF1F588CFF1FC59DFF1F7C
:1047D00010B5334C334808F03FF8237803BB012170
:1047E0003048314C07F08AFD06212E4807F080FD45
:1047F0002388092B4ED9632B4FF00A0294BF1F2147
:104800001146284807F070FD218826480AF0BAFFB3
:1048100024480AF067FF2348BDE8104008F0BEB9FD
:10482000FCF7D8FF2378012BD9D9022B4FF00101D7
:104830001C4817D007F062FD06211A4807F058FD02
:104840000A221146174807F04FFD03221749154861
:104850000AF034FF13480AF045FF1248BDE8104043
:1048600008F09CB907F04AFD06210E4807F040FD0C
:104870000A2211460B4807F037FD03220C4909486C
:104880000AF01CFF07480AF02DFF0648BDE810405B
:1048900008F084B90A223021024807F025FDB3E769
:1048A000669DFF1F0C9FFF1F709EFF1F5C3801005D
:1048B0005838010008B581B2394807F01FFD0221C0
:1048C000374807F015FD374B1B884BB1013B092BCF
:1048D00065D8DFE803F01C242C343C444C545C14B1
:1048E00021224F212E4807F0FFFC2F4903222C489C
:1048F0000AF0E4FE2A48BDE808400AF0F3BE21228F
:104900005321274807F0F0FC02222849EFE7212233
:104910005321234807F0E8FC02222549E7E721223A
:1049200053211F4807F0E0FC02222249DFE7212241
:1049300053211B4807F0D8FC02221F49D7E7212248
:104940005321174807F0D0FC02221C49CFE721224F
:104950004F21134807F0C8FC03221949C7E7212259
:104960004F210F4807F0C0FC03221649BFE7212260
:104970004F210B4807F0B8FC03221349B7E7212267
:104980004F21074807F0B0FC03221049AFE721226E
:104990005321034807F0A8FC02220D49A7E708BDF0
:1049A0000C9FFF1F9C9EFF1F303601007C380100CA
:1049B000483801006038010064380100683801009F
:1049C0006C3801007038010074380100783801003B
:1049D0005038010070B5194C82B0342600230125EF
:1049E00020460193009640230B223F2107F0B8F8A0
:1049F00040230B222046009601953F2107F032F913
:104A00002946204607F07AFC2946204607F070FC2C
:104A100020460F22442107F067FC0922084920465E
:104A20000AF04CFE20460AF05DFE2846FFF742FFE2
:104A3000204602B0BDE8704008F0B0B80C9FFF1FE0
:104A40002437010008B581B2414807F057FC022124
:104A50003F4807F04DFC3F4B1B880C2B77D8DFE815
:104A600003F0161E262E363E464E565E666E070034
:104A700021225321364807F037FC374902223448B7
:104A80000AF01CFE3248BDE808400AF02BBE212285
:104A900053212F4807F028FC02223049EFE721225A
:104AA00053212B4807F020FC02222D49E7E7212261
:104AB0005321274807F018FC02222A49DFE7212268
:104AC0005321234807F010FC02222749D7E721226F
:104AD0004F211F4807F008FC03222449CFE7212279
:104AE00053211B4807F000FC02222149C7E721227D
:104AF0005321174807F0F8FB02221E49BFE7212285
:104B00005321134807F0F0FB02221B49B7E721228B
:104B100053210F4807F0E8FB02221849AFE7212292
:104B200053210B4807F0E0FB02221549A7E7212299
:104B30005321074807F0D8FB022212499FE72122A0
:104B40005321034807F0D0FB02220F4997E708BD25
:104B50000C9FFF1FA49EFF1FB0380100803801008A
:104B600084380100883801008C3801009038010039
:104B700094380100983801009C380100A0380100E9
:104B8000A4380100A8380100AC38010070B5194CF8
:104B900082B034260023012520460193009640234D
:104BA0000B223F2106F0DCFF40230B22204600961B
:104BB00001953F2107F056F82946204607F09EFB55
:104BC0002946204607F094FB20460F22502107F08B
:104BD0008BFB0522084920460AF070FD20460AF0AA
:104BE00081FD2846FFF72EFF204602B0BDE8704049
:104BF00007F0D4BF0C9FFF1F4C37010000B5444B9A
:104C00001B78013B87B0052B16D8DFE803F0182D81
:104C100042576C0301233F4A194606201370FBF7E5
:104C2000DDFE3D4807F0BAFF3C4A3D4B1268059255
:104C3000059A1A60FDF7E8FE07B05DF804FB012352
:104C4000384A194618461370FBF7C8FE324807F079
:104C5000A5FF324A324B12680092009A1A60FFF7A1
:104C6000B9FE07B05DF804FB01232F4A1946022064
:104C70001370FBF7B3FE284807F090FF274A284B34
:104C800012680192019A1A60FEF760FC07B05DF8A5
:104C900004FB0123254A194603201370FBF79EFEEF
:104CA0001D4807F07BFF1D4A1D4B12680292029AB5
:104CB0001A60FDF7E3FF07B05DF804FB01231C4A0F
:104CC000194604201370FBF789FE134807F066FFAE
:104CD000124A134B12680392039A1A60FFF756FFA9
:104CE00007B05DF804FB0123124A19460520137032
:104CF000FBF774FE084807F051FF084A084B12689A
:104D00000492049A1A60FEF775FD07B05DF804FB83
:104D1000648AFF1FF09DFF1F0C9FFF1F489FFF1F0E
:104D2000449EFF1F5A9DFF1FDC9EFF1F8C9DFF1F8F
:104D3000379FFF1FBA9DFF1F2DE9F0430320ADF5FC
:104D4000257D08F0D5FFB0FA80F4042008F0D0FFEC
:104D5000002814BF00210221640905200C4408F03A
:104D6000C7FF002814BF0021042106200C4408F0CE
:104D7000BFFF9E4D9E4E2B68002814BF00210821C6
:104D800021449942316000F02D819A4C9A4B22685F
:104D90000492049A1A60236805939848059B00685A
:104DA000944F9B1A834220D9954B1A68914216D092
:104DB0003A680792934ADDF81CE093481960C2F8FC
:104DC00000E00AF0DFFC90480AF08CFC3B68069398
:104DD0008E4A8F4B06981060316801221A700129A3
:104DE00000F0E180042900F0DE808A4F29603D78E0
:104DF000002D00F0CD80236882490B93864A0B9BDF
:104E0000096812687B485B1A93423FD9834E8448F5
:104E10008449854A854D864CDFF864C2DFF864E238
:104E200001233370002303700B7013708148824993
:104E3000824A2B70237003700B701370804D814C6D
:104E400081488249824A2B70237003700B70137063
:104E5000804D814C81488249824A8CF800303B70F9
:104E60008EF800302B70237003700B701370AE211E
:104E70007D48674C07F0F8FC002333702378002B43
:104E800040F004810DF5257DBDE8F083022D00F092
:104E90003381012D00F0E681642D00F089810A2D17
:104EA00000F02A820B2D01F03B800C2D01F0478190
:104EB000142D01F05482152D00F0B883162D01F049
:104EC000B7841E2D01F0BE861F2D01F06487202DB2
:104ED00002F07480282D02F0D181292D02F0788211
:104EE0002A2D02F085833C2D02F073843D2D02F0C3
:104EF0002185502D02F08C865A2D02F0D3866E2D1E
:104F0000C0D1464E3378002B43F078804A4D2A7842
:104F1000002A02F076872368DFF86C818E93534A6B
:104F20008E9BD8F8001012685B1A934211D9504B2F
:104F30001A78012A0CBF002201221A701878FDF796
:104F40000DFE494807F02AFE23688F938F9BC8F80F
:104F500000302F4A1378002B94D0294B1B68002176
:104F6000013B1170072B8DD801A252F823F000BF2E
:104F70004D9500001F950000854E0000E99400004B
:104F8000854E0000854E0000854E0000BB94000059
:104F9000224E3378002B7FF46AAF1D4C2378002B10
:104FA0003FF470AF72E023681848324A08930668ED
:104FB000089B10680F4A9B1B83427FF616AF13684D
:104FC0002D4809932D4E099B07683668DB1BB342B9
:104FD0007FF60BAF13680A930A9A0D4B0260012209
:104FE0001A7002E7044B034C1A68D4E6289EFF1F90
:104FF000F89EFF1F489FFF1FA09EFF1F608CFF1F92
:10500000989EFF1F909DFF1F1094FF1F0C9EFF1F77
:10501000F89DFF1F109EFF1FF08DFF1F588CFF1F74
:105020005A9DFF1FDC9EFF1F8C9DFF1F509EFF1F80
:10503000589DFF1F649DFF1F389EFF1FC59DFF1FCA
:10504000969DFF1FBA9DFF1FF09DFF1F499EFF1FEA
:10505000EC9EFF1F5C9EFF1F049EFF1FE09DFF1F35
:10506000E89EFF1FE99EFF1F0C9FFF1F908DFF1FF3
:10507000949EFF1F508AFF1F889DFF1FB48CFF1F47
:10508000B29EFF1FF19DFF1F449EFF1F0023237050
:10509000FBF776FBB94ABA4BBA49BB4812781B7882
:1050A0000968007802EB43034A1E03EB80030E2AD3
:1050B0003FF6E8AE01A151F822F000BF67550000AD
:1050C0007F550000854E00002F550000854E0000E2
:1050D000854E0000854E0000F5540000854E00000E
:1050E000854E0000854E0000854E0000854E000074
:1050F000854E0000F1540000A44E3378002B40F0A0
:105100000287A34D2A6823680D93A2490D9B096865
:105110009B1A8B4211D9A048A0490122002302709A
:1051200026200B703B703270FBF7F4FC9C4B198807
:10513000884202D02620FBF7E1FC9A4B1A78002A1D
:105140003FF4A0AE00221A70FBF71AFB8B4A8C4B7F
:105150008C498D4812781B780968007802EB43036C
:105160004A1E03EB80030E2A3FF68CAE01A151F8D4
:1051700022F000BFAD5700007D570000854E0000B3
:1051800037570000854E0000854E0000854E000018
:1051900011570000854E0000F3570000854E0000B7
:1051A000854E0000854E0000854E0000F154000041
:1051B000764E3378002B41F0CC807B4D2B78002B42
:1051C00040F05081DFF8F89199F80050002D01F07F
:1051D0005D812368DFF8EC812493744AD8F80010CD
:1051E000249B12685B1A9342714A117800D8C1B1AE
:1051F000704B1878012802F0D78001201870002920
:1052000041F0D68618786C4B013D53F82510FDF718
:105210006DFD6A4807F0C2FC23682593259BC8F8FA
:105220000030604A1378002B3FF42CAE554B1B68BE
:105230000021013B1170072B3FF624AE01A252F86A
:1052400023F000BF7B5C00003B5C0000854E00004B
:10525000F15B0000854E0000854E0000854E000089
:10526000A35B0000494E3378002B40F06287DFF8E3
:10527000589199F80000002800F0A8802368DFF812
:1052800044811293494A129BD8F8001012685B1AA5
:10529000934210D9474B1A78012A0CBF00200120F5
:1052A0001870FDF7B7FE454807F078FC23681393A4
:1052B000139BC8F800303B4A1378002B3FF4E2AD53
:1052C000304B1B680021013B1170072B3FF6DAAD14
:1052D00001A252F823F000BF91590000615900006B
:1052E000854E00002B590000854E0000854E0000C1
:1052F000854E0000FB580000244E3378002B40F010
:105300008D812368DFF8BC802E93284A2E9BD8F825
:10531000001012685B1A934210D9264B1A78012AA2
:105320000CBF002001201870FBF76EFB234807F02C
:1053300035FC23682F932F9BC8F80030194A137847
:10534000002B3FF49FAD0F4B1B680021013B1170F8
:10535000072B3FF697AD01A252F823F0C558000085
:10536000BD580000854E000087580000854E0000A3
:10537000854E0000854E000053580000DD9EFF1F43
:10538000389FFF1F989EFF1F399FFF1F588CFF1FDC
:10539000AC9DFF1FEC8DFF1F959DFF1F669DFF1F9E
:1053A000709EFF1FF89DFF1F499EFF1F908DFF1FDE
:1053B000049FFF1F949EFF1F448CFF1F0C9FFF1F25
:1053C000EC9EFF1F449EFF1FB29EFF1FDFF8349329
:1053D00099F80030002B40F0E580DFF82C9399F825
:1053E0000020002A01F050812268DFF820831A9201
:1053F000B1491A9AD8F800000968121A8A4211D9DC
:10540000AE4A117801290BBF1846012013701070A5
:10541000FCF78EFDAA4807F0C1FB23681B931B9B7A
:10542000C8F80030A74A1378002B3FF42BADA64BE9
:105430001B680021013B1170072B3FF623AD01A231
:1054400052F823F09B5E00005F5E0000854E000076
:10545000D15E0000854E0000854E0000854E0000A4
:105460002F5E00002368DFF8A4822093924AD8F8C8
:105470000010209B12685B1A9342944A117800D85E
:10548000B1B18E4B1878012801F08E85012018707B
:10549000002941F0AB8318788D4B1968FDF726FC85
:1054A000874807F07BFB23682193219BC8F80030D5
:1054B000844A1378002B3FF4E5AC834B1B68002132
:1054C000013B1170072B3FF6DDAC01A252F823F02F
:1054D0009D5A0000695A0000854E0000315A0000B4
:1054E000854E0000854E0000854E0000C759000023
:1054F00008F024FF774B78491C78784B784A098864
:105500001B8812680B44002C01F08C80B2EB630FF7
:1055100081F28A86734B1B78002B01F03284AF2115
:10552000674807F0A1F901233B703370AAE4002B10
:1055300001F0A680013B6C4A32F813304BB16B4D41
:105540006B486C496C4A2B800123002505700B7059
:105550001370AF215A4807F087F9012302223A70ED
:10556000237033708EE463B901232370AF21544854
:1055700007F07AF9022201233A70337082E4002B9B
:10558000F4D0013B584A32F81330002BEED0574C80
:1055900057485849584A23800123002404700B704F
:1055A0001370E3E72368DFF864811693424A169B81
:1055B000D8F8001012685B1A93420FD93F4B1A7843
:1055C000012A18BF01201870FDF7A8FD3C4807F01C
:1055D000E5FA23681793179BC8F80030394A137807
:1055E000002B3FF44FAC384B1B680021013B11707E
:1055F000072B3FF647AC01A252F823F06D5B000089
:105600003D5B0000854E0000075B0000854E0000FA
:10561000854E0000854E0000D75A0000FEF794FC2E
:10562000364A01210023117033706AE62368DFF8DF
:10563000DC803A93204A3A9BD8F8001012685B1A33
:10564000934219D91D4A1E481378012B0CBF002321
:10565000012313702A4A0193B2F900301A22194625
:105660000092142206F0AEFA154807F097FA236864
:105670003B933B9BC8F80030124A1378002B3FF451
:1056800001AC114B1B680021013B1170072B3FF649
:10569000F9AB01A252F823F0AF5D0000895D000074
:1056A000854E0000095D0000854E0000854E00001B
:1056B000854E0000C75C0000908DFF1F949EFF1F69
:1056C0000C9FFF1FF89DFF1F989EFF1F049FFF1F49
:1056D000048BFF1F949DFF1F8E9DFF1F529EFF1F77
:1056E000C09DFF1FBB9DFF1F709DFF1F709EFF1F72
:1056F000F29DFF1F959DFF1F669DFF1F679DFF1F6A
:10570000609DFF1FB09DFF1FF19DFF1F449EFF1F67
:10571000BA4C2378012B41F253862620FBF7FAF985
:10572000B74B1988884202D02620FBF7E7F90023FF
:105730002370FFF7A7BB002B01F04185013BB14A65
:1057400032F8136096B1AE4BAF48B049AB4A1E80F9
:1057500000270123077026200B701370FBF7DAF97E
:10576000864203D031462620FBF7C8F9FFF730F810
:1057700023681093109B2B60FFF784BB83B1013B20
:10578000A04A32F813305BB19D4E9F489F499B4A17
:1057900033800123002606700B701370FFF718F892
:1057A00023680F930F9B2B60FFF76CBB002B01F05E
:1057B000F484013B934A32F8136096B1904B9248BF
:1057C00092498E4A1E8000270123077026200B7005
:1057D0001370FBF79FF9864203D031462620FBF772
:1057E0008DF9FEF7F5FF23680E930E9B2B60FFF7F4
:1057F00049BBFBF73FFD864807F02EF8012184489E
:1058000006F07CFD0221824806F072FD0F22232162
:105810007F4806F069FD05227E497D4809F04EFF6C
:105820007B4809F05FFF1E222321794806F05CFDCA
:1058300005227949764809F041FF754809F052FF81
:10584000734807F0ABF923681193119B2B60FFF7A6
:1058500019BB012302203B703370FBF75BF96F4BE0
:105860001988884202D00220FBF748F90420FBF790
:1058700051F96B4B198888423FF404AB0420FBF7C5
:105880003DF9FFF7FFBA01233C22022033703A7042
:10589000FBF740F9614B1988884202D00220FBF7E0
:1058A0002DF90420FBF736F95D4B198888423FF447
:1058B000E9AA0420FBF722F9FFF7E4BA0B233B70B7
:1058C000FFF7E0BA01231422022033703A70FBF78D
:1058D00021F9524B1988884202D00220FBF70EF9B9
:1058E0000420FBF717F94E4B198888423FF4CAAAE7
:1058F0000420FBF703F9FFF7C5BA0120FDF78AFB87
:10590000484B434800241C7007F048F90E2089F8E2
:105910000040FBF7FFF8444B198888423FF4B2AAD5
:105920000E20FBF7EBF8FFF7ADBA3F4D2B88172B96
:105930003FF6A8AA0020FDF76DFB2B880120034449
:105940002B80FDF767FB374B314800221A7007F0B8
:1059500025F923681593159BC8F80030FFF792BA14
:105960000120FDF757FB2F4B294800241C7007F03E
:1059700015F90E2089F80040FBF7CCF82A4B19885E
:1059800088423FF47FAA0E20FBF7B8F8FFF77ABAF7
:10599000254D2B88002B3FF475AA0020FDF73AFB1C
:1059A0002B880120013B2B80FDF734FB1D4B184851
:1059B00000221A7007F0F2F823681493149BC8F8B9
:1059C0000030FFF75FBA194C01202168FDF78EF90E
:1059D000144B0F4800261E7007F0E0F844202E708C
:1059E000FBF798F82168183188423FF44BAA89B236
:1059F0004420FBF783F8FFF745BA00BF669DFF1F01
:105A0000709EFF1F709DFF1FF29DFF1F959DFF1F42
:105A10000C9FFF1FB4380100BC3801001A9EFF1F05
:105A2000F49EFF1F949EFF1FA89DFF1F048BFF1F66
:105A3000AE4D296817293FF725AA0020FDF756F932
:105A40002B680133194601202B60FDF74FF9A84B55
:105A5000A84800221A7007F0A1F823682393239B1B
:105A6000C8F80030FFF70EBAA04C01202168FDF7FE
:105A70003DF99F4B9F4800261E7007F08FF8442089
:105A80002E70FBF747F82168183188423FF4FAA9D5
:105A900089B24420FBF732F8FFF7F4B9934D296837
:105AA00011F1170FFFF6EEA90020FDF71FF92B6883
:105AB000013B194601202B60FDF718F98C4B8D48EE
:105AC00000221A7007F06AF823682293229BC8F814
:105AD0000030FFF7D7B90120FDF720FB844B854844
:105AE00000241C7007F05AF8282089F80040FBF7C2
:105AF00011F8814B198888423FF4C4A92820FAF78D
:105B0000FDFFFFF7BFB97C4D2B88052B3FF6BAA9E7
:105B10000020FDF703FB2B88012003442B80FDF7B9
:105B2000FDFA734B734800221A7007F037F82368A8
:105B30001993199BC8F80030FFF7A4B90120FDF7AD
:105B4000EDFA6B4B6B4800241C7007F027F82820F7
:105B500089F80040FAF7DEFF674B198888423FF466
:105B600091A92820FAF7CAFFFFF78CB9624D2B885C
:105B7000002B3FF487A90020FDF7D0FA2B880120E5
:105B8000013B2B80FDF7CAFA594B5A4800221A7084
:105B900007F004F823681893189BC8F80030FFF743
:105BA00071B999F80030554E013B012056F8231089
:105BB000FDF79CF84E4B4F4800221A7006F0EEFF9E
:105BC00099F8005005F122046400E4B2013D20463A
:105BD000FAF7A0FF56F825101831884203D089B291
:105BE0002046FAF78BFF002389F80030FFF74AB907
:105BF00099F80030414D424E013B55F823101729CA
:105C00003FF740A90020FDF771F83378013B0120F0
:105C100055F823200244114645F82320FDF766F885
:105C2000334B344800221A7006F0B8FF23682793DC
:105C3000279BC8F80030FFF725B999F800302F4EA0
:105C4000013B012056F82310FDF750F8284B294856
:105C500000221A7006F0A2FF99F8005005F1220404
:105C60006400E4B22046013DFAF754FF56F82530AF
:105C70009842B8D003F11801B1E799F800301F4DF0
:105C80001F4E013B55F8231011F1170FFFF6FAA82C
:105C90000020FDF72BF83378013B012055F8232035
:105CA000013A114645F82320FDF720F8104B114822
:105CB00000221A7006F072FF23682693269BC8F80C
:105CC0000030FFF7DFB80F4B0A48B3F90030142457
:105CD00001221A2501920095194622463C7005F0D2
:105CE00071FF044806F05AFFFFF7CCB8048BFF1F82
:105CF000949EFF1F0C9FFF1FBE9EFF1F448CFF1F23
:105D0000EC9EFF1F609DFF1FB24EB34BB34F328816
:105D10001B6839681A448A42BFF6B4A8B04D328075
:105D2000B5F90030AF484FF0000E1A2219468DE841
:105D30000440142205F046FFAB4B3A6819683388DB
:105D4000521A5C2A42F34280591A5D23561C03FB07
:105D500001F393FBF6F61B3633B201211A220191AF
:105D60000092194614229F482E6005F02BFF9D4893
:105D700006F014FF23683D933D9A9C4BC8F8002021
:105D800000221A70FFF77EB8954B9648B3F90030A1
:105D900001241A228DE814001624194614223C709E
:105DA00005F010FF8F4806F0F9FEFFF76BB8894E3B
:105DB000894A8D4F3388126839689A1A8A427FF768
:105DC00061A8874D3280B5F9003086484FF0000E4B
:105DD0001A2219468DE80440142205F0F3FE7F4B89
:105DE00039681A683388521A5C2A41F3F887591ABD
:105DF0005D23561C03FB01F393FBF6F61B3633B20F
:105E000001211A22019100921946142275482E6030
:105E100005F0D8FE734806F0C1FE23683C933C9A17
:105E2000724BC8F8002000221A70FFF72BB801202F
:105E3000FCF77EF86D4B6B4800241C7006F0AEFE3C
:105E4000102089F80040FAF765FE694B19888842EE
:105E50003FF418A81020FAF751FEFFF713B8FAF72D
:105E60008FFC644B1C78002C41F0B8860120FCF7B5
:105E70005FF85E4B5B481C7006F090FE102089F8BE
:105E80000040FAF747FE5A4B198888423EF4FAAFB1
:105E90001020FAF733FEFEF7F5BF554D2B88012B86
:105EA0007EF6F0AF0020FCF743F82B880120013B81
:105EB0002B80FCF73DF84D4B4A4800221A7006F043
:105EC0006DFE23681C931C9BC8F80030FEF7DABFF8
:105ED000474D2B880F2B3EF6D5AF0020FCF728F856
:105EE0002B88012003442B80FCF722F83F4B3D48D0
:105EF00000221A7006F052FE23681D931D9BC8F8FD
:105F00000030FEF7BFBF0390FEF762FC03983A4DE6
:105F100003680C930C9A2A6000233370FFF7F3B8E0
:105F20000368DFF8E4803093344A309BD8F80010DF
:105F300012685B1A934219D92C4A2A481378012B0C
:105F40000CBF002301231370254A0193B2F90030DE
:105F50001A2219460092142205F034FE214806F058
:105F60001DFE23683193319BC8F80030244A137812
:105F7000002B3EF487AF234B1B680021013B1170BF
:105F8000072B3EF67FAF01A252F823F0B36000006A
:105F90008D600000854E00000D600000854E000001
:105FA000854E0000854E0000AD5F00000C4B0D4893
:105FB000B3F9003001241A228DE814000A2419468E
:105FC00014223C7005F0FEFD064806F0E7FDFEF7E2
:105FD00059BF00BFE89DFF1FC09EFF1FE48DFF1F3C
:105FE000609DFF1F0C9FFF1F688AFF1F949EFF1F6D
:105FF000649EFF1F949DFF1FAC9DFF1F908DFF1F90
:10600000F89DFF1F989EFF1F449EFF1FA24EA34BAB
:10601000A34F32881B6839681A448A42BEF632AFF1
:10602000A04D3280B5F900309F484FF0000E1A2283
:1060300019468DE80440142205F0C4FD9B4B3A68D4
:1060400019683388521A5C2A41F35A84591A5D231D
:10605000561C03FB01F393FBF6F61B3633B201210A
:106060001A2201910092194614228F482E6005F0E1
:10607000A9FD8D4806F092FD23683393339A8C4B2B
:10608000C8F8002000221A70FEF7FCBE854B864837
:10609000B3F9003001241A228DE814000C241946AB
:1060A00014223C7005F08EFD7F4806F077FDFEF768
:1060B000E9BE794E794A7D4F3388126839689A1A59
:1060C0008A427EF7DFAE774D3280B5F900307648F0
:1060D0004FF0000E1A2219468DE80440142205F0F4
:1060E00071FD6F4B39681A683388521A5C2A41F384
:1060F0001084591A5D23561C03FB01F393FBF6F63B
:106100001B3633B201211A22019100921946142242
:1061100065482E6005F056FD634806F03FFD236894
:106120003293329A624BC8F8002000221A70FEF7B0
:10613000A9BEFCF773FE00233370FFF798B803681D
:10614000DFF8848134935B4A349BD8F800101268DE
:106150005B1A934219D9564B53481A78012A0CBF3F
:10616000002201221A70544B0192B3F900303922F7
:1061700019460092322205F025FD4B4806F00EFD2F
:1061800023683593359BC8F800304C4A1378002BB0
:106190003EF478AE4A4B1B680021013B1170072B7F
:1061A0003EF670AE01A252F823F000BFCD620000AF
:1061B00073620000854E0000F3610000854E000010
:1061C000854E0000854E0000CD6100003A4B3648F8
:1061D000B3F90030012439228DE814000A2419464D
:1061E00032223C7005F0EEFC2F4806F0D7FCFEF79B
:1061F00049BE344E294B2A4F32881B6839681A44ED
:106200008A42BEF63FAE2C4D3280B5F900302648AA
:106210004FF0000E392219468DE80440322205F075
:10622000D1FC224B3A6819683388521A5C2A41F330
:10623000A484591A5D23561C03FB01F393FBF6F665
:106240001B3633B2012139220191009219463222C4
:1062500015482E6005F0B6FC134806F09FFC236835
:106260003793379A124BC8F8002000221A70FEF7B5
:1062700009BE114B0C48B3F90030012439228DE8D6
:1062800014000A24194632223C7005F09BFC064893
:1062900006F084FCFEF7F6BD1A9EFF1FA89EFF1FA6
:1062A000588AFF1F609DFF1F0C9FFF1F3C9EFF1F12
:1062B000949EFF1F908DFF1FB49EFF1FF89DFF1F30
:1062C000989EFF1FF49EFF1F449EFF1FC34FC44AAA
:1062D000C448C5493B881268008809689A1A43185F
:1062E0009A427EF7CFADC14D3A80B5F90030C04833
:1062F0003922002619468DE84400322205F062FC5E
:10630000BC4ABD4B11681A683B88521A5C2A41F39B
:106310003D84591A5D23561C03FB01F393FBF6F6EB
:106320001B3633B2012139220191009219463222E3
:10633000AF482E6005F046FCAD4806F02FFC236800
:106340003693369AAD4BC8F8002000221A70FEF73B
:1063500099BDFCF7D5FD00233370FEF72EBFA84E84
:106360003378002B40F004852368DFF8B08238933F
:10637000A44A389BD8F8001012685B1A934210D9CF
:106380009E4B1A78012A0CBF002001201870FAF7E2
:106390003BFB974806F002FC23683993399BC8F809
:1063A0000030994A1378002B3EF46CAD974B1B6874
:1063B0000021013B1170072B3EF664AD01A252F89B
:1063C00023F000BF576400004F640000854E0000BA
:1063D00019640000854E0000854E0000854E0000C7
:1063E000E5630000012306203B703370FAF792FB4F
:1063F000874B1988884202D00620FAF77FFB0820D5
:10640000FAF788FB834B198888423EF43BAD08209D
:10641000FAF774FBFEF736BD01230A22062033701B
:106420003A70FAF777FB7A4B1988884202D0062037
:10643000FAF764FB0820FAF76DFB764B198888425F
:106440003EF420AD0820FAF759FBFEF71BBD1523DB
:106450003B70FEF717BD01231E22062033703A70F1
:10646000FAF758FB6A4B1988884202D00620FAF7DF
:1064700045FB0820FAF74EFB664B198888423EF42C
:1064800001AD0820FAF73AFBFEF7FCBCDFF890916B
:10649000236899F80010DFF88481002900F0D88281
:1064A0002893584A289BD8F8001012685B1A934228
:1064B00011D9524B1A78012A15BF012028461870AD
:1064C0001D70FCF727FF4A4806F068FB23682993F4
:1064D000299BC8F800304C4A1378002B3EF4D2AC0C
:1064E0004A4B1B680021013B1170072B3EF6CAACDA
:1064F00001A252F823F000BFAB6500007B650000ED
:10650000854E000049650000854E0000854E000064
:10651000854E0000196500000120FCF7FBFE374B9B
:10652000334800241C7006F039FB4E2089F80040E7
:10653000FAF7F0FA384B198888423EF4A3AC4E20A3
:10654000FAF7DCFAFEF79EBC0020FCF7E3FE324AC5
:106550001388B3FA83F35B0901201380FCF7DAFE9A
:10656000264B234800221A7006F018FB23682B9351
:106570002B9BC8F80030FEF785BC0120FCF7CAFE53
:106580001E4B1B4800241C7006F008FB4E2089F8A7
:106590000040FAF7BFFA204B198888423EF472ACEB
:1065A0004E20FAF7ABFAFEF76DBC0020FCF7B2FE06
:1065B000194A1388B3FA83F35B0901201380FCF7AF
:1065C000A9FE0E4B0A4800221A7006F0E7FA23686B
:1065D0002A932A9BC8F80030FEF754BCF49EFF1F94
:1065E000A89EFF1F1A9EFF1F9C8DFF1FB49EFF1FBA
:1065F0000C9FFF1F3C9EFF1F588AFF1F949EFF1F8A
:10660000588CFF1F908DFF1FF89DFF1F989EFF1F46
:10661000E89DFF1FD49EFF1FC69DFF1F449EFF1FC6
:106620005C9EFF1FB2EB630FFEF679AFAD4EAE4D31
:1066300033782A88B3FA83F382F002025B091146A9
:10664000422033702A80FAF759FA21460D2007F0CC
:1066500049FB962007F082FB01210D2007F042FB49
:10666000962007F07BFB21460D2007F03BFB962090
:1066700007F074FB01210D2007F034FBFEF702BC8C
:1066800001232370FEF765BF2368DFF894821E9311
:1066900096481E9BD8F8001000685B1A834215D9F3
:1066A000934B1978012916BF01221A701A70914B69
:1066B00008BF154618782946FAF790F98E4806F073
:1066C0006DFA23681F931F9BC8F800308B4B1A7814
:1066D000002A3EF4D7AB00221A70FAF751F8884A24
:1066E000884B8949894812781B780968007802EB41
:1066F00043034A1E03EB80030B2A3EF6C3AB01A102
:1067000051F822F0EF670000E7670000854E0000B7
:10671000A5670000854E0000854E0000854E0000F4
:1067200099670000854E000035670000854E000027
:1067300067670000002B3EF4A5AB754A754D1288C3
:1067400003F11900013B4000022425F813201146F3
:10675000012300F0FE0033703C70FAF7CFF96E4B66
:106760001C70FEF78FBB002B3EF48CAB03F11900BD
:10677000684D013B0022400025F8132011460123FB
:1067800000F0FE00022433703C70FAF7B7F9624B58
:1067900003221A70FEF776BB002201233A70337091
:1067A000FEF770BB534C207801287EF66BAB0021BE
:1067B000FAF714F923784E4D013BDBB2184601215C
:1067C0002370FAF70BF9002434238DE818004A48A7
:1067D0002C7040230B223F2105F0C2F9464806F0F9
:1067E000DDF9FEF74FBBFCF71DFDFEF74BBB414C3F
:1067F000207805283EF646AB0021FAF7EFF823781B
:106800003B4D0133DBB2184601212370FAF7E6F85D
:10681000002434238DE8180037482C7040230B22C5
:106820003F2105F09DF9344806F0B8F9FEF72ABB80
:106830002368DFF8EC803E932C4A3E9BD8F800108A
:1068400012685B1A934219D9294A2B481378012BF5
:106850000CBF002301231370304A0193B2F90030BA
:10686000392219460092322205F0ACF9224806F08E
:1068700095F923683F933F9BC8F800301F4A13786F
:10688000002B3EF4FFAA204B1B680021013B117036
:10689000072B3EF6F7AA01A252F823F0CB690000BD
:1068A000A5690000854E000025690000854E0000A6
:1068B000854E0000854E0000BD680000174B0E4855
:1068C000B3F90030012439228DE81400142419464C
:1068D00032223C7005F076F9074806F05FF9FEF7C2
:1068E000D1BA00BFBE9DFF1FF69EFF1F908DFF1FF8
:1068F000949EFF1F3289FF1F0C9FFF1FF89DFF1FF3
:10690000DD9EFF1F389FFF1F989EFF1F399FFF1FAF
:10691000709EFF1F709DFF1F669DFF1FB49EFF1F8F
:10692000449EFF1FB44EB54BB54F32881B68396883
:106930001A448A42BEF6A6AAB24D3280B5F900309A
:10694000B1484FF0000E392219468DE8044032223A
:1069500005F038F9AD4B3A6819683388521A5C2A49
:1069600041F34682591A5D23561C03FB01F393FB46
:10697000F6F61B3633B201213922019100921946F5
:106980003222A1482E6005F01DF99F4806F006F955
:1069900023684193419A9E4BC8F8002000221A7048
:1069A000FEF770BA974B9848B3F9003001243922AA
:1069B0008DE814001424194632223C7005F002F9C7
:1069C000914806F0EBF8FEF75DBA8B4E8B4A914882
:1069D000914933881268008809689A1A43189A42C4
:1069E0007EF750AA874D3280B5F9003086483922AB
:1069F000002719468DE88400322205F0E3F8834A27
:106A00007F4B11681A683388521A5C2A41F33C8222
:106A1000591A5D23561C03FB01F393FBF6F61B3654
:106A200033B201213922019100921946322276486F
:106A30002E6005F0C7F8744806F0B0F8236840935C
:106A4000409A734BC8F8002000221A70FEF71ABA59
:106A50002C93724A2C9BD8F8000012681B1A9342A0
:106A600011D96B4B1A78012A18BF012119706C4B90
:106A70001878F9F7B3FF644806F090F823682D936F
:106A80002D9BC8F80030674B1A78002A3EF4FAA90B
:106A900000221A70F9F774FE634A644B6449654832
:106AA00012781B780968007802EB43034A1E03EB57
:106AB00080030B2A3EF6E6A901A151F822F000BF9F
:106AC000AB6B0000A36B0000854E0000616B000003
:106AD000854E0000854E0000854E0000556B00007D
:106AE000854E0000F16A0000854E0000236B000017
:106AF000002B3EF4C7A9504A504D128803F11900EB
:106B0000013B4000022425F813201146012300F028
:106B1000FE0033703C70F9F7F1FF494B1C70FEF733
:106B2000B1B9002B3EF4AEA903F11900434D013B6E
:106B30000022400025F813201146012300F0FE003A
:106B4000022433703C70F9F7D9FF3D4B03221A70D1
:106B5000FEF798B9002201233A703370FEF792B91C
:106B60002F4C207801287EF68DA90021F9F736FFF9
:106B70002378274D013BDBB2184601212370F9F73A
:106B80002DFF002434238DE818001F482C7040236B
:106B90000B223F2104F0E4FF1B4805F0FFFFFEF746
:106BA00071B9FCF715FCFEF76DB91D4C207805286E
:106BB0003EF668A90021F9F711FF2378144D01333F
:106BC000DBB2184601212370F9F708FF00243423B3
:106BD0008DE818000C482C7040230B223F2104F054
:106BE000BFFF094805F0DAFFFEF74CB9002101208C
:106BF00011701870FEF750BCD49EFF1FC09EFF1F7F
:106C0000E48DFF1FB49EFF1F0C9FFF1F688AFF1FAC
:106C1000949EFF1FE89DFF1F9C8DFF1F908DFF1FFF
:106C2000948DFF1FF89DFF1FDD9EFF1F389FFF1FE4
:106C3000989EFF1F399FFF1F709EFF1F709DFF1FB3
:106C4000669DFF1FAA4E3378002B40F0B183236866
:106C5000DFF8D0824293A74A429BD8F8001012680E
:106C60005B1A934210D9A44B1A78012A0CBF00205A
:106C700001201870F9F7C8FEA04805F08FFF2368BF
:106C80004393439BC8F800309D4A1378002B3EF491
:106C9000F9A89C4B1B680021013B1170072B3EF6A5
:106CA000F1A801A252F823F03B6D0000336D000003
:106CB000854E0000FD6C0000854E0000854E0000F2
:106CC000854E0000C96C000001230A203B70337020
:106CD000F9F720FF8C4B1988884202D00A20F9F777
:106CE0000DFF0C20F9F716FF884B198888423EF4F7
:106CF000C9A80C20F9F702FFFEF7C4B8012314223B
:106D00000A2033703A70F9F705FF7F4B19888842E3
:106D100002D00A20F9F7F2FE0C20F9F7FBFE7B4BBC
:106D2000198888423EF4AEA80C20F9F7E7FEFEF77A
:106D3000A9B81F233B70FEF7A5B8012328220A201B
:106D400033703A70F9F7E6FE6F4B1988884202D02B
:106D50000A20F9F7D3FE0C20F9F7DCFE6B4B1988FB
:106D600088423EF48FA80C20F9F7C8FEFEF78AB8D7
:106D7000FCF7C6FF664A0121002311703370FFF74C
:106D8000F3BAAF215D4805F06FFD642201233A702C
:106D90003370FEF777B82368DFF888814493554A4B
:106DA000449BD8F8001012685B1A934219D9524AD2
:106DB00052481378012B0CBF002301231370554A4E
:106DC0000193B2F900301A2219460092142204F0FD
:106DD000F9FE4A4805F0E2FE23684593459BC8F852
:106DE0000030474A1378002B3EF44CA8454B1B68F3
:106DF0000021013B1170072B3EF644A801A252F876
:106E000023F000BF296F0000CB6E0000854E00000C
:106E10004B6E0000854E0000854E0000854E000040
:106E2000256E00003B4B3548B3F9003001241A228F
:106E30008DE814001E24194614223C7004F0C2FE92
:106E40002E4805F0ABFEFEF71DB82F4E324B334FE8
:106E500032881B6839681A448A42BEF613A82D4D41
:106E60003280B5F9003025484FF0000E1A2219463D
:106E70008DE80440142204F0A5FE294B3A681968F5
:106E80003388521A5C2A41F3AB80591A5D23561C91
:106E900003FB01F393FBF6F61B3633B201211A22F2
:106EA000019100921946142214482E6004F08AFEC3
:106EB000124805F073FE23684793479A0E4BC8F8B3
:106EC000002000221A70FDF7DDBF124B0B48B3F90A
:106ED000003001241A228DE81400202419461422BF
:106EE0003C7004F06FFE054805F058FEFDF7CABF80
:106EF000588CFF1F908DFF1F949EFF1F0C9FFF1F3C
:106F0000F89DFF1F989EFF1F309EFF1FB89DFF1F1B
:106F1000679DFF1F609DFF1FAC9EFF1F3C8BFF1FE7
:106F2000E88DFF1F449EFF1FAD4EAE4AAE4F338823
:106F3000126839689A1A8A427DF7A4AFAB4D328045
:106F4000B5F90030AA484FF0000E1A2219468DE814
:106F50000440142204F036FEA64B39681A683388C0
:106F6000521A5C2A41F39480591A5D23561C03FB84
:106F700001F393FBF6F61B3633B201211A2201917D
:106F80000092194614229A482E6004F01BFE98487D
:106F900005F004FE23684693469A974BC8F80020F4
:106FA00000221A70FDF76EBF00201870FEF770BA4D
:106FB0000021012011701870FEF725B92368DFF851
:106FC000648248938D4A489BD8F8001012685B1A77
:106FD000934219D9884A86481378012B0CBF0023A5
:106FE00001231370864A0193B2F900303922194601
:106FF0000092322204F0E6FD7D4805F0CFFD2368C3
:107000004993499BC8F800307E4A1378002B3DF421
:1070100039AF7D4B1B680021013B1170072B3DF6FA
:1070200031AF01A252F823F015710000EF7000009B
:10703000854E00006F700000854E0000854E0000F8
:10704000854E0000497000006D4B6948B3F900306F
:10705000012439228DE814001E24194632223C7086
:1070600004F0B0FD624805F099FDFDF70BBF674ED7
:107070005C4B604F32881B6839681A448A42BDF6FF
:1070800001AF5F4D3280B5F9003059484FF0000E26
:10709000392219468DE80440322204F093FD524B08
:1070A0003A6819683388521A5C2A41F37D80591A6C
:1070B0005D23561C03FB01F393FBF6F61B3633B23C
:1070C00001213922019100921946322248482E604E
:1070D00004F078FD464805F061FD23684B934B9A18
:1070E000454BC8F8002000221A70FDF7CBBE444B78
:1070F0003F48B3F90030012439228DE814001E24E2
:10710000194632223C7004F05DFD394805F046FD19
:10711000FDF7B8BE3D4E334A31483D4933881268C9
:10712000008809689A1A43189A427DF7ABAE344D2D
:107130003280B5F900302E483922002719468DE8F3
:107140008400322204F03EFD274A2A4B11681A6857
:107150003388521A5C2A41F34780591A5D23561C22
:1071600003FB01F393FBF6F61B3633B20121392200
:1071700001910092194632221D482E6004F022FD32
:107180001B4805F00BFD23684A934A9A1A4BC8F82E
:10719000002000221A70FDF775BE1E4A1E4E13888D
:1071A0001E48012B8CBF03F1FF33802313801C4A40
:1071B00000230121337003701170FEF712BB154AD2
:1071C000154E138815487F2B94BF0133012313807C
:1071D000134A00230121337003701170FEF7C6BA01
:1071E000309EFF1FAC9EFF1FE88DFF1F609DFF1F9D
:1071F0000C9FFF1F3C8BFF1F949EFF1F908DFF1F56
:10720000B49EFF1FF89DFF1F989EFF1FB89DFF1F94
:107210009C8DFF1F709EFF1FF29DFF1F669DFF1F2D
:10722000959DFF1F449EFF1FC04DC14C2B782288A7
:10723000B3FA83F382F004025B09114642202B70FB
:107240002280F9F75BFC00210D2006F04BFD962013
:1072500006F084FD01210D2006F044FD962006F085
:107260007DFD00210D2006F03DFD962006F076FD07
:1072700001210D2006F036FDFDF704BEAD4E33783A
:10728000002B40F04F832368DFF8E0824C93AA4A3A
:107290004C9BD8F8001012685B1A934210D9A74B88
:1072A0001A78012A0CBF002001201870F9F7ACFBF6
:1072B000A34805F073FC23684D934D9BC8F800303C
:1072C000A04A1378002B3DF4DDAD9F4B1B680021D5
:1072D000013B1170072B3DF6D5AD01A252F823F00A
:1072E000737300006B730000854E0000357300005F
:1072F000854E0000854E0000854E000001730000A1
:10730000012322203B703370F9F704FC8F4B19885E
:10731000884202D02220F9F7F1FB2420F9F7FAFB8A
:107320008B4B198888423DF4ADAD2420F9F7E6FB7C
:10733000FDF7A8BD01231E22222033703A70F9F711
:10734000E9FB824B1988884202D02220F9F7D6FB4C
:107350002420F9F7DFFB7E4B198888423DF492AD7B
:107360002420F9F7CBFBFDF78DBD29233B70FDF7FA
:1073700089BD01233C22222033703A70F9F7CAFB01
:10738000724B1988884202D02220F9F7B7FB2420DB
:10739000F9F7C0FB6E4B198888423DF473AD242089
:1073A000F9F7ACFBFDF76EBD00201870FDF727BFA5
:1073B000FCF7EEFE674A012100231170337046E4AA
:1073C0006549012300220B7033703A70FEF7A5B9AE
:1073D0002368DFF898814E93574A4E9BD8F80010E7
:1073E00012685B1A93421AD9544B5C491A78544874
:1073F000012A0CBF002201221A701A78B1F900305C
:1074000001921A2219460092142204F0DBFB4C4828
:1074100005F0C4FB23684F934F9BC8F80030494ADE
:107420001378002B3DF42EAD474B1B680021013B28
:107430001170072B3DF626AD01A252F823F000BFD4
:107440007175000007750000854E0000877400000C
:10745000854E0000854E0000854E000061740000DE
:107460003E4B3748B3F9003001241A228DE814004E
:107470002824194614223C7004F0A4FB304805F07F
:107480008DFBFDF7FFBC314E354B364F32881B6804
:1074900039681A448A42BDF6F5AC304D3280B5F9F0
:1074A000003027484FF0000E1A2219468DE804409C
:1074B000142204F087FB2C4B3A6819683388521A5F
:1074C0005C2A41F32882591A5D23561C03FB01F301
:1074D00093FBF6F61B3633B201211A22019100927A
:1074E0001946142216482E6004F06CFB144805F06F
:1074F00055FB23685193519A104BC8F80020002285
:107500001A70FDF7BFBC154B0D48B3F900300124CC
:107510001A228DE814002A24194614223C7004F023
:1075200051FB074805F03AFBFDF7ACBC189EFF1F66
:10753000F69EFF1F588CFF1F908DFF1F949EFF1F0C
:107540000C9FFF1FF89DFF1F989EFF1F8E9DFF1F22
:10755000529EFF1F679DFF1F959DFF1F609DFF1F90
:10756000589EFF1F5C8AFF1FFC8DFF1F449EFF1F5C
:10757000B94EBA4ABA4F3388126839689A1A8A42A1
:107580007DF780ACB74D3280B5F90030B6484FF08A
:10759000000E1A2219468DE80440142204F012FB52
:1075A000B24B39681A683388521A5C2A41F3C58194
:1075B000591A5D23561C03FB01F393FBF6F61B36A9
:1075C00033B201211A220191009219461422A648D1
:1075D0002E6004F0F7FAA44805F0E0FA236850930F
:1075E000509AA34BC8F8002000221A70FDF74ABC3D
:1075F0002368DFF89C8252939E4A529BD8F8001071
:1076000012685B1A93421AD9994B9B491A7896488B
:10761000012A0CBF002201221A701A78B1F9003039
:107620000192392219460092322204F0CBFA8E4898
:1076300005F0B4FA23685393539BC8F800308F4A7F
:107640001378002B3DF41EAC8D4B1B680021013BD1
:107650001170072B3DF616AC01A252F823F000BFC3
:107660004D77000027770000854E0000A7760000C8
:10767000854E0000854E0000854E0000817600009A
:107680007D4B7948B3F90030012439228DE814008C
:107690002824194632223C7004F094FA724805F00E
:1076A0007DFAFDF7EFBB774E6C4B704F32881B684D
:1076B00039681A448A42BDF6E5AB6F4D3280B5F9A0
:1076C000003069484FF0000E392219468DE8044019
:1076D000322204F077FA624B3A6819683388521AFA
:1076E0005C2A40F34986591A5D23561C03FB01F3BB
:1076F00093FBF6F61B3633B2012139220191009239
:107700001946322258482E6004F05CFA564805F0BB
:1077100045FA23685593559A554BC8F80020002226
:107720001A70FDF7AFBB544B4F48B3F9003001243A
:1077300039228DE814002824194632223C7004F0C6
:1077400041FA494805F02AFAFDF79CBB4D4E434AE1
:1077500041484D4933881268008809689A1A4318CD
:107760009A427DF78FAB444D3280B5F900303E48E8
:107770003922002719468DE88400322204F022FACB
:10778000374A3A4B11681A683388521A5C2A41F317
:10779000DD80591A5D23561C03FB01F393FBF6F6BB
:1077A0001B3633B20121392201910092194632224F
:1077B0002D482E6004F006FA2B4805F0EFF92368F7
:1077C0005493549A2A4BC8F8002000221A70FDF7EF
:1077D00059BB2E4E3378002B40F0F0822368DFF83F
:1077E000B0805693234A569BD8F8001012685B1A53
:1077F000934211D91E4B1A78012A0CBF0022012294
:107800001A701878F9F700F9174805F0C7F92368D6
:107810005793579BC8F80030184A1378002B3DF453
:1078200031AB174B1B680021013B1170072B3DF654
:1078300029AB01A252F823F0DF780000D7780000CE
:10784000854E0000B5780000854E0000854E000092
:10785000854E0000957800008E9DFF1F589EFF1FEB
:10786000FC8DFF1F609DFF1F0C9FFF1F5C8AFF1F89
:10787000949EFF1F908DFF1FB49EFF1FF89DFF1F5A
:10788000989EFF1F529EFF1F9C8DFF1F588CFF1F4D
:10789000449EFF1F01232A203B703370F9F73AF909
:1078A000BF4B198888423DF4EDAA2A20F9F726F942
:1078B000FDF7E8BA012328222A2033703A70F9F73D
:1078C00029F9B74B198888423DF4DCAA2A20F9F738
:1078D00015F9FDF7D7BA3D233B70FDF7D3BA012365
:1078E0000A222A2033703A70F9F714F9AC4B198840
:1078F00088423DF4C7AA2A20F9F700F9FDF7C2BA79
:107900005E1A5C2303FB06F393FBF2F61B36FEF7CD
:10791000A5BB5E1A5C2303FB06F393FBF2F61B3652
:10792000FEF7EFBBFCF7C8F89E4A01210023117057
:107930003370A8E42368DFF89C8258939A4A589BD6
:10794000D8F8001012685B1A93421AD9974B9849DD
:107950001A789848012A0CBF002201221A701A785E
:10796000B1F9003001921A2219460092142204F053
:1079700029F9904805F012F923685993599BC8F8E2
:1079800000308D4A1378002B3DF47CAA8B4B1B688A
:107990000021013B1170072B3DF674AA01A252F899
:1079A00023F000BFC77A0000A17A0000854E0000D6
:1079B000EB790000854E0000854E0000854E0000EA
:1079C000C57900007A4B7B48B3F9003001241A22B4
:1079D0008DE814003C24194614223C7004F0F2F89F
:1079E000744805F0DBF8FDF74DBA6D4E744A754FDB
:1079F00033881268D7F800E01A447245BDF642AAEF
:107A00007149724BDFF8D09108681D68D9F80010F1
:107A100093B2CEEB01012A1A91423380644DCEEB32
:107A20000303CCBF02FB03335343694AC8BF013190
:107A300093FBF1F3B5F90010034413604FF0000E0F
:107A40001A220B468DE804405A48142204F0BAF872
:107A5000D9F800103A683388521A5C2A40F36487D8
:107A6000591A5D23561C03FB01F393FBF6F61B36F4
:107A700033B201211A2201910092194614224D4875
:107A80002E6004F09FF84B4805F088F823685B935C
:107A90005B9A464BC8F8002000221A70FDF7F2B935
:107AA000434B4448B3F9003001241A228DE81400F6
:107AB0003C24194614223C7004F084F83D4805F03B
:107AC0006DF8FDF7DFB9364E3D4ADFF80C9133888B
:107AD0001268D9F800509A1AAA427DF7D3A93B4BF5
:107AE000384F3949D7F800E01868096893B2CEEBEF
:107AF0000505421A95423380CEEB030341F3A08380
:107B000002FB03336A1C93FBF2F31944284D304AFD
:107B1000B5F9003011604FF0000E1A2219468DE8B9
:107B200004402448142204F04DF8D9F800103A68B3
:107B30003388521A5C2A41F37A83591A5D23561C02
:107B400003FB01F393FBF6F61B3633B201211A2235
:107B5000019100921946142216482E6004F032F862
:107B6000144805F01BF823685A935A9A0F4BC8F82B
:107B7000002000221A70FDF785B95E1A5C2303FB12
:107B800006F393FBF2F61B36FEF75BBB5E1A5C2333
:107B900003FB06F393FBF2F61B36FEF7C2BB00BFF6
:107BA000FC9EFF1F679DFF1F908DFF1F949EFF1F70
:107BB000609DFF1F0C9FFF1FF89DFF1F989EFF1FDA
:107BC000DC9DFF1F408CFF1F608AFF1F5C8CFF1F26
:107BD000548CFF1F449EFF1FF48DFF1FAF4A137884
:107BE000B3FA83F35B0901201370FAF7A1F9AC4BE8
:107BF000AC4800221A7004F0D1FFAB4A138883F01E
:107C00000803194642201380F8F778FFFDF73AB9C8
:107C1000A64E33781BB1FBF799F900233370A44DBE
:107C20002978002900F086802368DFF8A4825C931D
:107C3000A04A5C9BD8F8001012685B1A934211D9D5
:107C4000974B1A78012A0CBF002201221A7018786B
:107C5000FCF730FE934804F0A1FF23685D935D9B21
:107C6000C8F80030944A1378002B3DF40BA9934BCD
:107C70001B680021013B1170072B3DF603A901A2EF
:107C800052F823F0F9890000C7890000854E0000F2
:107C900091890000854E0000854E0000854E000051
:107CA0005F890000814E3378002B40F0A281844D23
:107CB0002A78002A00F00E812368DFF81482789376
:107CC0007C4A789BD8F8001012685B1A934211D94D
:107CD000734B1A78012A0CBF002201221A701878FF
:107CE000FCF7F0FB6F4804F059FF23687993799B08
:107CF000C8F80030704A1378002B3DF4C3A86F4BCE
:107D00001B680021013B1170072B3DF6BBA801A2A7
:107D100052F823F0098B0000DB8A0000854E00003A
:107D2000A78A0000854E0000854E0000854E0000A9
:107D3000798A0000634D2A78002A00F0B281236816
:107D4000DFF88C8162935B4A629BD8F8000012686E
:107D50001B1A934211D9524B1A78012A16BF0122DD
:107D600019701A701878FBF7CBFB4E4804F016FF19
:107D700023686393639BC8F800304F4A1378002B45
:107D80003DF480A84D4B1B680021013B1170072B6F
:107D90003DF678A801A252F823F000BFA593000099
:107DA00073930000854E000041930000854E000053
:107DB000854E0000854E00000F930000FBF7C0FDCC
:107DC000414A012100231170337007E55E1A5C23DC
:107DD00003FB06F393FBF2F61B36FDF7BDBF5E1AFD
:107DE0005C2303FB06F393FBF2F61B36FEF707B8A2
:107DF0005E1A5C2303FB06F393FBF2F61B36FEF7D9
:107E0000B9BD324D2978002900F0FE802368DFF8E3
:107E1000C08092932749929BD8F8000009681B1AEA
:107E20008B4210D91E4B1978012918BF01221A70F4
:107E30001878F8F709FE1B4804F0B0FE2368939306
:107E4000939BC8F800301C4A1378002B3DF41AA805
:107E50001A4B1B680021013B1170072B3DF612A83D
:107E600001A252F823F000BF859400003B9400006B
:107E7000854E000005940000854E0000854E0000F0
:107E8000854E0000D79300005E1A5C2303FB06F3C7
:107E900093FBF2F61B36FEF7C3BD00BFEA9EFF1F41
:107EA000949EFF1F0C9FFF1FF69EFF1F588CFF1F05
:107EB0005A9DFF1F908DFF1FF89DFF1F989EFF1F6B
:107EC000509EFF1FDC9EFF1F679DFF1F049EFF1F2C
:107ED000449EFF1FB94D297800293DD02368DFF863
:107EE00004837C93B6497C9BD8F8000009681B1A70
:107EF0008B4210D9B34B1978012918BF01221A708F
:107F00001878FAF7B9FDB04804F048FE23687D936D
:107F10007D9BC8F80030AD4A1378002B3CF4B2AF1B
:107F2000AB4B1B680021013B1170072B3CF6AAAF3D
:107F300001A252F823F000BF6D8600003F860000CA
:107F4000854E000009860000854E0000854E000029
:107F5000854E0000DB8500009E4D2A78002A00F047
:107F60001D872368DFF87C828093954A809BD8F830
:107F7000000012681B1A934211D9924B1A78012AF9
:107F800016BF012219701A701878FCF7FFFA8E4894
:107F900004F004FE23688193819BC8F800308B4A6B
:107FA0001378002B3CF46EAF894B1B680021013B1A
:107FB0001170072B3CF666AF01A252F823F000BF08
:107FC0003387000005870000854E0000D186000041
:107FD000854E0000854E0000854E0000A3860000FF
:107FE0005E1A5C2303FB06F393FBF2F61B36FEF7E7
:107FF00054BFFAF7CDFF0023337058E6FAF7EAFFD3
:1080000000233370FCF782BF734D2A78002A00F0FA
:1080100005862368DFF8CC819693694A969BD8F849
:10802000000012681B1A934211D9664B1A78012A74
:1080300016BF012219701A701878F8F723FD6248EC
:1080400004F0ACFD23689793979BC8F800305F4A13
:108050001378002B3CF416AF5D4B1B680021013BED
:108060001170072B3CF60EAF01A252F823F000BFAF
:10807000B18B0000838B0000854E0000E18B000077
:10808000854E0000854E0000854E0000558B000097
:108090005E1A5C2303FB06F393FBF2F61B36FEF736
:1080A0006BBF4E4D297800293CD02368DFF834811E
:1080B00066934349669BD8F8000009681B1A8B42F7
:1080C00010D9404B1978012918BF01221A7018786D
:1080D000FAF7AAFD3C4804F061FD23686793679BAB
:1080E000C8F80030394A1378002B3CF4CBAE384B3B
:1080F0001B680021013B1170072B3CF6C3AE01A2A7
:1081000052F823F0DB88000073880000854E0000E1
:10811000A1880000854E0000854E0000854E0000BD
:10812000678700002E4D2A78002A66D02368DFF882
:10813000B4806A93224A6A9BD8F8000012681B1A1E
:10814000934211D91F4B1A78012A16BF01221970C8
:108150001A701878FCF776FC1B4804F01FFD2368A2
:108160006B936B9BC8F80030184A1378002B3CF4D3
:1081700089AE174B1B680021013B1170072B3CF6A1
:1081800081AE01A252F823F041880000F787000079
:10819000854E0000C3870000854E0000854E00001C
:1081A000854E0000958700005E1A5C2303FB06F3F2
:1081B00093FBF2F61B36FEF782BF00BF589DFF1FF0
:1081C000908DFF1F949EFF1F0C9FFF1FF89DFF1FA8
:1081D000989EFF1F649DFF1FE09DFF1F8C9DFF1F4A
:1081E000379FFF1F449EFF1F5E1A5C2303FB06F3AD
:1081F00093FBF2F61B36FEF7B8BFBA4D297800297B
:108200003CD02368DFF800836E93B7496E9BD8F8A3
:10821000000009681B1A8B4210D9B44B1978012948
:1082200018BF01221A701878FBF7AEFAB04804F0B4
:10823000B5FC23686F936F9BC8F80030AD4A137884
:10824000002B3CF41FAEAC4B1B680021013B1170AE
:10825000072B3CF617AE01A252F823F06985000007
:108260003B850000854E00009B850000854E000088
:10827000854E0000854E00000D8500009F4D23684F
:108280002A78DFF88482002A3AD07293964A729B49
:10829000D8F8000012681B1A934211D9934B1A7830
:1082A000012A16BF012219701A701878FAF77EFB9E
:1082B0008F4804F073FC23687393739BC8F80030F5
:1082C0008C4A1378002B3CF4DDAD8B4B1B680021EE
:1082D000013B1170072B3CF6D5AD01A252F823F0FB
:1082E000B184000083840000854E00004F840000AC
:1082F000854E0000854E0000854E00002184000060
:1083000076937949769BD8F8000009681B1A8B424E
:1083100012D9764B1978012918BF01221A70784AB0
:1083200019781078F8F75AFB714804F037FC236885
:108330007793779BC8F800306E4A1378002B3CF493
:10834000A1AD6D4B1B680021013B1170072B3CF662
:1083500099AD01A252F823F0DF830000D78300001B
:10836000854E000095830000854E0000854E00007C
:10837000854E00008B8300005E1A5C2303FB06F32E
:1083800093FBF2F61B36FFF7B6B901233B7033704F
:10839000FCF778BD5A4C207801287CF673AD00219B
:1083A000F8F71CFB2378514D013BDBB21846012145
:1083B0002370F8F713FB002434238DE818004C4891
:1083C0002C7040230B223F2103F0CAFB484804F0E5
:1083D000E5FBFCF757BDFCF711FCFCF753BD484C1F
:1083E000207805283CF64EAD0021F8F7F7FA2378FF
:1083F0003E4D0133DBB2184601212370F8F7EEFA47
:10840000002434238DE8180039482C7040230B22B7
:108410003F2103F0A5FB364804F0C0FBFCF732BD5A
:108420000120FAF7C3FA314B314800241C7004F0E4
:10843000B5FB30202C70F8F76DFB324B1988884261
:108440003CF420AD3020F8F759FBFCF71BBD0020B1
:10845000FAF7ACFA2B4A1388082B94BF0133002398
:1084600001201380FAF7A2FA204B214800221A704B
:1084700004F094FB23687593759BC8F80030FCF7F3
:1084800001BD0120FAF792FA184B194800241C701C
:1084900004F084FB30202C70F8F73CFB194B198852
:1084A00088423CF4EFAC3020F8F728FBFCF7EABC3C
:1084B0000020FAF77BFA134A1388002B00F087801C
:1084C000013B13800120FAF771FA084B084800229B
:1084D0001A7004F063FB23687493749BC8F800302F
:1084E000FCF7D0BCBA9DFF1F908DFF1F949EFF1F0D
:1084F0000C9FFF1FF89DFF1F989EFF1FF09DFF1F01
:10850000648AFF1FA69DFF1F449EFF1F0120FBF7EB
:108510003BF9C44BC44800241C7004F03FFB2E20E0
:108520002C70F8F7F7FAC14B198888423CF4AAACD2
:108530002E20F8F7E3FAFCF7A5BC0120FBF724F99D
:10854000B84BB94800241C7004F028FB2E202C7076
:10855000F8F7E0FAB54B198888423CF493AC2E202A
:10856000F8F7CCFAFCF78EBC0020FBF70DF9AF4A08
:108570001388002B2ED0013B13800120FBF704F958
:10858000A84BA94800221A7004F008FB23687093D6
:10859000709BC8F80030FCF775BC0020FBF7F4F8BE
:1085A000A24A13881D2B94BF01330023012013809E
:1085B000FBF7EAF89B4B9C4800221A7004F0EEFA95
:1085C00023687193719BC8F80030FCF75BBC0923EA
:1085D000138077E71E231380CFE70120FAF74CFAC8
:1085E000904B914800241C7004F0D8FA1A202C708B
:1085F000F8F790FA8E4B198888423CF443AC1A2065
:10860000F8F77CFAFCF73EBC894D2B880B2B3CF627
:1086100039AC0020FAF730FA2B88012003442B8074
:10862000FAF72AFA7F4B804800221A7004F0B6FA53
:1086300023687F937F9BC8F80030FCF723BC0120A0
:10864000FAF71AFA774B784800241C7004F0A6FA5F
:108650001A202C70F8F75EFA754B198888423CF4A2
:1086600011AC1A20F8F74AFAFCF70CBC704D2B88B5
:10867000002B3CF407AC0020FAF7FEF92B88012010
:10868000013B2B80FAF7F8F9664B674800221A7015
:1086900004F084FA23687E937E9BC8F80030FCF7D0
:1086A000F1BB0120FBF772FF5E4B5F4800241C709A
:1086B00004F074FA1C202C70F8F72CFA5D4B198822
:1086C00088423CF4DFAB1C20F8F718FAFCF7DABB61
:1086D0000020FBF75BFF574A1388032B94BF01333D
:1086E000002301201380FBF751FF4E4B4E48002220
:1086F0001A7004F053FA23688393839BC8F8003000
:10870000FCF7C0BB0120FBF741FF464B4648002465
:108710001C7004F043FA1C202C70F8F7FBF9454B51
:10872000198888423CF4AEAB1C20F8F7E7F9FCF757
:10873000A9BB0020FBF72AFF3E4A1388002B00F05C
:10874000C980013B13800120FBF720FF354B3648E1
:1087500000221A7004F022FA23688293829BC8F8E0
:108760000030FCF78FBB0120FAF75EFA2D4B2E4844
:1087700000241C7004F012FA16202C70F8F7CAF9C5
:108780002D4B198888423CF47DAB1620F8F7B6F9DA
:10879000FCF778BB0120FCF755F9224B2248002456
:1087A0001C7004F0FBF92C202C70F8F7B3F9234B64
:1087B000198888423CF466AB2C20F8F79FF9FCF747
:1087C00061BB0020FCF73EF91C4A13880B2B94BFB9
:1087D0000133002301201380FCF734F9114B1248B8
:1087E00000221A7004F0DAF923686D936D9BC8F8C3
:1087F0000030FCF747BB0120FCF724F9094B0A487D
:1088000000241C7004F0CAF92C202C70F8F782F9AF
:108810000A4B198888423CF435AB2C20F8F76EF9E6
:10882000FCF730BB949EFF1F0C9FFF1FC49EFF1FD1
:10883000D09DFF1FC89DFF1F5C9DFF1FA49EFF1FB3
:108840000020FCF7FFF8BD4A1388002B5DD0013BE8
:1088500013800120FCF7F6F8B94BBA4800221A70D1
:1088600004F09CF923686C936C9BC8F80030FCF70B
:1088700009BB0120FAF7D8F9B14BB24800241C70AB
:1088800004F08CF916202C70F8F744F9AE4B1988D7
:1088900088423CF4F7AA1620F8F730F9FCF7F2BA50
:1088A0000020FAF7C1F9A84A13887E2B94BF013340
:1088B000002301201380FAF7B7F9A14BA148002249
:1088C0001A7004F06BF923686993699BC8F800304B
:1088D000FCF7D8BA0423138035E70020FAF7A4F98F
:1088E000994A1388A3B1013B13800120FAF79CF940
:1088F000934B944800221A7004F050F9236868934F
:10890000689BC8F80030FCF7BDBA0C231380A0E7C1
:108910007F231380E9E75E1A5C2303FB06F393FBD6
:10892000F2F61B36FEF7D7BD5E1A5C2303FB06F397
:1089300093FBF2F61B36FFF79BB85E1A5C2303FB32
:1089400006F393FBF2F61B36FEF73ABE5E1A5C2383
:1089500003FB06F393FBF2F61B36FEF722BF012062
:10896000FBF7A8FF764B774800241C7004F016F93B
:1089700012202C70F8F7CEF8744B198888423CF41A
:1089800081AA1220F8F7BAF8F8F768FCFCF77ABA6F
:108990006E4D2B88092B4FF0000046D8FBF78AFF5D
:1089A0002B88012003442B80FBF784FF644B654830
:1089B00000221A7004F0F2F823686093609BC8F8F4
:1089C0000030FCF75FBA0120FBF774FF5C4B5D4899
:1089D00000241C7004F0E2F812202C70F8F79AF8CA
:1089E0005A4B198888423CF44DAA1220F8F786F8B1
:1089F000F8F734FCFCF746BA544D2E8846B30020F5
:108A0000FBF758FF2B880120013B2B80FBF752FF1F
:108A10004B4B4C4800221A7004F0C0F823685E9358
:108A20005E9BC8F80030FCF72DBAFBF743FF002629
:108A300001202E80FBF73EFF414B42481E7004F0A0
:108A4000ADF823686193619BC8F80030FCF71ABA4F
:108A50003046FBF72FFF0A2301202B80FBF72AFF6C
:108A6000374B38481E7004F099F823685F935F9B7A
:108A7000C8F80030FCF706BA0120FBF723FD304BA5
:108A8000304800241C7004F089F818202C70F8F786
:108A900041F82F4B198888423CF4F4A91820F8F7C4
:108AA0002DF8FCF7EFB90020FBF70CFD284A1388DE
:108AB000012B94BF0133002301201380FBF702FD3B
:108AC0001F4B204800221A7004F068F823687B933B
:108AD0007B9BC8F80030FCF7D5B90120FBF7F2FC0E
:108AE000174B184800241C7004F058F818202C70FC
:108AF000F8F710F8164B198888423CF4C3A91820DF
:108B0000F7F7FCFFFCF7BEB90020FBF7DBFC104ACF
:108B10001388002B7FD0013B13800120FBF7D2FC90
:108B2000074B084800221A7004F038F823687A933B
:108B30007A9BC8F80030FCF7A5B900BFA49EFF1FC0
:108B4000949EFF1F0C9FFF1F5C9DFF1F9C9EFF1F9D
:108B5000249EFF1F0120F7F795FFB14BB148002479
:108B60001C7004F01BF852202C70F7F7D3FFAE4BAB
:108B7000198888423CF486A95220F7F7BFFFFCF71A
:108B800081B90120F7F77EFFA54BA64800241C7091
:108B900004F004F852202C70F7F7BCFFA24B1988A0
:108BA00088423CF46FA95220F7F7A8FFFCF76AB996
:108BB0000020F7F767FF9C4A13880BB1013B138035
:108BC0000120F7F75FFF964B964800221A7003F0DA
:108BD000E5FF23689893989BC8F80030FCF752B9DA
:108BE0000020F7F74FFF904A1388032B98BF0133FB
:108BF0004FF0010098BF1380F7F744FF884B894876
:108C000000221A7003F0CAFF23689993999BC8F851
:108C10000030FCF737B9022313807EE7834D2978B3
:108C200000293DD02368DFF820829A9380499A9BDF
:108C3000D8F8000009681B1A8B4210D9784B1978B4
:108C4000012918BF01221A701878F7F739FF754803
:108C500003F0A4FF23689B939B9BC8F80030754AE0
:108C60001378002B3CF40EA9734B1B680021013BC9
:108C70001170072B3CF606A901A252F823F000BFA1
:108C800015960000E7950000854E0000B1950000A4
:108C9000854E0000854E0000854E00008395000043
:108CA000664D23682A78DFF8A081002A3AD09E9387
:108CB0005F4A9E9BD8F8000012681B1A934211D994
:108CC000574B1A78012A16BF012219701A701878AA
:108CD000FAF774FC534803F061FF23689F939F9B4E
:108CE000C8F80030534A1378002B3CF4CBA8524B01
:108CF0001B680021013B1170072B3CF6C3A801A2A1
:108D000052F823F0DD920000AF920000854E000083
:108D10007D920000854E0000854E0000854E0000CB
:108D20004F920000A2934249A29BD8F80000096824
:108D30001B1A8B4212D93A4B1978012918BF01220C
:108D40001A703F4A19781078F7F748FE354803F053
:108D500025FF2368A393A39BC8F80030354A1378F6
:108D6000002B3CF48FA8344B1B680021013B117091
:108D7000072B3CF687A801A252F823F0ED910000E2
:108D8000E5910000854E0000A3910000854E000093
:108D9000854E0000854E000097910000294D2978EE
:108DA000002953D02368DFF8A08084932049849B56
:108DB000D8F8000009681B1A8B4210D9184B197893
:108DC000012918BF01221A701878FAF74BFD1548CF
:108DD00003F0E4FE23688593859BC8F80030154AAC
:108DE0001378002B3CF44EA8134B1B680021013B69
:108DF0001170072B3CF646A801A252F823F000BFE1
:108E0000619100000B910000854E0000D59000009C
:108E1000854E0000854E0000854E0000A7900000A2
:108E2000949EFF1F0C9FFF1F948AFF1FE89EFF1F49
:108E3000908DFF1FF89DFF1F989EFF1FE99EFF1F4B
:108E4000488AFF1FC59DFF1F449EFF1FBA4D236820
:108E50002A78DFF80883002A3AD08893B74A889B9B
:108E6000D8F8000012681B1A934211D9B44B1A7833
:108E7000012A16BF012219701A701878FBF7ACFA94
:108E8000B04803F08BFE23688993899BC8F80030B3
:108E9000AD4A1378002B3BF4F5AFAC4B1B680021B7
:108EA000013B1170072B3BF6EDAF01A252F823F006
:108EB0007190000043900000854E0000778F000005
:108EC000854E0000854E0000854E0000498F000051
:108ED0008C939A498C9BD8F8000009681B1A8B4226
:108EE00012D9974B1978012918BF01221A70984A94
:108EF00019781078F7F772FD924803F04FFE236857
:108F00008D938D9BC8F800308F4A1378002B3BF46B
:108F1000B9AF8E4B1B680021013B1170072B3BF64C
:108F2000B1AF01A252F823F001900000F98F0000C8
:108F3000854E0000B78F0000854E0000854E000072
:108F4000854E0000AD8F00000120FBF745FA7C4BF9
:108F50007C4800241C7003F021FE32202C70F7F7AF
:108F6000D9FD7C4B198888423BF48CAF3220F7F74F
:108F7000C5FDFBF787BF774D2B88172B3BF682AFDC
:108F80000020FBF729FA2B88012003442B80FBF7F4
:108F900023FA6B4B6B4800221A7003F0FFFD236825
:108FA0008B938B9BC8F80030FBF76CBF01233B70A1
:108FB0003370FBF767BF664C207801287BF662AF01
:108FC0000021F7F70BFD23785D4D013BDBB218461E
:108FD00001212370F7F702FD002434238DE81800E7
:108FE00058482C7040230B223F2102F0B9FD554810
:108FF00003F0D4FDFBF746BFFBF756FBFBF742BF80
:10900000534C207805283BF63DAF0021F7F7E6FCEE
:1090100023784B4D0133DBB2184601212370F7F75B
:10902000DDFC002434238DE8180046482C704023D2
:109030000B223F2102F094FD424803F0AFFDFBF705
:1090400021BF0120FBF7C8F93D4B3E4800241C70AE
:1090500003F0A4FD32202C70F7F75CFD3D4B19881E
:1090600088423BF40FAF3220F7F748FDFBF70ABF09
:10907000384D2B88002B3BF405AF0020FBF7ACF9F3
:109080002B880120013B2B80FBF7A6F92C4B2D48A8
:1090900000221A7003F082FD23688A938A9BC8F825
:1090A0000030FBF7EFBE0120FAF7DCFB244B25482C
:1090B00000241C7003F072FD20202C70F7F72AFDAD
:1090C000254B198888423BF4DDAE2020F7F716FDCA
:1090D000FBF7D8BE204D2B88452B3BF6D3AE0020A6
:1090E000FAF7C0FB2B88012003442B80FAF7BAFB68
:1090F000134B144800221A7003F050FD2368879325
:10910000879BC8F80030FBF7BDBE0120FAF7AAFB29
:109110000B4B0C4800241C7003F040FD20202C70E9
:10912000F7F7F8FC0C4B198888423BF4ABAE2020D3
:10913000F7F7E4FCFBF7A6BE969DFF1F908DFF1F7F
:10914000949EFF1F0C9FFF1FF89DFF1F989EFF1FFF
:10915000548AFF1FD69EFF1FE69EFF1F449EFF1FDF
:10916000C14D2B88002B3BF48DAE0020FAF77AFB23
:109170002B880120013B2B80FAF774FBBB4BBC48CA
:1091800000221A7003F00AFD23688693869BC8F8B4
:109190000030FBF777BE5A2201233A703370FBF799
:1091A00071BEB44C207801287BF66CAE0021F7F735
:1091B00015FC2378AD4D013BDBB21846012123702D
:1091C000F7F70CFC002434238DE81800A8482C7015
:1091D00040230B223F2102F0C3FCA54803F0DEFC34
:1091E000FBF750BEFAF748FAFBF74CBEA14C2078CB
:1091F00004283BF647AE0021F7F7F0FB23789B4DA0
:109200000133DBB2184601212370F7F7E7FB002496
:1092100034238DE8180096482C7040230B223F2100
:1092200002F09EFC924803F0B9FCFBF72BBE5E1ADD
:109230005C2303FB06F393FBF2F61B36FEF785BCBB
:1092400002FB03F393FBF5F21144FEF75FBC012030
:10925000FAF7B4F9854B864800241C7003F09EFC95
:1092600056202C70F7F756FC834B198888423BF444
:1092700009AE5620F7F742FCFBF704BE0020FAF7D0
:109280009DF97D4A1388B3FA83F35B0901201380AB
:10929000FAF794F9754B764800221A7003F07EFCB9
:1092A0002368A193A19BC8F80030FBF7EBBD012018
:1092B000FAF784F96D4B6E4800241C7003F06EFCC5
:1092C00056202C70F7F726FC6B4B198888423BF42C
:1092D000D9AD5620F7F712FCFBF7D4BD0020FAF702
:1092E0006DF9654A1388B3FA83F35B090120138093
:1092F000FAF764F95D4B5E4800221A7003F04EFCE9
:109300002368A093A09BC8F80030FBF7BBBD0120E9
:10931000FAF7F6F8554B564800241C7003F03EFC53
:1093200014202C70F7F7F6FB544B198888423BF455
:10933000A9AD1420F7F7E2FBF7F790FFFBF7A2BD0A
:109340000020FAF7DDF84D4A1388B3FA83F35B097E
:1093500001201380FAF7D4F8444B454800221A70D4
:1093600003F01CFC23686593659BC8F80030FBF78D
:1093700089BD0120FAF7C4F83C4B3D4800241C701D
:1093800003F00CFC14202C70F7F7C4FB3B4B19883E
:1093900088423BF477AD1420F7F7B0FBF7F75EFF98
:1093A000FBF770BD0020FAF7ABF8344A1388B3FA24
:1093B00083F35B0901201380FAF7A2F82B4B2C48AA
:1093C00000221A7003F0EAFB23686493649BC8F8D8
:1093D0000030FBF757BD0120F7F736FB234B24483D
:1093E00000241C7003F0DAFB50202C70F7F792FB7E
:1093F000234B198888423BF445AD5020F7F77EFB9C
:10940000FBF740BD1E4D2B880B2B3BF63BAD0020E0
:10941000F7F71AFB2B88012003442B80F7F714FB86
:10942000124B134800221A7003F0B8FB236895937F
:10943000959BC8F80030FBF725BD0120F7F704FB2A
:109440000A4B0B4800241C7003F0A8FB50202C7022
:10945000F7F760FB0A4B198888423BF413AD5020A4
:10946000F7F74CFBFBF70EBDE69EFF1F949EFF1F18
:109470000C9FFF1F488AFF1FFA9DFF1F169EFF1FAC
:10948000B88CFF1F714D2B88012B7BF6FBAC0020A5
:10949000F7F7DAFA2B880120013B2B80F7F7D4FA93
:1094A0006B4B6C4800221A7003F078FB236894938E
:1094B000949BC8F80030FBF7E5BC0120F9F74EFBA0
:1094C000634B644800241C7003F068FB1E202C7062
:1094D000F7F720FB604B198888423BF4D3AC1E2081
:1094E000F7F70CFBFBF7CEBC5B4D2B88082B3BF64C
:1094F000C9AC0020F9F732FB2B88012003442B80F4
:10950000F9F72CFB524B534800221A7003F046FB2C
:1095100023689193919BC8F80030FBF7B3BC0120FE
:10952000F9F71CFB4A4B4B4800241C7003F036FB38
:109530001E202C70F7F7EEFA474B198888423BF44F
:10954000A1AC1E20F7F7DAFAFBF79CBC424D2B8842
:10955000002B3BF497AC0020F9F700FB2B8801208F
:10956000013B2B80F9F7FAFA394B3A4800221A707E
:1095700003F014FB23689093909BC8F80030FBF72E
:1095800081BC0120F7F79CFA314B324800241C7053
:1095900003F004FB54202C70F7F7BCFA2F4B19880A
:1095A00088423BF46FAC5420F7F7A8FAFBF76ABC8B
:1095B0002A4D2B881D2B3BF665AC0020F7F780FA6F
:1095C0002B88012003442B80F7F77AFA204B21489F
:1095D00000221A7003F0E2FA23689D939D9BC8F85D
:1095E0000030FBF74FBC0120F7F76AFA184B194817
:1095F00000241C7003F0D2FA54202C70F7F78AFA7A
:10960000164B198888423BF43DAC5420F7F776FAA4
:10961000FBF738BC114D2B88012B7BF633AC0020B7
:10962000F7F74EFA2B880120013B2B80F7F748FA19
:10963000074B084800221A7003F0B0FA23689C9385
:109640009C9BC8F80030FBF71DBC00BFB88CFF1F07
:10965000949EFF1F0C9FFF1FBC9DFF1FBA8CFF1F16
:109660002DE9F04F0E2093B003F010FD07F0EEF956
:1096700001469348934F944E02F024F9904802F02B
:10968000F7F807F013FC3D6880F30C00012D306003
:1096900000F0B980022DDFF89CB200F0D181032DDB
:1096A00000F04F82894C8A4DDFF88C92DFF88C8273
:1096B0002368884F0E930E9B3A689B1A022B1ED983
:1096C000DFF87CA29AF80030002B00F03B83824B3D
:1096D0001A78002A0CBF012200221A7000F02D8394
:1096E0009AF80030002B40F03083F7F7B5FEF6F71C
:1096F000E5FFF7F7CFFD23680F930F9B3B602368CF
:10970000764F1093764A109B396812685B1A934221
:1097100061D82968734B74481A78C9F800102A2355
:10972000183903FB01F10160002A51D06F4A136818
:10973000994240F374816E480068D0F17F0048BFC1
:10974000033003EBA0030133994280F2768111606C
:10975000684B1B68A92202FB03F3002BBCBF03F577
:109760007F533F339B13543B1944282081F30C0152
:1097700004F028F93368BBF80000B8F800208342F1
:109780001FDA0024111A40F60B639942C3BF40F65A
:109790000C62013102FB04F3634393FBF1F000F52B
:1097A000FA70F6F79DFE0146142004F00BF9002034
:1097B00005F000FB0028FAD1FBF7BEFA13B0BDE8B4
:1097C000F08F9342D4BFC0EB0304C0EB0204D9E78F
:1097D000464B1960BCE7F8F74FF8474B1B7823B9A5
:1097E000464B1B78002B00F001820D2004F080FA1C
:1097F000B0FA80F149090D2004F074FA236811933E
:10980000119B3B6085E7DFF83C913D4AB9F8003099
:109810001178994209D0DBB21370002B00F050820E
:10982000102BA8BF1023374A1360DFF81C81364A7B
:10983000B8F800301178994204D0344C21780029CE
:1098400040F02E82DFF8ECB0204CBBF800308342B1
:1098500080F2C68122682E4B099209992D4A19601F
:10986000022310603B602C4B187800286ED12B4BE4
:109870001B78002B6AD12A4B1F68002003F006FCDE
:10988000A7F21F37874202DC264B00221A70002005
:1098900004F056FC244B254D1A682978244F904239
:1098A000D4BF002301238B423B7002D0904200F3CF
:1098B00085832B70DFF88090054DDFF88080F7E618
:1098C000749EFF1FD09EFF1FB89EFF1F489FFF1F63
:1098D000009FFF1F4C9EFF1FC49DFF1F089EFF1F80
:1098E000F88BFF1FEA9DFF1F349EFF1F9C9DFF1FEB
:1098F000F09EFF1F988DFF1FBC9EFF1FB19EFF1F94
:10990000399EFF1F009EFF1FF29DFF1F959DFF1FA9
:10991000EC9DFF1F689EFF1FBE9DFF1F189EFF1F2F
:109920006C9DFF1FE59EFF1F548CFF1F599DFF1F5D
:10993000BB9DFF1F1A9EFF1F209EFF1FF49EFF1F4F
:10994000EA9EFF1F649EFF1F709EFF1FB84BDFF84B
:1099500040A31F88BAF80020DFF838E31744DEF888
:1099600000207F109742B34A05DA11688F4202DA6D
:10997000002840F059830293AF4B03921F4600200A
:10998000CDF810E0019303F081FB3F68029B039A3E
:10999000A7F5487E704580F29581A8480078002898
:1099A00000F090811888DDF810E0BAF80030DEF899
:1099B0000010126803445B108B4280F2898193424D
:1099C00040F38681F6F7DCFE9D490A68531C002BA4
:1099D00040F31985802B00F315859A4D9A482F88FE
:1099E0009A4D00882D680B603918B5EB610FC1F2F4
:1099F0002980A2F148030F2B00F29C81473A0021F5
:109A00000D20A9F8002004F06DF9962004F0A6F9C5
:109A100001210D2004F066F9019B1F682DE7BFF6B8
:109A200096AE8B480068D0F17F0048BF03308010AD
:109A300001301B1A99423FF78AAE1360194687E638
:109A4000BBF80030834280F2EB80824C824923686D
:109A50000A93824A0A9B096812885B1A934202D8C9
:109A6000002A7FF420AEF6F78BFE7D4A336811683A
:109A7000BBF80020DFF820828B42B8BF0B469A4229
:109A8000B8F80000774940F3FD85774B09881A60E4
:109A9000002900F00A83754B05931970744DF7F790
:109AA00075FC28687F2840F3E985724B7F3883FB7B
:109AB0000032C317C3EB620303EB4303A0EB830045
:109AC00073306D4B02931B882860002B40F0928707
:109AD0006A4B01931B78002B00F0EE83684B1A460B
:109AE0001B78002B00F0E8830394CDF81080DFF89A
:109AF0009891059CA8464FF0000A15460BE003F12B
:109B00007300C0B22178F7F729FE2B780AF1010A19
:109B1000534540F3CD83D8F8003059F8040F554A27
:109B20001844A0F17F0382FB032ED917C1EB6E010D
:109B300001EB41017F28A3EB8103E0DCF6F7BEFCDB
:109B4000DFE7BBF80030834240F302814D4B1B78C6
:109B5000002B40F0FD80DFF844A19AF800007F2838
:109B600000F39382F6F7AAFC434B02931B88C0B222
:109B70008AF80000002B40F01987404B01931B78B6
:109B8000002B00F0D1823E4B1A461B78002B00F0D0
:109B9000CB823D4C374D4FF0000891460BE003F16E
:109BA0007300C0B2F6F7E8FF99F8003008F1010839
:109BB000434540F3B98254F8043F9AF80000184432
:109BC000A0F17F0385FB0321DA17C2EB610202EBF0
:109BD00042027F28A3EB8203E1DCF6F76FFCE0E7AB
:109BE000284B1B78002B3FF43EAE33E6234B1B780B
:109BF000002B7FF4FAAD254B1B78002B7FF4F5ADDD
:109C0000204B1B78002B7FF4F0AD0D2004F070F892
:109C100000287FF4F3AD01210D2004F063F8EDE599
:109C2000184B1B78002B7FF410AF01233B6039E504
:109C3000B89DFF1F089FFF1F6C9DFF1F189EFF1FF1
:109C4000F49DFF1F8E9DFF1F529EFF1FC09DFF1F93
:109C5000F09EFF1F489FFF1FEC9DFF1FC49EFF1F2C
:109C6000689EFF1F5C9DFF1FE09EFF1FFC9DFF1F66
:109C7000009FFF1FABAAAA2AC69DFF1FEB9EFF1FD6
:109C8000008BFF1FA49DFF1FD88AFF1F5B9DFF1F36
:109C9000309EFF1FCC9DFF1FF49EFF1FB09EFF1F35
:109CA000DBB218461370F6F745FFA84BA84A306898
:109CB000194600231370A74A23700B701370C1E577
:109CC0002B46B0E51988BAF8003012680B445B10D7
:109CD0009342BFF6D2AD002003F0D8F9019B1F6874
:109CE000A7F548739842BFF6C8AD9B4B1A78002A77
:109CF0007FF4C3AD994F01251D70F6F741FD3B7808
:109D0000002B40F0DF84964B1B78002B00F0A586DB
:109D1000944B1B78002B00F02287934B1B784BB998
:109D2000924B1B7833B1B8F80030914A0A3BA8F83F
:109D300000301570019B1F689FE5F6F7ADFFF7F740
:109D4000C3FCD8E4F7F722FBC1E4F7F71FFBCCE430
:109D5000884DDFF85C92F6F713FD2868D9F80030DB
:109D6000984200F08084844C844B22680B920B9ABA
:109D70001A6023680C9382490C9B09889B1A8B42BA
:109D800040F2D4807F2840F375847E4B7F3883FB7C
:109D90000032C317C3EB620303EB4303A0EB830062
:109DA0007330DFF810A29AF80070874200F0BE808E
:109DB000754B1988002900F0C184DFF8FC817F2FE2
:109DC00040F3CD856F48A7F17F0280FB0230D317A7
:109DD000C3EB600000EB4000A2EB800073305B4BF4
:109DE00001931B78C0B28AF80000002B40F0EB848E
:109DF000584B04931B78002B40F06686634B03930B
:109E00001B78002B40F0D186614B0293039B1B789B
:109E100083B3604B9AF800001B6818447F2840F316
:109E20006F86584B7F3883FB0032C317C3EB620346
:109E300003EB4303A0EB83007330C0B2F6F79CFE44
:109E4000554A564B12789AF8000053F822301844BD
:109E50007F2840F351864B4B7F3883FB0032C3177A
:109E6000C3EB620303EB4303A0EB83007330C0B288
:109E7000F6F782FE019B1B78002B00F0C285029B47
:109E8000434F1B880593002B00F0278628687F2806
:109E900040F361853B4B7F3883FB0032C317C3EB34
:109EA000620303EB4303A0EB83007330059B286040
:109EB000002B40F0EA85019B1B78002B00F0D2823A
:109EC000374B1A461B78002B00F0CC82354B3649B5
:109ED00005940027CDF818B0CDF81C801C46B84674
:109EE0008B462F4615460CE003F17300C0B29BF879
:109EF0000010F7F733FC2B7808F10108434540F3D5
:109F0000AB823B6854F8040F1E4A1844A0F17F034B
:109F100082FB032ED917C1EB6E0101EB41017F28B3
:109F2000A3EB8103E0DCF6F7C9FADFE7DFF888800E
:109F3000BBF8002033689A42BFF6BAAB23680D9392
:109F40001A4B0D9A1A60FFF7B3BB00BFEB9EFF1FC1
:109F5000B19EFF1F5B9DFF1FE59EFF1F489EFF1FD9
:109F6000CC9EFF1F349FFF1F359FFF1F369FFF1F93
:109F7000959DFF1F009FFF1F489FFF1F6C9EFF1FA7
:109F8000E69EFF1FABAAAA2A5C9DFF1FBC9EFF1F77
:109F9000C69DFF1F048BFF1FFD9DFF1F448CFF1FED
:109FA000008BFF1FD88AFF1FFC9DFF1F449EFF1FD1
:109FB000209EFF1FB09EFF1FF49EFF1FF6F7E0FBE1
:109FC000A34B1978002932D1A24B1B7843B1A24A86
:109FD00001921278002A00F0ED84019800220270AC
:109FE0009E4A1278002A00F021839D4B0493194663
:109FF0001B78002B40F0D5849A4A9B481278037056
:10A00000012303900B70002A00F02A83924B974A99
:10A01000019300211170019A3B781170039F049AFB
:10A0200001203870117044E4914B0193CAE48F4AC7
:10A0300092F800C0BCF1000F40F0CD84864801903A
:10A040008948844B039084481B7880F800C0864878
:10A050004FF0010E80F800C082F800E0002B40F0C5
:10A06000AC847E4B1B78002BBFD17E4B1B78002B22
:10A0700000F0F6827C4B03931B78002B00F0F585F3
:10A0800003993B7800220A7013E4A3F155337F381B
:10A0900003F1004383FB0032C317C3EB620303EBFE
:10A0A0004303A0EB830073305EE513468342D4BFC5
:10A0B000C2EB0303C2EB0003821AB2F5804FAABFC2
:10A0C0009B03C3EB8333013293FBF2F0F6F708FAFC
:10A0D000C0F3C61006F0BAFC664B0546188806F0B9
:10A0E000B5FC65498146284606F004FD0146484610
:10A0F00006F000FD294606F0F5FB4FF07E510546BF
:10A1000006F096FE002840F027855C49284606F0B8
:10A11000ADFE002840F01B85284606F0EDFEC0B2DB
:10A12000574B05931870B9E44D4B1B78002B45D065
:10A130009AF80030A3F10C007F2840F35784514A6D
:10A140008B3B82FB0321DA17C2EB610202EB420276
:10A15000A3EB820303F17300C0B2F6F70DFD019B80
:10A160001B785BB3484B1A461B783BB3474C454DB5
:10A170004FF0000891460AE003F17300C0B2F6F711
:10A18000FBFC99F8003008F10108434516DD54F84E
:10A19000043F9AF800201A44A2F18B0385FB0310B8
:10A1A000D917C1EB6001A2F10C0001EB41017F283E
:10A1B000A3EB8103E0DCF6F781F9DFE72A4B1B789C
:10A1C00083B3334B9AF800001B6818447F2840F390
:10A1D00009842C4B7F3883FB0032C317C3EB620327
:10A1E00003EB4303A0EB83007330C0B2F6F7C4FC6B
:10A1F000284A294B12789AF8000053F82230184464
:10A200007F2840F3EC831F4B7F3883FB0032C3175A
:10A21000C3EB620303EB4303A0EB83007330C0B2D4
:10A22000F6F7AAFC029B1B88002B00F0B5830F4BAE
:10A230001B78002B40F0AB83184B194C194DDFF8FD
:10A240006890DFF8688000221A6001233B606FE6A7
:10A25000369FFF1FDD9EFF1FEB9EFF1FCC9EFF1F43
:10A260005B9DFF1F949DFF1FBC9EFF1FB19EFF1FA4
:10A270006C9DFF1FA69DFF1FCDCCCC3D0000FE4274
:10A28000FC9DFF1FABAAAA2A008BFF1FD88AFF1FC5
:10A29000048BFF1FFD9DFF1F448CFF1FE09EFF1FCF
:10A2A000489FFF1F009FFF1F209EFF1FF49EFF1F60
:10A2B0004546039CDDF81080954B1B78002B40F041
:10A2C000B6832A68934B1B78002B51D0A2F10C0067
:10A2D0007F2840F3BF839049A2F18B0381FB0321C8
:10A2E000DA17C2EB610202EB4202A3EB820303F135
:10A2F0007300059BC0B21978F7F730FA019B1B7801
:10A30000ABB3864B1A461B788BB30194CDF80C8007
:10A31000DFF83C92059CA8464FF0000A15460AE07B
:10A3200003F17300C0B22178F7F718FA2B780AF11D
:10A33000010A534517DDD8F8003059F8041F764A52
:10A340001944A1F18B03D81782FB032EC0EB6E0ECC
:10A35000A1F10C000EEB4E0E7F28A3EB8E03DFDC89
:10A36000F6F7ACF8DEE74546019CDDF80C802A687C
:10A370006B4B1B78002B38D06A4B1B68D0187F289A
:10A3800040F36583644B7F3883FB0032C317C3EB14
:10A39000620303EB4303A0EB83007330059BC0B261
:10A3A0001978F7F7DBF960490B78022B9ABF5A1C32
:10A3B000D2B200220A705D492B6851F8220018447D
:10A3C0007F2840F34183544B7F3883FB0032C3170F
:10A3D000C3EB620303EB4303A0EB83007330059BE5
:10A3E000C0B21978F7F7BAF92A68029B1B88002BCC
:10A3F00000F016834E4BDFF85C911A7003233B602C
:10A40000FFF756B980254B4A4B4B10884B4A1B88A7
:10A4100012680D600344B2EB630FBFF68BAC484B80
:10A420001978002940F0A082B8F80030454AAB42C4
:10A430003FF480AC444B158001250D201D7003F0C6
:10A4400051FC962003F08AFC29460D2003F04AFCBB
:10A45000019B1F68FFF711BA059CDDF818B0DDF805
:10A460001C803D46049B1B78002B7AD02B68A3F1FF
:10A470000C007F2840F3578327488B3B80FB032049
:10A48000DA17C2EB600000EB4000A3EB800303F19E
:10A4900073002E4B05931978C0B2F7F75FF9019A54
:10A4A0001378002B5DD01D4A13781146002B58D02D
:10A4B000274A0694CDF81C800027DDF81480CDF8DB
:10A4C0001490144689460BE003F17300C0B298F86B
:10A4D0000010F7F743F999F800300137BB423BDD34
:10A4E0002B6854F8041F0C4A1944A1F18B03D817A8
:10A4F00082FB032EC0EB6E0EA1F10C000EEB4E0E94
:10A500007F28A3EB8E03DFDCF5F7D8FFDEE700BF83
:10A51000B19EFF1F5B9DFF1FABAAAA2A008BFF1FE6
:10A52000BC9EFF1F048BFF1FFD9DFF1F448CFF1F60
:10A53000B09EFF1F8E9DFF1F529EFF1FC09DFF1FDD
:10A54000949DFF1F709EFF1F959DFF1FFC9DFF1F89
:10A55000D88AFF1F209EFF1F069CDDF81C80DDF8B7
:10A560001490039B1B78002B39D0B14B28681B68D3
:10A5700018447F2840F39982AE4B7F3883FB00322A
:10A58000C317C3EB620303EB4303A0EB83007330F9
:10A59000A94B05931978C0B2F7F7E0F8A7490B78F3
:10A5A000022B9ABF5A1CD2B200220A70A4492B680F
:10A5B00051F8220018447F2840F374829D4B7F3865
:10A5C00083FB0032C317C3EB620303EB4303A0EB2F
:10A5D00083007330059BC0B21978F7F7BFF8029B70
:10A5E0001B88002B00F05882019B1B783BB9049B11
:10A5F0001B7823B9039B1B78002B00F03D83914B04
:10A600001B78002B34D090480378082B30D88F4922
:10A610002A6809688E4F0133DBB203F1FF3E511AFD
:10A6200047F82E1003708AF8002081E400297FF497
:10A630001CAD002B7FF419AD8649874891F800E0E6
:10A64000864904918649039184497E4A0B70844966
:10A650000190137003700B70BEF1000F7FF4D9AC42
:10A660003B78FFF726B97F4B7F4C1A68FFF781BB19
:10A670002A68D8E7F5F722FFFFF793BBF5F71EFF2F
:10A68000FFF71FBA794D09888342A8BF03462B60A4
:10A6900000297FF400AA9A42C8BF0B463FF70CADD1
:10A6A00004E5734B1B78002B7FF444AB714B724A6B
:10A6B0001B78243B83F3470319465B201360F6F7AE
:10A6C0008BFD3B78032B7FF435ABDFF8DC8198F80A
:10A6D0000020002A40F0B282684F3B78002B40F007
:10A6E000A182634D2B78002B40F09082644B1B7845
:10A6F000002B40F07F82634A1380634B1B78002B52
:10A7000040F0A782614B7F221A8098F80030002B1E
:10A710007FF410AB3B78002B7FF40CAB2B78002B35
:10A720007FF408AB5A4A7F2107201380F6F754FDC7
:10A730007F210B20F6F750FDFFF7FCBA4B4BBBF81F
:10A7400000001B68DFF864818342B8F8002080F2C3
:10A75000CC810B46101AB0F5804FAABF9B03C3EB08
:10A760008333013093FBF0F0F5F7BAFEC0F3C61067
:10A7700006F06CF9474B0190188806F067F94649D6
:10A780000290019806F0B6F9029B0146184606F0C1
:10A79000B1F9019906F0A6F84FF07E51019006F04C
:10A7A00047FB002840F008823C49019806F05EFB18
:10A7B000002840F0CF81019806F09EFBC0B21E4BEE
:10A7C0001870FFF7FCBA364B02931B88002B40F041
:10A7D0006F81224B0493224B03931B4B1A461B7829
:10A7E000002B67D02F4B0594069500271C46154675
:10A7F00008E003F17300C0B2F6F7BEF92B78013719
:10A80000BB4255DD54F8043F9AF80000094A184449
:10A81000A0F17F0382FB032ED917C1EB6E0101EB80
:10A8200041017F28A3EB8103E3DCF5F747FEE2E774
:10A83000048BFF1FABAAAA2AFC9DFF1FFD9DFF1FD3
:10A84000448CFF1FB19EFF1F008BFF1F989DFF1FB1
:10A85000DC8AFF1F949DFF1FEB9EFF1F5B9DFF1F68
:10A86000BC9EFF1F6C9EFF1F489FFF1FE09EFF1FA7
:10A87000369FFF1FFE9EFF1FB49DFF1F359FFF1FCA
:10A88000349FFF1F169EFF1FDD9EFF1F5C9DFF1F55
:10A890009C9EFF1FA69DFF1FCDCCCC3D0000FE421D
:10A8A000C69DFF1FD88AFF1FCC9EFF1FF49EFF1F6F
:10A8B000059C069D049B1B78002B3FF4A7AA9AF8E1
:10A8C0000030A3F10C007F2840F31E81BB488B3B76
:10A8D00080FB0320DA17C2EB600000EB4000A3EB23
:10A8E000800303F17300C0B2F6F746F9019B1B78B1
:10A8F000002B00F00C81B24B1A461B78002B00F0A5
:10A90000C581B04B0594002706951C463D46174669
:10A9100009E003F17300C0B2F6F72EF93B78013578
:10A92000AB4240F3108154F8043F9AF80010A34A58
:10A930001944A1F18B03D81782FB032EC0EB6E0ED6
:10A94000A1F10C000EEB4E0E7F28A3EB8E03E0DC92
:10A95000F5F7B4FDDFE7F5F7B1FDFFF7A7BA384625
:10A96000F5F7ACFDFFF73BBA4B2D00F3DF80243D3C
:10A97000002DB8F8003040F38481AB423FF4DAA9EF
:10A98000ADB2914BA8F800500125002155E50021FA
:10A990004020F6F721FC4FE49AF80000F6F7ECF8B7
:10A9A00045E4049A00231370FFF75FBBF6F7E4F861
:10A9B000FFF7E3B88548864A03904FF0000C82F811
:10A9C00000C00198039A4FF0010E80F800E082F871
:10A9D00000C0FFF705BB00231370FFF7F5BAF5F7CA
:10A9E0006DFD1CE4F5F76AFDFFF7FFBBF5F766FDAB
:10A9F000FFF7B2BB059BC0B21978F6F7AFFEFFF7C1
:10AA000067B8049B1B78002B7FF439AA039B1B7843
:10AA1000002B7FF434AA029B1B880593FFF736BAFC
:10AA2000059BD0B21978F6F799FE2A68E2E47F21F7
:10AA30004020F6F7D1FB6749614B2A680A60002184
:10AA400019703FE41D46EAE4F5F738FDC7E4F5F771
:10AA500035FDA3E4F5F732FD4BE45F4B1B78002B8B
:10AA600000F090805D4B1B78002B7FF463A95C4B5A
:10AA70001B78002B3FF45EA9B8F80030524A0A3325
:10AA8000A8F800301570FFF755B9564BC0B21978C9
:10AA9000F6F764FEFFF70FBA524B28781978F6F7ED
:10AAA0005DFEA1E5F5F70AFD94E5F5F707FD6FE515
:10AAB0004D4B0493454B0393F6F75EF8019B1B78CF
:10AAC000002B7FF48AAEF5E6484B02931B88002BDF
:10AAD00040F0E3803D4B0393F1E69AF80000F6F76F
:10AAE0004BF83B880593FFF7D1B99342D4BFC0EB35
:10AAF0000303C0EB02032DE6F5F7E0FCFFF7B7B95F
:10AB0000F5F7DCFCFFF799B9F5F7D8FCEBE6039B0A
:10AB10001B78002B7FF47DA9049B1B78002B3FF44E
:10AB20007AAFFFF7ACB9F5F7C9FCB2E41835802D60
:10AB3000B8F800302E4AA8BF80259D423FF4FAA8FD
:10AB4000214B158020E7059C069DFFF75FB97F200C
:10AB5000FFF7E6BA7F2032E60120FFF7E1BA1F4B8C
:10AB60001B78002B7FF4E6A81D4B1B78002B3FF4CD
:10AB7000E1A8B8F80030144A013BA8F8003015707D
:10AB8000FFF7D8B8154B1B78002B7FF48AAD144B18
:10AB90001B78002B3FF4CEA8B8F800300A4A0133E6
:10ABA000A8F800301570FFF7C5B8104B02931B884A
:10ABB000002B3FF42BA97FE7012000E6ABAAAA2ACD
:10ABC000008BFF1FD88AFF1F959DFF1FBC9EFF1F94
:10ABD000B19EFF1F989DFF1F349FFF1F359FFF1FD2
:10ABE000369FFF1FFC9DFF1F5B9DFF1FC69DFF1F24
:10ABF000709EFF1F2A4B01227F2107201A80F6F743
:10AC0000EBFA7F210B20F6F7E7FA76E5254B0422D5
:10AC10007F2107201A80F6F7DFFA00210B20F6F7D4
:10AC2000DBFA63E51F4B02227F2107201A80F6F72B
:10AC3000D3FA7F210B20F6F7CFFA52E5194A00210B
:10AC400007201380F6F7C8FA7F210B20F6F7C4FA25
:10AC500042E5154B00227F2107201A80F6F7BCFA47
:10AC60007F210B20F6F7B8FA4FE5104B0193104BFC
:10AC7000104A0493FFF7CDB99AF80000F5F77CFF6E
:10AC8000BDE4012B3FF456A801257AE6039B1B780F
:10AC9000002B3FF4F4A8FFF7BCB8074B03930BE776
:10ACA000169EFF1F9C9EFF1F5C9DFF1FEB9EFF1FBC
:10ACB0005B9DFF1FB19EFF1FBC9EFF1F00207047C2
:10ACC00090F8392090F83800101A704790F8383012
:10ACD00090F839209A4205D95A1C034480F838204C
:10ACE000187E70474FF0FF30704700BF90F8383043
:10ACF00090F839209A4286BF1B18187E4FF0FF301B
:10AD0000704700BF704700BF38B50546B0F85E0019
:10AD100090B195F85D301446C3F1210294420CD8ED
:10AD200005F13B001844224601F0D0FF95F85D3054
:10AD3000234485F85D30204638BD01201446287133
:10AD4000EEE700BFB0F85E306BB190F85D30202BBD
:10AD500007D8C218013380F85D30012082F83B101B
:10AD60007047012303710020704700BF0023426930
:10AD700080F8383080F8393080F85C3080F85D3009
:10AD800080F85E3080F85F3006CA30B40D68046920
:10AD900043662A4383660A60A370426990F8613073
:10ADA0001649146813441D7A5B7B01EBC5051B0231
:10ADB0006D6803F4E06343F064032B6090F8623045
:10ADC00013449D7CDB7D01EBC5011B02496803F444
:10ADD000E06343F064030B6021685368194205D0B7
:10ADE000036927225A70036904229A710369202299
:10ADF0005A71036980229A7030BC704794430100F5
:10AE000043690CCB12681A420CD0094B99420AD9FB
:10AE1000084B9942036994BF1A220D225A700369A4
:10AE200004229A717047036927225A70F7E700BF1E
:10AE30007F1A06003F420F0010B50269D378DBB2DB
:10AE4000D90604463DD510215806D17038D503F0F7
:10AE5000040303F0FF02002B51D03D49626E002332
:10AE60000B7084F85D30002A5BD0904794F85D3019
:10AE7000002B56D02369D0229A70236994F83B2086
:10AE80001A712369012284F85C200222DA7010BD55
:10AE9000304B84F860009C424AD02F4B9C4252D0E9
:10AEA00094F8391013791F29DBB207D828480078A5
:10AEB00020B16018013184F8391003760223D37071
:10AEC00010BD5906C3D4917801F0100101F0FF00C4
:10AED0000029DDD013F001031ED194F85C1094F822
:10AEE0005D00884281BF4B1C091984F85C3091F8E1
:10AEF0003B3013712369D0229A702269DEE72369FF
:10AF000084F83920C0229A702369114A19790121E5
:10AF100011700222DA7010BDC02393702269137978
:10AF2000CCE70122002384F85D2084F83B30A1E7C0
:10AF3000626994F86130094913440322187A02F0D7
:10AF40006FFC2269ACE7626994F861300449F3E769
:10AF5000409FFF1F008EFF1F6C8EFF1FC1AF0000C0
:10AF6000CDAF00000369DB7803F0200373B190F8E4
:10AF700060300133DBB2012B80F860301AD94269AE
:10AF800090F861301344187A02F0C6BC70B542697B
:10AF900003F0FF0590F8613013440446187A02F07C
:10AFA000BBFCA36E5BB184F8385094F83900BDE85F
:10AFB0007040184790F85F30002BE0D0704770BDAC
:10AFC0000148FFF7CFBF00BF008EFF1F0148FFF70A
:10AFD000C9BF00BF6C8EFF1F2DE9F047374FDFF868
:10AFE000E0903B68026982B006460093DDF800807D
:10AFF0000021A025D3789B065BD53B680193019B7C
:10B00000C8EB03030F2BF5D949B1102BF2D0002068
:10B010009070336980229A7002B0BDE8F08772693F
:10B0200096F8613013440521187A02F06FFE7269B8
:10B0300096F861301344012193F812A0504602F0B3
:10B0400065FE09240021504602F04CFE2B46013BD0
:10B05000FDD10121504602F045FE2B46013BFDD1BA
:10B06000013CEFD1706996F8611001444FF4A07271
:10B070000C7A4B7B09EBC4011B02496803F4E063C3
:10B0800043F064030B6096F862300344997CDB7DE7
:10B0900009EBC1011B02496803F4E06343F0640358
:10B0A0000B60013AFDD13269D3789B064FF0010164
:10B0B000A3D4012002B0BDE8F08700BF489FFF1F66
:10B0C00094430100F0B503691222DA7002699378A3
:10B0D00003F0200385B004460D46002B5ED0B42358
:10B0E00093703C4922690B680093009E05E00B6851
:10B0F0000193019B9B1B042B42D8D37803F02003C0
:10B1000003F0FF00002BF2D094F85D30002B31D01B
:10B110004FF0000E4FF0020C04EB0E0393F83B309F
:10B1200013710B680393039F206907E09B060DD5FD
:10B130000B680293029BDB1B052B28D8C378DBB27C
:10B1400003F0020202F0FF06002AEFD080F803C0ED
:10B150002669F378DBB2DF0632462DD49F062BD565
:10B16000DB0731D40EF1010E94F85D305FFA8EFEEC
:10B170007345D1D800201DBB002384F85E3004E065
:10B180009070236980229A70042005B0F0BD86700B
:10B190002369802204209A7005B0F0BD03F0FF06F9
:10B1A000FFF71AFF10B9042005B0F0BD236984F839
:10B1B0005F60B0229A7094E78023B3700420DAE7CE
:10B1C00026698023B370D7E7BEF1000F0CBF0220C1
:10B1D0000320F6E7489FFF1F2DE9F041066900258F
:10B1E000122780F8385080F83950F770D0F810C026
:10B1F0009CF802E00EF0200E88B004468846154602
:10B200001E46BEF1000F49D0B4238CF80230784BB3
:10B2100021691A680092DDF800E006E01A680192E0
:10B220000198CEEB0000042830D8C87800F0200048
:10B2300000F0FF070028F1D04FEA480242F0010277
:10B24000D2B20A711A680292DDF808E0206906E0BD
:10B250001A6803920399CEEB010105292AD8C17817
:10B2600001F0020101F0FF070029F1D04FF0020CBC
:10B2700080F803C02269D17811F0110722D12DBBCB
:10B28000002E0CBFA0238023937003E08F702369EE
:10B2900080229A70384608B0BDE8F0810EF0FF07B2
:10B2A000FFF79AFE0028F5D0236984F85F70B0227A
:10B2B0009A70ACE787702369802238469A7008B08C
:10B2C000BDE8F081802393700027E3E7012D75D05E
:10B2D000A021917021690A79BE4667464FF0A80CFB
:10B2E0001A680492049805E01A680592059A121AE1
:10B2F000052A4AD8CA7802F0020202F0FF08002AA2
:10B30000F2D0CF702169CA78D2B212F0100F08467D
:10B310005AD1920658D5013DEDB2012D49D0BEF16A
:10B320001F0F3BD90A79012DDAD11A680692069DC2
:10B3300005E01A680792079A521B052A46D8C27878
:10B3400002F0020202F0FF01002AF2D00223C370D1
:10B350002269D378DBB2D9063AD49B0634D5B02320
:10B36000BEF11F0F93703FD8226904EB0E031279D0
:10B370001A760EF1010E5FFA8EFE16B12369802255
:10B380009A7084F839E0774684E781F8028023696F
:10B3900080229A70774684F839E07BE704EB0E024E
:10B3A00091F8048082F818800EF1010E5FFA8EFE8B
:10B3B000B9E781F802C021690846B0E7A821917079
:10B3C0002069BE460279B0E7774663E78170DEE721
:10B3D0001021A023D170013BFDD12269937803F0A5
:10B3E000F7037746937055E723691B79C5E700BFDC
:10B3F000489FFF1F0148FFF71FBD00BF008EFF1FC2
:10B400000148FFF719BD00BF6C8EFF1F704700BFDA
:10B4100038B5144C037801225B000546204684F8B9
:10B420003B3084F85E2084F85D20FFF78BFC2046DB
:10B430000021FFF747FE0B4C2978012320461A46CE
:10B44000FFF7CAFE0128F6D194F8383094F8392075
:10B450009A4205D9E218013384F83830107E38BD9D
:10B46000FF2038BD008EFF1F38B51B4C037801222A
:10B470005B000546204684F83B3084F85E2084F863
:10B480005D20FFF75FFC20460021FFF71BFE124CFA
:10B490002978204601230222FFF79EFE0228F6D1DA
:10B4A00094F8382094F839108A420FD2531CDBB23A
:10B4B000A018994284F83830007E0AD92344023219
:10B4C0001B7E84F8382040EA032038BD4FF6FF7019
:10B4D00038BD40F47F4038BD008EFF1F0C2901D9D4
:10B4E000002070470231490001F0FE01FFF7BCBFA8
:10B4F00070B50C4C0378164601255B00204684F895
:10B500003B3084F85E5084F85D50FFF71BFC3146F9
:10B510002046FFF717FC29462046BDE87040FFF79C
:10B52000D1BD00BF008EFF1FF8B505460F46164679
:10B53000412421463A462846FFF7DAFF611C0234CF
:10B54000C9B232462846E4B2FFF7D2FF592CF0D1F7
:10B55000F8BD00BF38B504460D463548FFF706FC78
:10B560006322802120462570FFF7C2FF012002F0F0
:10B57000F5FB204600225E21FFF7BAFF20465D2141
:10B58000FFF746FF242801D0002038BD20460622C0
:10B590000C21FFF7C9FF204601222B21FFF7A8FF4E
:10B5A000204601222C21FFF7A3FF20460E222D2149
:10B5B000FFF79EFF204600222E21FFF799FF20462D
:10B5C00001222F21FFF794FF204605223021FFF7AB
:10B5D0008FFF204601223121FFF78AFF20460022FB
:10B5E0003221FFF785FF204600223321FFF780FF3D
:10B5F000204600223421FFF77BFF20460022352120
:10B60000FFF776FF204600225B21FFF771FF2046FF
:10B6100010225C21FFF76CFF204620225D21FFF7FE
:10B6200067FF20468F225E21FFF762FF012038BDB1
:10B63000008EFF1F10B4047F4160022CC26002D054
:10B6400010BC03F04FBF836810BC1847F0B4464BE2
:10B65000464A186BDC6A01791170454922790A70F3
:10B660009A6A00790870002A46D05968C9688A42E7
:10B670003ED82168CC8B240402F1FF3065D4C0F39E
:10B680000E00C883C88B80B2C882196B0968C88B4A
:10B69000000452D4C2F30E00C883C88B002480B2C9
:10B6A00012F1FF32C88218BF01229C62D96A2E486B
:10B6B00009680D6800F12404A54236D00068C4680A
:10B6C00014F0804F0C680D6815BF2488247802356B
:10B6D000013544F000440D604463196B254B097932
:10B6E0001970214912B1CA6A12791A70F0BC7047F8
:10B6F000521A9A620122D9E7586B196805681E4CE4
:10B700000A63CC62CC682D681C4E24F08044032769
:10B71000B542CC6083F825701FD1037F4260022BB5
:10B72000C2601ED0F0BC03F0DDBE016890F82400BA
:10B73000CC6840F000404863CFE7CC8BC2F30800F0
:10B7400004F47E442043C883A7E7CC8BC0F30800F1
:10B7500004F47E442043C88394E72B461146F0BC92
:10B7600018478368F0BC1847D88EFF1F1F80004021
:10B770001C8000401B80004000000FFF35B6000019
:10B7800090E80C00F0B41C6859682568164F174EF5
:10B7900029432160164D17491760D6601561116065
:10B7A000417A154A5C180A3194F8244053F8215024
:10B7B00002EBC40149680D60017A5C1803EB81015A
:10B7C000247ECD6902EBC40149680D60817A581866
:10B7D00003EB810390F83000596B02EBC002F0BC20
:10B7E00053681960704700BF01401F000110003806
:10B7F0000110007800001F809443010038B5044612
:10B80000104621700A491D4605F074F901464FF0B3
:10B810007E5005F023FA074905F06CF9E560606099
:10B820002561656102F078FAE061204638BD00BF0D
:10B83000DB0FC9400024744938B504461046217016
:10B8400009491D4605F056F901464FF07E5005F0B6
:10B8500005FA064905F04EF9E5606060256165610D
:10B8600002F05AFAE06138BDDB0FC9400024744988
:10B8700038B503780446032B20D8DFE803F01A1804
:10B880001002C168406905F02BF80D490546606853
:10B8900005F0E4F90146284605F0E0F938BD08490D
:10B8A000406805F0DBF9E16805F024F938BDC068AF
:10B8B00038BDC168406905F013F838BD002038BDB7
:10B8C0000024744970B504460E4602F025FA054678
:10B8D000E069281A05F0BAF8E3682361E56166615A
:10B8E000A0610146606805F0B9F90146A060104802
:10B8F00005F0B4F904F08AFC04F02AF904F09CFF86
:10B90000054601464FF07E5004F0EAFF616905F0FC
:10B91000F1F821690646284605F0ECF80146304664
:10B9200004F0E0FFE0602046BDE87040FFF7A0BFF4
:10B93000000080BF704700BF2DE9F04F85B09946E9
:10B94000BDF93870BDF83CA0BB1AC1EB090B002B48
:10B95000B8BF5B42BBF1000FB8BFCBF1000B5B453A
:10B960000D4616460093804648DC4D453A46334620
:10B970004CDC194613460A46C5EB09019B1A89B2ED
:10B98000002B0CB2B8BF5B4204EBD474BE42ACBF18
:10B990004FF0FF3201224D45039102924FEA6404B9
:10B9A00029DC9BB201930DE0D8F80070BF69B8475D
:10B9B000019BE41AA3B21CB20135002C2DB211DB9D
:10B9C000A94518DB009B5B452A4653463146404655
:10B9D000EADCD8F8002053469769294632464046AB
:10B9E000B847E5E7029A1644039AA94502EB030417
:10B9F00036B224B2E6DA05B0BDE8F08F4A462B46EF
:10BA0000B94635464D4517461E46B2DD30462946F5
:10BA10003E464D4607468946AEE700BF10B404686F
:10BA20002469A44610BC604730B40468BDF80850CF
:10BA30000295A46BA44630BC604700BF30B40468D4
:10BA4000BDF808500295E46BA44630BC604700BFC7
:10BA500070B40468BDF90C60BDF8105003960495ED
:10BA6000246CA44670BC6047704700BF10B582B01C
:10BA7000B0F90C2001910168009200220C6CB0F921
:10BA80000A301146A04702B010BD00BF704700BF8A
:10BA900001F003010129C17506D0032904D0C28831
:10BAA00003894281838170470289C38842818381EF
:10BAB000704700BF2DE9F0410568134E6F6986B0ED
:10BAC000B7420446BDF8308010D1013B13441BB28D
:10BAD0000093CDF804800B46AD6A2046A847236842
:10BAE000DB6AB3420AD106B0BDE8F0810593049247
:10BAF0000391B84703A925680EC9E6E7204606B0BA
:10BB0000BDE8F041184700BF69BA00002DE9F041D7
:10BB10000568124E6F6986B0B7420446BDF83080A2
:10BB20000FD1013BCDF804800B4400921BB2AD6AEB
:10BB30002046A8472368DB6AB3420AD106B0BDE8B5
:10BB4000F081059304920391B84703A925680EC9B3
:10BB5000E7E7204606B0BDE8F041184769BA0000A3
:10BB60002DE9F04F0568DFF858B06F6985B05F4583
:10BB70000646BDF93890BDF83CA00C46904615D15C
:10BB80001F19BC420CDACDF800A0214601342D6A01
:10BB90004B464246304624B2A847BC423568F2DBE9
:10BBA000EB6A5B4507D105B0BDE8F08F0393B8475A
:10BBB0003568039BE4E7304605B0BDE8F04F184711
:10BBC00069BA00002DE9F04387B099420546BDF9F6
:10BBD0003840BDF83C6025D0A24212D00768DFF89B
:10BBE0008080D7F81490C14532D18DE850002846A6
:10BBF000BC6AA0472B68DB6A434524D107B0BDE887
:10BC0000F083994202DD08461946034628680E96DD
:10BC1000C46B01335B1A1BB22846A44607B0BDE8CB
:10BC2000F0436047A24202DD134622461C462868C4
:10BC30000E96631C846B9B1A1BB22846A44607B061
:10BC4000BDE8F0436047284607B0BDE8F043184719
:10BC5000059304920391C84703A92F680EC9C4E74E
:10BC600069BA00002DE9F04FD0F800E0DFF89090BD
:10BC7000DEF814B083B0CB450446BDF93080BDF882
:10BC800034A00D4617461E4631D1CDF800A0DEF88F
:10BC900024B0294633463A462046D8472368CDF893
:10BCA00000A008F1FF323A44D3F824B0294612B27A
:10BCB00033462046D8472368CDF800A02946D3F85C
:10BCC00020B03A4643462046D8472068CDF800A029
:10BCD000711E29444346056A09B23A462046A847E0
:10BCE0002368DB6A4B4506D103B0BDE8F08FD84727
:10BCF000D4F800E0C9E7204603B0BDE8F04F18478C
:10BD000069BA0000F0B4002401264FF6FF75094F10
:10BD100007600471C475C48104824476C461867569
:10BD2000067685824582C180028141818281F0BC94
:10BD3000704700BFA83D01002DE9F04F85B00668AF
:10BD4000BDF84450BDF93880CDF800800446019517
:10BD5000D6F848B00392BDF93C60BDF94070894601
:10BD60009A46D84723680195009742465146D3F832
:10BD7000488020463346C0472068039B0E930F95AA
:10BD8000856C4B463A4631462046AC4605B0BDE888
:10BD9000F04F60472DE9F04F87B01746BDF940409E
:10BDA00000912546E91D059344BF2B4603F10E0182
:10BDB0000268BDF8486053690294C91003912B4989
:10BDC000BDF9444001968B42824645D1002C3CDDB2
:10BDD000029B3C445E1EB6B24FF0000923B20493AE
:10BDE00001364D46029B002B28DD059B002403EB0A
:10BDF000090806E0EDB22B0604F1010411D4A642B5
:10BE00001CD0A1B211F0070F23B24FEA4505F1D1C2
:10BE1000002BB8BF0733DB10013418F803502B0692
:10BE2000EDD5009BD2F818B019443A4609B2019BEF
:10BE30005046D847A642DAF80020E2D1039B0137EA
:10BE40009944049B3FB2BB42CCD1D36A074A934288
:10BE500006D107B0BDE8F08F9847DAF80020B5E7C3
:10BE6000504607B0BDE8F04F184700BF69BA000060
:10BE700070B4BDF90C60BDF91050BDF814400396C4
:10BE80000495059470BCFFF785BF00BF2DE9F04F06
:10BE900093B090460591C1691090BDF8700007906D
:10BEA000BDF874909DF878A00493002900F0CD802F
:10BEB0000A7A0AC9894604998A1AD2B203EBC203E4
:10BEC000BAF1010FDA780B9293F905201E8893F8E6
:10BED00002B00F9293F9064079D913B2099323B2B5
:10BEE0000C93109B1A68A94B1193194653698B4206
:10BEF00040F0A6800B9B002B55D01FFA88F3002141
:10BF00000D93C8462344DDF8409006910E930F46EA
:10BF10000C46BBF1000F3FD0BDF818100C9B0397E7
:10BF20001FFA8AF0CB1813FB00F304900E9801441B
:10BF30000D98034409B21BB20A910893002505E04D
:10BF40000135EBB264009B45E4B222D9039B2B443C
:10BF5000590703D1731C18F806409EB22306EFD58B
:10BF6000099BBDF81000E91811FB00F10598BAF122
:10BF7000010F0FFA8AF301441CD007980190009337
:10BF8000D26909B217464846089AB847D9F800203E
:10BF9000D6E7039F5F44FFB2069B0B9901330693DC
:10BFA000DBB29942B5D8D36A119A934243D113B008
:10BFB000BDE8F08F0F9B191893690A9A29441F4610
:10BFC00009B2079B4846B847D9F80020B8E70023D4
:10BFD0000C93099385E70A9A0D9B0132013B52B2FB
:10BFE00013F0FF030A920D936FD1DDF81890079BB1
:10BFF000DDF83C80DDF820A04B4517D0BAF1010FE9
:10C0000000F0C8800B9A109DCDF804900BEB8B01CB
:10C010004FEACB030A4400931146DEF81C40534616
:10C02000424609B22846A047D5F800E0DEF82C3099
:10C03000119A9342BBD0109813B0BDE8F04F184747
:10C04000109D284698472A6854E7109A0598B2F937
:10C050000A308342ABDDB2F90C304345A7DD06233D
:10C0600013FB0A03002BA2DD08EBCA03002B9EDDA5
:10C07000537E2BB9049BAF2B02D90133DBB204935F
:10C08000109BD3F800E0414B11931A46DEF81430B0
:10C09000934240F08E801FFA88F30E9308339BB2D0
:10C0A000BDF81420059305230D9300230A93CDF8C2
:10C0B0003C800FFA8AF3DDF84080CDF818900B929F
:10C0C0001FFA8AFBCDF820A099460A9ABDF8100005
:10C0D0000B9C0E9D0523194611FB00232C4811468D
:10C0E000C75C039702FB0B4214FA81F312B21BB236
:10C0F00009920C932C462E461CE0089B0999012BB3
:10C100002AB24B4640462DD0079F0197CDF80090AC
:10C11000DEF81CA0D047D8F800E0039B5B08013490
:10C120000393059BA4B25D445E44A342ADB2B6B294
:10C130003FF451AF039BD807DFD4079B069A934285
:10C14000EBD0089B012B16D0069B0193CDF80090F5
:10C15000DEF81CA009994B4632B24046D047D8F8C9
:10C1600000E0DAE7DEF818A0079B0C9922B2D0476E
:10C17000D8F800E0D1E7DEF818A00C991346404645
:10C1800022B2D047D8F800E0C7E700BF69BA000084
:10C19000F83D01000B99109DCDF800900531DEF8B7
:10C1A000204009B2424608232846A047D5F800E0BF
:10C1B0003CE7109C20469847D4F800E06BE700BFAE
:10C1C000F0B5C36985B004462BB30A2968D00D29A0
:10C1D0004AD01A7A914247D3587A884244D35D684C
:10C1E0008A1A05EBC205AA78002A50D0E878002800
:10C1F0004DD0207E00283AD095F905E0B4F90E0024
:10C20000A67DB4F90A70724406FB0202BA4262DCEF
:10C21000B4F9102030E00A2956D00D2924D0027E2E
:10C22000002A4BD0B0F90E00A57DB4F90A600622B1
:10C2300012FB0502B2423EDD228AE38102EBC50217
:10C2400012B218462282A78A668A02950B468DE8AA
:10C25000C00001462046FFF719FEA37DE28903EBEB
:10C26000430302EB4303E381012005B0F0BDA67D4B
:10C27000B4F90E00B4F91020B4F814E0678A0296FD
:10C280000B468DE8804001462046FFF7FFFD2979E7
:10C29000E389A27D012001FB0233E38105B0F0BDFB
:10C2A0000022C2819A7A817D038A01FB02330382D4
:10C2B000012005B0F0BDB4F91020C4E7857DB4F9C4
:10C2C0001020B0F90E00BEE7028A817DC38102EB27
:10C2D000C1030382C8E70020E0819B7A228A03FB26
:10C2E000062212B22282C7E7C1810282704700BFD4
:10C2F000002908BF01218175704700BF81824182FA
:10C30000704700BFC07D7047B0F90A00704700BF9A
:10C31000B0F90C00704700BFF0B5C47DBDF81450F3
:10C32000022C75D0032C6ED0012C32D0002A79DB80
:10C33000B0F90840944265DD002978DBB0F9066069
:10C340005818B042C4BF731A1BB2002B5ADD002A22
:10C350001046B8BFD01D012440F3CF0002F0070201
:10C36000704E01EBC01104FA02F2A5423144D2B280
:10C3700000F0A480C0F09580022D43D1013B11FA5A
:10C3800083F04B1E13F8011F514083421970F9D1FD
:10C39000F0BDC488013CA21A12B2002A7BDBB0F9BE
:10C3A000064094422EDD00293DDBB0F908605818A4
:10C3B000B042C4BF731A1BB2002B23DDC9B2C80838
:10C3C000584C02EBC01211F00701DBB204EB020083
:10C3D00039D0C1F10801C9B2534E8B42765C2AD2E2
:10C3E000C3EB010EFF2747FA0EF7012D06EA0706F9
:10C3F00074D06ED3022D40F09480A75C7E40A6548A
:10C400008B421DD2F0BD0489E41A611A09B2C4E757
:10C410000689C488013EB21AE41A12B2611A002ACF
:10C4200009B285DAF0BD0B441BB20021BDE70B4415
:10C430001BB2002182E7012D50D04AD3022DDCD05F
:10C440005B1ADBB28030072B18D9022D4ED0A3F136
:10C450000806C6F3C406B11C00EBC111012D0CBFC8
:10C46000FF24002400F1800202F8804C80328A42CE
:10C47000FAD1013600EBC61003F00703002BC1D040
:10C480002A4A012DD35C2DD006D3022DBAD10278D1
:10C4900053400370F0BDF0BD027822EA030303703D
:10C4A000F0BD013BD24311FA83F0D2B24B1E13F818
:10C4B000011F114083421970F9D1F0BD013B11FAFF
:10C4C00083F04B1E13F8011F114383421970F9D1F9
:10C4D000F0BDA75C27EA0606A65491E7A75C3E4399
:10C4E000A6548DE7027813430370F0BDA3F108054D
:10C4F000C5F3C405AC1C00EBC41400F1800212F8B3
:10C50000801CC94302F8801C8032A242F7D1013559
:10C5100013F0070300EBC5103FF474AF034AD35C7C
:10C52000B5E7F0BD208FFF1F188FFF1F108FFF1F73
:10C53000F0B5C47DBDF81450022C76D0032C6FD01A
:10C54000012C37D000297ADBB0F906408C4230DD6F
:10C55000002A79DBB0F908609818B042C4BFB31A5A
:10C560001BB2002B25DDD2B2D008754C01EBC011F7
:10C5700012F00702DBB204EB010071D0C2F1080235
:10C58000D2B2704E9342B65C62D2C3EB020EFF276A
:10C5900047FA0EF7012D06EA070600F0AC80C0F05E
:10C5A000A580022D40F0CA80675C7E4066549342AD
:10C5B00053D2F0BDC488E41AA21A12B2002977DB64
:10C5C000B0F908408C42F4DD002A39DBB0F906608E
:10C5D0009818B042C4BFB31A1BB2002BE9DD002982
:10C5E0000846B8BFC81D012440F3CF0001F0070181
:10C5F000534E02EBC01004FA01F1A54206EB000213
:10C60000C9B268D05AD3022DD3D1013B12FA83F0BC
:10C61000531E13F8012F4A4083421A70F9D1F0BD1E
:10C620000489013C611A09B2C8E7C6880489013E41
:10C63000711AE41A09B2A21A002912B284DAF0BD02
:10C6400013441BB20022C1E713441BB2002281E74E
:10C65000012D50D04AD3022DA6D09B1ADBB28030D8
:10C66000072B18D9022D4ED0A3F10806C6F3C40635
:10C67000B11C00EBC111012D0CBFFF24002400F1FF
:10C68000800202F8804C80328A42FAD1013600EBF7
:10C69000C61003F00703002B8BD02B4A012DD35C6F
:10C6A0002DD006D3022D84D1027853400370F0BD03
:10C6B000F0BD027822EA03030370F0BD013BC943D9
:10C6C00012FA83F0C9B2531E13F8012F0A408342B5
:10C6D0001A70F9D1F0BD013B12FA83F0531E13F822
:10C6E000012F0A4383421A70F9D1F0BD675C27EA33
:10C6F000060666545BE7675C3E43665457E702787C
:10C7000013430370F0BDA3F10805C5F3C405AC1CC9
:10C7100000EBC41400F1800111F8802CD24301F821
:10C72000802C8031A142F7D1013513F0070300EBD3
:10C73000C5103FF43EAF044AD35CB5E7F0BD00BF7F
:10C74000208FFF1F188FFF1F108FFF1FF8B50D1EC2
:10C7500006DB14461F460646FFF7D6FD854200DB82
:10C76000F8BD002CFCDB3046FFF7D2FD8442F7DA3F
:10C770003046FFF7C7FD02284BD0032843D00128DD
:10C7800004D1F388013B1B1B2C461DB2012F03D0A3
:10C7900026D3022F12D0F8BD002C2346B8BFE31DCC
:10C7A00043F3CF0305EBC3151E4804F00704435DB4
:10C7B000012101FA04F41C434455F8BD002C234622
:10C7C000B8BFE31D43F3CF0305EBC315154804F0D1
:10C7D0000704435D012101FA04F45C404455F8BDAF
:10C7E000002C2346B8BFE31D43F3CF0305EBC3156D
:10C7F0000C4804F00704435D012101FA04F423EA24
:10C8000004044455F8BD3389013B5B1B25461CB22B
:10C81000BCE7F18832890139013A4D1B141B2DB256
:10C8200024B2B3E7208FFF1F38B5402204460D46DF
:10C830008021FFF767FAFF23064A84F8255084F821
:10C84000223084F8263084F8243084F823302260A3
:10C85000204638BD004301004FF4806200210148AA
:10C8600004F0FCBE208FFF1FF8B590F92230013391
:10C8700004460F4642D0012190F8260001F032FA1A
:10C88000002194F8240001F02DFA002194F82600EC
:10C8900001F028FA94F8273083B1254B1A684FF03D
:10C8A0000043D3625763D36A002BFCDA936B94F88E
:10C8B00026000121BDE8F84001F014BA08268025C1
:10C8C000002194F8230001F00DFA17EA05034FF058
:10C8D000010194F8220008BF194601F003FA012172
:10C8E00094F82300CD4001F0FDF9013EE8D194F821
:10C8F00026000121BDE8F84001F0F4B90D4C90F894
:10C90000203001255B002046002184F83B3084F86C
:10C910005E5084F85D50FEF715FA39462046FEF762
:10C9200011FA29462046BDE8F840FEF7CBBB00BF10
:10C93000D88EFF1F008EFF1FF8B50D4690F922100C
:10C9400080F820200131044680F821501F4600F075
:10C95000AD80012190F8240001F0D8F9012194F86C
:10C96000260001F0D3F994F82730002B00F0D38093
:10C97000804E3046FEF704FFF37A002B40F0DB8058
:10C9800033687D4AD968914206D07C4E7C487D4907
:10C990001E60DA6018611960E7B194F9250000287B
:10C9A00018DBC0B2012101F0B1F9012194F8250092
:10C9B00001F098F9012001F0D1F9002194F8250047
:10C9C00001F090F90A2001F0C9F9012194F825003D
:10C9D00001F088F9AE212046FFF746FFD521204619
:10C9E000FFF742FF80212046FFF73EFFA8212046A7
:10C9F000FFF73AFF3F212046FFF736FFD3212046BD
:10CA0000FFF732FF00212046FFF72EFF402120468E
:10CA1000FFF72AFF8D212046FFF726FF012D4DD07D
:10CA200014212046FFF720FF20212046FFF71CFF9E
:10CA300000212046FFF718FFA1212046FFF714FF31
:10CA4000C8212046FFF710FFDA212046FFF70CFF30
:10CA500012212046FFF708FF81212046FFF704FF3F
:10CA6000CF212046FFF700FFD9212046FFF7FCFE2B
:10CA7000F1212046FFF7F8FE2046DB21FFF7F4FE08
:10CA800020464021FFF7F0FE2046A421FFF7ECFEF0
:10CA90002046A621FFF7E8FE20462E21FFF7E4FE00
:10CAA0002046AF21BDE8F840FFF7DEBE3648FEF76E
:10CAB0005DF936493448FEF7A3F96DE720461021A9
:10CAC000FFF7D2FE20462021FFF7CEFE20460021B0
:10CAD000FFF7CAFE2046A121FFF7C6FE2046C82167
:10CAE000FFF7C2FE2046DA21FFF7BEFE20461221E4
:10CAF000FFF7BAFE20468121FFF7B6FE20469F21B0
:10CB0000FFF7B2FE2046D921FFF7AEFE22212046D4
:10CB1000FFF7AAFEB0E7012194F8220001F0F6F831
:10CB2000012194F8230001F0F1F894F82730002B4C
:10CB30003FF432AF1CE772B6F37AD8071A4606D52F
:10CB40001349F26808680240B2610A601A46990700
:10CB500006D5104933690868F27A0340F3610B6027
:10CB6000530705D50C4A736911680B403362136093
:10CB700062B605E7D88EFF1F0000013801403F0074
:10CB80000000017800003F80008EFF1F801A060021
:10CB900080E100E084E100E088E100E02DE9F84F69
:10CBA00021210546FFF760FE28460021FFF75CFEC5
:10CBB00028467F21FFF758FE28462221FFF754FE22
:10CBC00028460021FFF750FE28460721FFF74CFEBC
:10CBD00095F92230013349D0012195F82600DFF87C
:10CBE000E480DFF8E4B001F07DF8012195F824003D
:10CBF00001F078F8002195F8260001F073F808F5A7
:10CC000080694FF0004A95F8273018F8017F0BBB78
:10CC100008268024002195F8230001F063F817EA24
:10CC200004034FF0010195F8220008BF194601F0F6
:10CC300059F8012195F82300CC4001F053F8013E4A
:10CC4000E8D1C845DFD195F826000121BDE8F84FAD
:10CC500001F048B8DBF80020C2F82CA05763D36A73
:10CC6000002BFCDAC845936BCDD1ECE7DFF85080A0
:10CC7000124F00244FF0010995F82030104888F831
:10CC80005E905B00402188F83B3088F85D90FEF7AD
:10CC900059F804F11006B6B2395D09480134A4B25E
:10CCA000FEF750F8B442F7D101210548FEF70AFA21
:10CCB000B4F5806FE0D1BDE8F88F00BF208FFF1F73
:10CCC000008EFF1F1F8FFF1FD88EFF1F844641EA73
:10CCD000000313F003036DD1403A41D351F8043BF4
:10CCE00040F8043B51F8043B40F8043B51F8043B46
:10CCF00040F8043B51F8043B40F8043B51F8043B36
:10CD000040F8043B51F8043B40F8043B51F8043B25
:10CD100040F8043B51F8043B40F8043B51F8043B15
:10CD200040F8043B51F8043B40F8043B51F8043B05
:10CD300040F8043B51F8043B40F8043B51F8043BF5
:10CD400040F8043B51F8043B40F8043B51F8043BE5
:10CD500040F8043B51F8043B40F8043B403ABDD254
:10CD6000303211D351F8043B40F8043B51F8043BF6
:10CD700040F8043B51F8043B40F8043B51F8043BB5
:10CD800040F8043B103AEDD20C3205D351F8043B85
:10CD900040F8043B043AF9D2043208D0D2071CBF51
:10CDA00011F8013B00F8013B01D30B88038060467A
:10CDB000704700BF082A13D38B078DD010F00303F0
:10CDC0008AD0C3F10403D21ADB071CBF11F8013B60
:10CDD00000F8013B80D331F8023B20F8023B7BE7AF
:10CDE000043AD9D3013A11F8013B00F8013BF9D2DA
:10CDF0000B7803704B7843708B7883706046704774
:10CE0000374A384913681B06FCD40B6813F08003BB
:10CE1000F8D172B634490A78002A5FD0334A3448D0
:10CE2000F0B4344C176806682568D4680C303E446A
:10CE3000143200681268304F35442C4420440244B8
:10CE4000C2F34E022D4E2E482E4D2F4C42F400427E
:10CE50003A60376806682D682C4A24680C303E44D6
:10CE6000006812682A4F35442C4420440244C2F31F
:10CE70004E02284E2848294D294C42F400423A607F
:10CE8000376806682D68274A24680C303E440068DD
:10CE90001268254F35442C4420440244C2F34E020C
:10CEA000224E2348234D244C42F400423A60376816
:10CEB00006682D68214A24680C303E4400681268D8
:10CEC00035442C4420440244C2F34E021C4842F430
:10CED000004202600B7062B6F0BC704762B67047E9
:10CEE00024B0034024B00B40429FFF1F38B00340E2
:10CEF0003CB0034040B003402CB0034058B0034066
:10CF00005CB0034060B0034064B003406CB00340C9
:10CF100030B0034038B00B403CB00B4040B00B4049
:10CF200044B00B404CB00B402CB00B4058B00B4001
:10CF30005CB00B4060B00B4064B00B406CB00B4079
:10CF400030B00B4030B42948294A2A4B2A4D60247E
:10CF5000E121047011701B78284C082B30D00A2B6B
:10CF60002748284937D00C2B0CBF35223D221223ED
:10CF70002A60236002600B60234B24491B78244AFB
:10CF8000BBB101230B601360224B23491B78234A5A
:10CF9000012B26D9042B0FD9082B1ED9102B94BF97
:10CFA000862387230B6013601D4B01221A7030BC4F
:10CFB00070470B601360E7E784230B601360F3E7AF
:10CFC00000F58E200F490830012213232A602360C8
:10CFD00002600B60D0E73922F7E785230B6013600E
:10CFE000E2E780230B601360DEE700BF00400740EC
:10CFF000014007402093FF1F08B003400CB00340DE
:10D0000008B00B400CB00B40459FFF1F20B0034001
:10D0100020B00B402193FF1F24B0034024B00B40ED
:10D02000429FFF1F0C2830B417D91023984228BF05
:10D0300018461C46104A114D1178181A8C42287057
:10D0400018D00F4913700B7823B10E490E4A0023F4
:10D050000B60136030BCFFF775BF0A2802D90C23A0
:10D060001C46E7E7082802D90A231C46E2E7082302
:10D070001C46DFE730BC70472093FF1F419FFF1F16
:10D08000429FFF1F24B0034024B00B4028282FD814
:10D09000334B2DE9F0411E5CFF2E2BD0314B1B781A
:10D0A000002B2AD132062CD472B62F4D2F4C2F468E
:10D0B000012326602B7062B672B623681B060CD45F
:10D0C0003B781BB9F4E72B78002BF1D062B602F065
:10D0D0007DFB72B623681806F5D5254B1B68002228
:10D0E0002A7062B6234A107843FA00F0BDE8F08156
:10D0F000002070470020BDE8F081FFF781FE320676
:10D10000D2D572B61C4DDFF87C801C4C06F040076F
:10D11000FFB206F03F06D8F80030DFB123F010036D
:10D12000C8F8003001232660134A2B7062B672B62D
:10D13000236819060CD413781BB9ECE72B78002B65
:10D14000E9D062B602F042FB72B623681B06F5D541
:10D150000B4BC3E743F01003C8F80030E2E700BF11
:10D1600050430100429FFF1F449FFF1F00B0034038
:10D1700010B00340419FFF1F439FFF1F00B00B40B3
:10D1800010B00B400CB00B400A4A0B49136843F433
:10D19000805313600B7843B9084BC0221A70084BB8
:10D1A00080F30C0000B218807047044B80221A7084
:10D1B000F5E700BF2C800440459FFF1F21C00C40B5
:10D1C00000C00C40F0B51B4B1B4E596818689A689C
:10D1D000DB6885B06C460FC4337899071DD5174AB4
:10D1E000174C1378174913F0700318BF1370164AC1
:10D1F000164B8027177000263320032226706D46B9
:10D2000008701A7072B6043C45F001052046A84724
:10D2100062B6237813F0700309D10D4B064901E083
:10D22000013B02D00A78D207FAD505B0F0BD2370D1
:10D2300005B0F0BD7C430100010002400000024047
:10D24000040002400B000240070002400A000240B6
:10D25000410D0300B0F5006F0AD210B5094B1B78E1
:10D26000DB07044606D504F1A0500078C0B210BD1B
:10D2700000207047FFF7A6FF04F1A0500078C0B26D
:10D2800010BD00BF01000240B0F5006F17D238B5E5
:10D290000F4B1B78DA070D46044611D504F1A05058
:10D2A0000378AB420AD00B4A137813F0700318BF0F
:10D2B0001370074A05701378DB07FCD538BD70473B
:10D2C000FFF780FF04F1A0500378AB42EBD1F5E704
:10D2D000010002400000024008B5104C08E023683D
:10D2E00059050DD423681A050FD42368DB0411D423
:10D2F00023685803F3D501F023F823685905F1D5C5
:10D3000002F0C2FA23681A05EFD502F053FB236836
:10D31000DB04EDD500F0A8FEEAE700BF348004404E
:10D3200008B5FFF7D9FF00BF014B10221A807047E4
:10D3300000200540704700BF094908B50B6830B1AF
:10D340006A461844A2F58052904202D208601846FC
:10D3500008BD03F031FE0C2303604FF0FF3008BD21
:10D360002493FF1FFEE700BFEFF3138070B9EFF3C4
:10D3700010836BB9EFF305825AB94FF48070EFF365
:10D3800011832BB1984228BF184670474FF0FF30E9
:10D3900070470F2A01D81846F1E7014BD05CEEE741
:10D3A000F0E300E0F0B44D1E2E46002400E001340E
:10D3B000B0FBF2F302FB1300092800F130078ABF2B
:10D3C0003730F8B2C0B206F8010F1846002BEED184
:10D3D0000A1953704CB1107815F8016F2870013399
:10D3E000E01A834202F80169F5DB0846F0BC704799
:10D3F0002DE9F04F0D4685B085EAE5790146824674
:10D4000017461C46A9EBE57903F03AFD002840F0E9
:10D410002F812AF000484046C74903F031FD00281B
:10D4200047D14046C44903F00DFD0646002840D1CF
:10D430000021504603F0FCFC002814BF0420032008
:10D4400048451DDB002DC0F274815046002103F0D9
:10D45000EFFC254648BB49214E22462321706270CD
:10D46000A3700334002E00F07681A019202304F865
:10D47000013BA042FBD10023037005B0BDE8F08F53
:10D48000002DC0EB0906E0DA002E00F05281A5194C
:10D49000202304F8013BAC42FBD15046002103F0AD
:10D4A000C7FC002800F0228100262D232B706C1C65
:10D4B000D1E702AB01AA3946504603F06DFDBB46E9
:10D4C0008046DDF80490002F57D0C9F10003BB421D
:10D4D00000F39480404604F033FB0646B145B8BFE4
:10D4E0000136B9F1000F40F098800136DDF808E010
:10D4F000BEF1000F53D00136A81B002804EB060133
:10D5000053DC23462D221A700133B9F1000F63D189
:10D5100037B11A46302002F8020B2E2058701346FD
:10D520008B4220D25F1C98F800201A708F4208F1BD
:10D53000010819D0019A4FF02E0E0BE083F801E09C
:10D5400002338B4203F101070DD218F8010B18705A
:10D550008F4209D0013A0192002AEFD03B468B421C
:10D5600003F10107F1D31946002DC0F2A980002371
:10D5700020460B7005B0BDE8F08FB9F1000FA4D1C3
:10D5800090F800806D496E4A012301939946B8F1E5
:10D59000340F8CBF884690464FF0FF3397E7A81BA7
:10D5A000002804EB060140F3D880014422460138EC
:10D5B0004FF0200C02F801CBC2F1010303442344D5
:10D5C000002BF7DC20EAE07301332344BEF1000FA7
:10D5D00098D1B9F1000F9BD0A2DA002FA0D01A4643
:10D5E000302002F8020B2E275F70C9EB020302F80D
:10D5F000010B9342FBD10022019291E7C7F1000990
:10D600000126B1453046B8BF0136B9F1000FDFF849
:10D610003081CDF804903FF468AFBFF667AF002FBC
:10D620003FF464AF09EB0703984207F102067FF667
:10D630005DAF002F07DD5046424903F05BFABBF1B6
:10D64000010B8246F7D102AB03AA5946504603F0BC
:10D65000A3FCDDF80490039A7B1CC9EB02029A42FA
:10D6600008BF09F10109804608BFCDF804903DE7E5
:10D670000021504603F0DCFB002814BF04200320E7
:10D6800048453BDA002DC0EB09063BDB4FF07E53EB
:10D690005046002163F31E0003F0CAFB2546002814
:10D6A00041D14E2341222370A37062700334002EB7
:10D6B00051D0A019202304F8013B8442FBD1DAE6C3
:10D6C000A8194342002B6FEA00007FF750AF0A46CB
:10D6D000202502F8015BC2F1010303440B44002B37
:10D6E000F7DC20EAE0730133194440E749214E2278
:10D6F000462329706A70AB70E81CBCE6002D16DB6F
:10D700000026C3E79EB1A519202304F8013BAC42D3
:10D71000FBD14FF07E535046002163F31E0003F00F
:10D7200087FB88B100262D232B706C1CB9E725469A
:10D73000EFE72546B1E600BFFFFF7F7F9043010082
:10D740008C430100000020414E2341222B70AB701E
:10D750006A70E81C8FE620468DE62346D5E600BFBA
:10D76000704700BF10B40F4B53F8302092F880423E
:10D770002CB1012369B182F8803010BC704703EBF3
:10D78000C0035B681A6841B922F002021A6010BC3B
:10D79000704782F8003110BC704742F003021A60F3
:10D7A00010BC7047944301001C4A02EBC0030129DE
:10D7B0005B6811D004291BD052F83000002280F899
:10D7C000802229B1022920D0032922D01A60704773
:10D7D0004FF480721A60704752F830004FF4A27212
:10D7E00080F880121A601A6822F020021A607047CE
:10D7F00052F830104FF4A272012081F880021A60B2
:10D800001A6842F020021A60704740F203121A6050
:10D8100070474FF481721A60704700BF9443010053
:10D82000212817D8F8B5042A13D8DFE802F0494CAC
:10D830004F1446002C4872B6236823F4702343F03B
:10D840008072C4F384011643236040F8215026609F
:10D8500062B6F8BD70474FF41026244B03EBC003AB
:10D860000D465C68216811F4E06134D0204B214AF8
:10D870002149C3F89C2104F140422048C3F8A41177
:10D88000A2F592211E4FC3F8A0017C291D48C3F8C0
:10D89000A871C3F8AC01CDD9A2F594237C2B18D97B
:10D8A000A2F596237C2B19D9A2F598237C2B17D9A6
:10D8B000A2F59A227C2A15D9F8BD4FF43026CCE780
:10D8C0004FF40026C9E74FF44026C6E74FF4202660
:10D8D000C3E70D48AFE7FFF767FFC7E70B48AAE7C5
:10D8E0000B48A8E70B48A6E72893FF1F94430100C5
:10D8F0000082FF1FF188FF1F9988FF1FC588FF1F47
:10D900006D88FF1F4188FF1F6093FF1FB093FF1FAB
:10D91000E093FF1F0094FF1F1A4B03EBC00010B4ED
:10D92000426802F14043A3F592217C2905D9A3F571
:10D9300094217C2913D8144900E0144972B6136865
:10D94000134C23F08773C2F3840023F4803343F035
:10D950008073136041F8204062B610BC7047A3F595
:10D9600096217C2909D9A3F598217C2907D9A3F50B
:10D970009A237C2BF1D80749E0E70749DEE70749FE
:10D98000DCE700BF944301006093FF1F2893FF1F53
:10D9900061D700000094FF1FB093FF1FE093FF1FAB
:10D9A00030B4054B054D064C002210211A602A6048
:10D9B0002060196030BC704714D0034004D003408D
:10D9C00000D00340282838B52ED0002904464FDD6A
:10D9D0005F4B1B78012505FA03F28A4202D8212801
:10D9E00037D938BD0338C2B2012A3AD9202C4AD0DF
:10D9F000192C48D0574A126802FB011222FA03F38D
:10DA00001D2800F29B80DFE800F0928B847D9999BD
:10DA1000766F99999999999999999968615A5399B1
:10DA20004C99999999999945494B1B780B2B08D991
:10DA30000C2B1CBF0C3B19410846BDE83840FFF7D2
:10DA4000A3BBC3F10C0399400846BDE83840FFF77B
:10DA50009BBB2946FFF786FE2946BDE83840FFF705
:10DA6000A3BE3D4A126802FB011222FA03F3C7E784
:10DA70002128B6D80021FFF775FE20460121BDE818
:10DA80003840FFF791BE354A126802FB011222FAB4
:10DA900003F3B5E73249334A0B604FF45173136017
:10DAA00038BD3149314A0B604FF45173136038BDB2
:10DAB0002F49304A0B6040F24443136038BD2E4971
:10DAC0002E4A0B6040F24443136038BD2C492D4A66
:10DAD0000B6040F24443136038BD2B492B4A0B6066
:10DAE00040F24443136038BD29492A4A0B6040F292
:10DAF0004443136038BD2849284A0B6040F2444330
:10DB0000136038BD2649274A0B6040F24443136036
:10DB100038BD2549254A0B6040F24443136038BDA7
:10DB20002349244A0B604FF45173136038BD2249D6
:10DB3000224A0B604FF45173136038BD212C3FF61D
:10DB400050AF7F29D4BF00210121204693E700BFB9
:10DB50000894FF1F088003400890034008800B4092
:10DB600010800B4048A0044018800B404CA004409B
:10DB70001880034008B004401080034004B0044003
:10DB80004080034018C004403880034014C0044063
:10DB90002880034010B00440208003400CB00440B3
:10DBA0003080034010C00440488003401CC0044043
:10DBB000189003403490044010900340309004408B
:10DBC00038B1102828BF1020044AC3B2107813704F
:10DBD0007047024A01231078137070470894FF1FA2
:10DBE0002DE9F8430E4680463249334D304603F066
:10DBF0001FF947F6122300281ABF1D464FF00209ED
:10DC00004FF00109002425FA04F002F01BFF4FF049
:10DC10005E51074602F06EFF0146304603F01CF9E4
:10DC200030B90134072CEED1E80902F00BFF0746AA
:10DC30003146384603F012F84FF07C5102F050FEA6
:10DC400003F05AF94FF6FF729042A8F1030328BF80
:10DC50001046012B29D9B8F1170F17D8174B23FA03
:10DC600008F303F0010383F0010223B9B8F1190F9F
:10DC70000FD0BDE8F883124B124D13491A6044EAE5
:10DC8000C9042A6008601C60BDE8F883B8F1200F61
:10DC9000ECD10E4B0E4D0F49002244EAC9041A6024
:10DCA0002A6008601C60BDE8F8830B4B0B4D0C49E3
:10DCB000F2E700BF001BB740006CDC026006F0001A
:10DCC00000800340048003400880034000800B4034
:10DCD00004800B4008800B400090034004900340F8
:10DCE00008900340212801D8FFF73CBD704700BFD2
:10DCF000212806D8044B53F8303093F80002C0B204
:10DD000070470020704700BF94430100212801D8CC
:10DD1000FFF74ABD704700BF72B60C490C4B0D4A65
:10DD20001B680868126862B6520102D5322B88BFA0
:10DD300001300949C3F5BB334FF47A72FF33A1FBBD
:10DD4000031302FB00F000EB93107047489FFF1F86
:10DD500018E000E004ED00E0ABAAAAAA2DE9F84320
:10DD6000054672B6204F214B214A1B683C68126859
:10DD700062B6520102D5322B88BF013495B3C3F588
:10DD8000BB331C4EDFF86490DFF86480FF334FF440
:10DD90007A72A6FB031302FB04F404EB931472B62D
:10DDA000D9F800103A68D8F800E062B6C1F5BB3384
:10DDB000FF33A6FB03031EF0806FC4EB93134FF4F5
:10DDC0007A7002D0322988BF013200FB0233B3F5EA
:10DDD0007A7F04D3013D05D004F57A74DFE701F0C2
:10DDE000F5FCDCE7BDE8F883489FFF1F18E000E082
:10DDF00004ED00E0ABAAAAAAF8B52D4B2D49DFF837
:10DE0000D0E0DFF8D0C02C4E2C4D2D4C2D4A2E4F9B
:10DE10004FF4000018604FF0807018604FF00070F1
:10DE200018604FF0806018604FF0006018600020AC
:10DE3000086028234BF6FF71CCF80010CEF80030B4
:10DE4000336013602B6023603B60B36293620922EE
:10DE500045F8242CC4F8D80F05F57F65C7F8D41F02
:10DE600007F5FF2707F5FA67C6F8F83F2B6006F5B8
:10DE7000FF26C4F8D42F05F5FD2504F5FF243860EE
:10DE800006F2F4761148316005F5FF6504F5FD648E
:10DE90002B6023600260FFF755F81920FFF75EFF43
:10DEA00000F05AFE40F21310BDE8F840FFF756BFED
:10DEB00008E100E004800340148003402480034014
:10DEC0002C8003401C8003403480034000800B40C2
:10DED0000C800340088003402DE9F84F214B1B685C
:10DEE00007460BB101221A70DFF888901E4D99F891
:10DEF0000040DFF884801D4E0134272C8ABF4FF08C
:10DF0000000A5FFA84FA5446AB462B78A34216D136
:10DF1000FFF72AFA40281FDC33791B06F5D59BF85A
:10DF200000300133272B86BF00221346DAB218F8DF
:10DF30000330DBB2F3712A702B78A342E8D00C498E
:10DF40000A4BFFB208F804700120AC22087089F86F
:10DF500000A0DA70BDE8F88FFF28D6DD01F036FCAE
:10DF6000D3E700BFC09FFF1FBD9FFF1F00C006403B
:10DF7000BC9FFF1FC49FFF1F549FFF1F1C4BDFF858
:10DF800094C01A681B49F0B542F480521A4D1A60C9
:10DF9000DFF884E0194F1A4E1A4C00238CF8003039
:10DFA0004FF451722B701F2840F213358EF8003059
:10DFB0003B70337025600A6012D819460124124A5A
:10DFC000124D11701248547000212C274026937274
:10DFD0004FF4003491701174D7702E700460F0BD4E
:10DFE000C0F34431C0F3471400F01F03E7E700BF5C
:10DFF000348004400CC00440519FFF1FBD9FFF1F91
:10E00000BC9FFF1F08C0044000C0064031E400E090
:10E0100004E100E0509FFF1FC49FFF1F034B1B68DC
:10E02000DB0401D5FFF758BF704700BF34800440C0
:10E0300010B5044C237823B101F0C8FB2378002BE2
:10E04000FAD110BDBC9FFF1F054A064B10781B7804
:10E05000C0B2DBB2984238BF4030C01A704700BF30
:10E06000509FFF1F519FFF1F30B42B4B1A7994060E
:10E070001FD52A48DA790378294901333F2B0978DB
:10E08000C8BF00238B42D2B203D0264CD9B2E2548F
:10E090000170254A116861B1244A1278D2B29342C4
:10E0A00036BFC2F140029B1A9B18272BC4BF012325
:10E0B0000B70194AD378DBB2180611D45A060DD565
:10E0C000154B1B795B0609D5194B1A491B680022B1
:10E0D0000A7003B11A70104B2C22DA7030BC7047F2
:10E0E00011790906EAD5144910480C780178C9B2AB
:10E0F0008C420DD04A1C272A84BF00210A460F4DAE
:10E10000054C98BFD1B2AA5CD2B2E2710170D5E7DA
:10E110006C21D170D2E700BF00C00640509FFF1FA6
:10E12000519FFF1F7C9FFF1F4C9FFF1FBD9FFF1F25
:10E13000C09FFF1FBC9FFF1FC49FFF1F549FFF1F57
:10E1400021282FD8184B195CFF292BD0174B184AC0
:10E15000DFF870C003EBC000F0B54368DFF868E09B
:10E16000144F154D154E00241C60DEF800300120C0
:10E1700043F020038840CEF8003014604FF4A073C1
:10E1800038602E60C2F800C0013BFDD113689B05CA
:10E19000FCD42023013BFDD1094B09B233F8110017
:10E1A00080B2F0BD00207047A444010094430100F8
:10E1B0000050044008500440045004400000020392
:10E1C0000051044080014A0038800440431E032B64
:10E1D00014D872B60A4951F8230068B170B4094CDA
:10E1E000058834F81320466841F82360521B24F850
:10E1F000132062B670BC704762B67047002070474B
:10E2000020A0FF1F88A2FF1F013803280BD872B679
:10E21000074B53F8203043B100205B680130002BDE
:10E22000FBD162B67047002070471846F9E700BF7F
:10E2300074A0FF1FF0B472B61A491B4E012311F8E7
:10E24000014B194F9A00240742F0010505D556F8F5
:10E25000324064B156F83520BAB10133052BEED106
:10E2600062B6124B00221A70F0BC00F0F1BC0F4CE9
:10E270000F4D217847F8325007EB431308304A1E00
:10E280005860227062B6F0BC70470849094B0A78A2
:10E2900047F8353007EBC5030830013A58600A707B
:10E2A00062B6F0E7F04401000080FF1F9DA0FF1F51
:10E2B00088004000C8004000431E032B1DD81B4AA5
:10E2C000400140F0100030B4104472B6184CE25CCB
:10E2D000032A1BD8DFE802F00212151703220D886B
:10E2E000E25410F0080F14BFC823882343EA054303
:10E2F00008310360416062B630BC704708300222CA
:10E30000EDE70522EBE708300422E8E7094A52F876
:10E31000230038B1084A52F82300416042F8231024
:10E3200062B6E9E742F82310034AF7E70080FF1FCF
:10E33000ACA0FF1F74A0FF1F84A0FF1F00BE70478A
:10E340002DE9F04FDFF814A3DFF814B387B044E0F1
:10E35000AC4F4FEA930807EBC809013ED9F80420F7
:10E3600003F00803F6B2A2F1080003F0FF04002B4B
:10E3700040F0FE8057F838301B0C99B222F8081C88
:10E38000002B00F0EC80A04B22F8064C42F8044C25
:10E3900053F82620002A00F0CD819C4D55F82630F8
:10E3A00058609B4C45F8260034F81630194424F880
:10E3B000161000F02DFC002800F0C081954A964B05
:10E3C00019F0080F00F1080018BF1346C9F804003F
:10E3D00047F8383008238AF800309AF80040E4B251
:10E3E00061071CD58D4B1B78B3B18D490A7802F0BB
:10E3F000FF0322B1013BDBB20B7003B900BE8949B8
:10E400000A7802F0FF032AB1013BDBB20B70002B4C
:10E4100000F0668100F0B6FC04238AF8003004F0B6
:10E42000080303F0FF02002B00F0C6809BF80030C9
:10E43000DBB21E098CD19A08724F57F8321007EBE5
:10E44000C200C1F38301013940680C2900F28380C6
:10E45000DFE801F078788181818181814281818149
:10E4600007000168704D714B40680193694B47F894
:10E4700032306F4E686040F2816288B26B4B296027
:10E480000024012190421C603C61BC61317000F2AB
:10E49000E980B0F5D06F80F00F82B0F5817F00F099
:10E4A000DA8100F26B81802800F00182822840F03E
:10E4B000D881A8885F4B00F07F00042800F2D28149
:10E4C0005D4A80000344147054701878840740F14A
:10E4D00002831170022174E1544B01931A6832B324
:10E4E000564B534E564819883478057840298E4645
:10E4F00045F0020828BF4FF0400E002C84F00104C4
:10E500003470CEEB01010CBF8824C82407EBC80689
:10E5100089B285F0010544EA0E447260198047F81B
:10E52000384072440570002966D0019B1A603E4B4A
:10E530001A88B2F5A06F0ED100219A785970414B1C
:10E540001A7008E03849404C0D68A54200F09980E7
:10E55000304947F832103D4A012313703AE72D4AFB
:10E560002D4B19F0080F18BF134647F8383031E724
:10E5700000F06EFB364A374952F82630002B00F087
:10E58000E48058688C5D42F8260003F10802C9F85F
:10E590000420032C05D8DFE804F02C0229260222EF
:10E5A0008A551A8819F0080F0CBF8823C82343EA3C
:10E5B000024347F838300DE7E00700F19480210668
:10E5C00000F1D280A20706D5234A244913780220FD
:10E5D000DBB213700870E30602D5204B10221A70CC
:10E5E00007B0BDE8F08F04228A55DAE705228A5584
:10E5F000D7E703228A55D4E7BEF1400F18BF0022A7
:10E6000093E700BF0080FF1F20A0FF1FCC9FFF1FCC
:10E6100088A2FF1FC800400088004000A8A0FF1F7C
:10E6200031A0FF1F20A1FF1F94A0FF1FC89FFF1F45
:10E6300030A0FF1FC0200740A0A0FF1FDC9FFF1FCE
:10E640009CA0FF1F98200740210900039420074049
:10E6500074A0FF1FACA0FF1F882007408020074048
:10E6600090200740B0F5106F00F03E8140F2A2808C
:10E6700040F62112904240F01C82A44A01231370FC
:10E6800069E74C68A2498C427FF462AF0178A929FE
:10E690007FF45EAF417845297FF45AAF8178C22973
:10E6A0007FF456AFC1786B297FF452AF99489A4EE8
:10E6B0000178347881F00105002C41F002010570E9
:10E6C0000CBF8820C82084F0010447F8310007EB14
:10E6D000C10192483470002505244D60047037E76D
:10E6E00000F0E0FE96E68E4B88488A491A614FF0AA
:10E6F000020E80F800E08B4F0A708B491960996018
:10E700008A4E8B4D8B4C9A610D213970FF213170EF
:10E71000DFF848E229702270874D884A8EF8001091
:10E720009F27012406F8047C5D600470DA6007B05E
:10E73000BDE8F08F43F82600814D32E6814A47F864
:10E74000380013780133137044E68B5D032B00F21D
:10E75000A78001A252F823F0D5E30000D5E3000022
:10E76000AFE70000A9E700006E49714B80220D2041
:10E7700008701A70A2077FF52EAF25E740F202322B
:10E78000904240F08E81AA8802F07F02042A68D865
:10E790006D88002D65D16348029192001044027883
:10E7A00042F00202027048E101238B5512E6002379
:10E7B0008B550FE6B0F5086F53D16348634A007874
:10E7C0001070ED888D4280F09B815248047844F0AF
:10E7D000020C07EBCC01402DAE464FF0010328BFE1
:10E7E0004FF0400E4A6002EB0E09CEEB05014FEAF6
:10E7F0000E4802930025C82242EA080384F0010271
:10E8000047F83C3035700270DFF814C1424BDFF836
:10E81000048151BBBEF1400F7FF42FAF42F00202E2
:10E8200007EBC203DFF8F8E0C3F8049095BB0D04D2
:10E8300045F088059DF8083033704029047009EBD5
:10E8400001034EF832507FF418AF0021404A01987E
:10E850001180036011E7AA8802F07F02042A40F2C7
:10E860002D81304B0F221A7007E74029D6D942F08C
:10E8700002020CEBC200C0F804907DB135489DF84F
:10E8800008501D70403988F8004009F140034CF8E9
:10E890003200DBE70D0445F0C805CBE72248EEE780
:10E8A00019F0080F0CBF022303238B5592E5274A6A
:10E8B00002211470547084E727494A68002AD0D096
:10E8C0006C88B5F804E003E00C314A68002AC8D02F
:10E8D0000B88A342F8D14B887345F5D1240A032C49
:10E8E0000CBF117809896CE7174A0D4CA978117093
:10E8F00004F1800502E00834AC4231D0236A1A06E4
:10E90000F9D5606A083800F0A3F9F4E794200740CD
:10E91000010004009CA0FF1F30A0FF1F31A0FF1FBB
:10E920000080FF1FC020074088004000882007406B
:10E930008020074098200740E09FFF1F34A0FF1F62
:10E94000CC9FFF1F9DA0FF1FA8A0FF1FA0A0FF1F1F
:10E95000DC9FFF1FC8004000F44401008C200740EA
:10E960006F49704B704A02917049714D714C059618
:10E9700003954FF00009884616461D460494286802
:10E9800028B1446800F064F92046002CF9D1002336
:10E990002B60039B30681A46002342F8293028B1C7
:10E9A000446800F055F92046002CF9D1002232606D
:10E9B000029A98F800301146002241F8042B049A7C
:10E9C0000291023B4FF0000122F81910032B07D8E7
:10E9D000DFE803F0470247024FF0010388F80030F8
:10E9E00009F10109B9F1040F05F1040506F1040666
:10E9F00008F10108C3D1504B059EDFF85491DFF8B0
:10EA0000548100211970012518F8013B09F8043BD5
:10EA10001B072BD4AC0044F0020244F00304002393
:10EA200047F8323047F83430444B994505F1010539
:10EA3000EAD13378029383F00105002189468846A4
:10EA40008E460A463E48047844F0020C07EBCC039D
:10EA50000393029B002B039B5A600CBF8822C822A1
:10EA6000CAE64FF0000388F80030B9E700F0D0F8AC
:10EA7000AC0007EB451300F10802002837D05A60BC
:10EA8000304B47F8343000F0C3F844F0010307EB93
:10EA9000C30200F1080100B351602B4A47F833204C
:10EAA000B9E7B0F5A06F7FF4DCAE01230025029337
:10EAB000C3E740F621229042F7D0D2E66D88002DC0
:10EAC0007FF4CFAE2148029192001044027822F0E8
:10EAD00002020270B1E7022173E6174B44F0010213
:10EAE0001B7847F83200144A0133137093E7124B36
:10EAF000114A1B78AC00013347F834001370C2E7A9
:10EB000040298E464FF0010328BF4FF0400ECEEB58
:10EB100001014FEA0E4802EB0E090025029391E72E
:10EB200084A0FF1F20A0FF1F74A0FF1FACA0FF1F29
:10EB3000CC9FFF1F88A2FF1F9DA0FF1FD42007406E
:10EB40009CA0FF1F88004000C8004000C020074074
:10EB5000C4200740F04401002DE9F843204C00F0A8
:10EB6000AFFF002204F1880023461A605A60083380
:10EB700083424FF00001F8D11A4A1B4F13681B4D16
:10EB80001B481C4EDFF87880DFF878C0DFF87890FB
:10EB9000DFF878E043F480231360C4F307233B706D
:10EBA000C4F307432B70240EFF2302F528320470B0
:10EBB000114D88F8003011488CF80030D432337091
:10EBC000012389F8003070268EF800104FF400748D
:10EBD000102107F8183C2E7004601170BDE8F8830E
:10EBE0000080FF1F348004409C200740B020074075
:10EBF000B42007401020074049E400E008E100E0AD
:10EC000080200740882007409420074000210740CB
:10EC100072B60D480268B2FA82F30F2B10DC4FF087
:10EC20000041D94022EA0102026062B6074803EBC4
:10EC3000C303DB00C2180021C15010465160704769
:10EC400062B60020704700BF0C94FF1FBC83FF1FFB
:10EC50000D4B0E4AC31AA2FB03231B090F2B0CD822
:10EC60000B4A127852B972B60A484FF00041026856
:10EC700021FA03F31A43026062B67047064A12781B
:10EC8000002AF0D0FFF7D6BABC83FF1F398EE338D5
:10EC90009DA0FF1F0C94FF1FA8A0FF1F38B50E4BAF
:10ECA0000E4C1B68218805468BB1B1F5917F05D2CA
:10ECB0000B4A4B1C55549BB2238038BD0022084898
:10ECC00098470021064A55540123238038BDB1F5E9
:10ECD000917FEDD338BD00BFD4A0FF1F92A2FF1FCC
:10ECE00098A2FF1F2DE9F843224E234F31680123DC
:10ECF00080463B70C1B1214D4B8801EB830001334D
:10ED000000220F2BC0F808802A7004D84B80002303
:10ED10003B70BDE8F88340230B800320FFF7CCFA5B
:10ED2000FFF776FF3060F2E7DFF8549099F8003093
:10ED3000002BEED0114D45F6215408E0013C12D0D5
:10ED40002B7883B900F042FD99F800307BB10320A5
:10ED5000FFF75AFA0528F1D8FFF75AFF014630604D
:10ED60000028EBD0C8E701232B70BDE8F883BDE88D
:10ED7000F88300BFF0A0FF1FC4A0FF1FF4A0FF1F77
:10ED8000A8A0FF1F094B1B787BB910B5084C216860
:10ED900009B14B8803B910BD9B000B800320FFF71E
:10EDA0008BFAFFF735FF206010BD7047C4A0FF1F2E
:10EDB000F0A0FF1F2DE9F041AD4E33680746002B50
:10EDC00000F092801D885A88910803EB810104327B
:10EDD000AA428C6842D25A8004F00F064FEA1428E7
:10EDE000A449A6F1080208F00F00C4F30313062A91
:10EDF00000F101050B701AD9B31E012B5FFA88F0E0
:10EE00004ED9052E48D0042E00F0A481731F022B8A
:10EE10007FD90F2E0ED1F72842D8F02802D0964B7A
:10EE20001B883BB1FFF73AFF0020BDE8F08127B116
:10EE3000BD4202D00020BDE8F081082EC4F30333A8
:10EE400000F08780092E11D00A2E40F094800A2B02
:10EE5000F0D18A4B8A4A1B68A02181E01846FFF74F
:10EE6000F7FE0420FFF7B2F93060B5E7092BE1D1D6
:10EE7000270E00F07B81834B814A1B689021C4F3ED
:10EE800007461170EDB2FCB2002B00F09D802246C7
:10EE900031462846984797E0F02843D9F72841D0D3
:10EEA000F1380E28C6D801A353F820F063F0000013
:10EEB00047F0000035F0000035EE000035EE0000B0
:10EEC00027F0000035EE000007F1000035EE0000ED
:10EED000D1F00000EBF000000FF0000035EE000074
:10EEE000F7EF0000DBEF0000674B1B78002BA1D091
:10EEF0000420FFF76BF90346306000289AD005889C
:10EF0000002D7FF460AFFFF7A3FE35602846BDE813
:10EF1000F081FFF7C3FEC4F30740FFF7BFFE072EE3
:10EF200002D1200EFFF7BAFE534B584A19885848B1
:10EF30001468584D524A017000270E0AF0201F80B5
:10EF40002E7010700CB301225348A0470120BDE879
:10EF5000F081082B7FF46EAF504B494A1B6880212B
:10EF6000C4F307461170EDB2240E6BB32846224657
:10EF70003146984728E00B2E11D10B2B7FF45AAF66
:10EF8000474B3F4A1B68B021EAE7464B1B68002B02
:10EF900000F0FB80404898470120BDE8F0810C2E2E
:10EFA00040F000810C2B7FF445AF3F4B344A1B6887
:10EFB000C0211170EDB2C4F30746002B00F0C880E9
:10EFC00028463146240E98473849314A314B0D7056
:10EFD00016701C700120BDE8F081354B1B68002BBA
:10EFE00000F0D6809847C4F30746254BEDB2240EB7
:10EFF00083F80080E8E72F4B1B68002BF2D12E4BE3
:10F000001B68A3B1FE209847C4F30746EDE72B4BDE
:10F010001B68002BE6D1284B1B6843B1FC209847A6
:10F02000C4F30746E1E7264B1B68002BDAD1C4F393
:10F030000746DAE7234B1B68C4F30746002BD4D0FE
:10F0400030469847D1E7204B1A68002AEFD0260CAB
:10F05000630C06F07F0003F47E531843F6B290472A
:10F06000C3E71A4B1B68C4F30746002BE8D1BCE783
:10F07000FCA0FF1F96A2FF1F92A2FF1FD8A0FF1F98
:10F0800090A2FF1F0CA1FF1FA8A0FF1FD4A0FF1F6D
:10F0900094A2FF1F95A2FF1F98A2FF1F04A1FF1FAC
:10F0A00008A1FF1FECA0FF1FC8A0FF1F97A2FF1F12
:10F0B000B4A0FF1FB8A0FF1FBCA0FF1FF8A0FF1F38
:10F0C000E8A0FF1F00A1FF1FD0A0FF1FE4A0FF1FAB
:10F0D0003F4B1B68002B85D13E4B1B68002BA6D0F5
:10F0E000FA209847C4F307467FE73B4B1B68002B89
:10F0F0007FF478AF374B1B68002B98D0FB209847E4
:10F10000C4F3074671E7354B1B68002B7FF46AAFE9
:10F11000304B1B68002B8AD0F8209847C4F3074671
:10F1200063E70E2B7FF486AE2D4A2E4B1268E0214A
:10F130001970002A47D0260C610C06F07F0301F4F9
:10F140007E511943EDB2A1F5005128469047F6B221
:10F15000240E39E7FFF7A2FDC4F30740FFF79EFD39
:10F16000200EFFF79BFD0020BDE8F0811E4B1D4ADD
:10F170001B6880211170EDB2C4F3074683B131469C
:10F1800028463A4698473C461EE70120BDE8F081F4
:10F19000104B1B68002B3FF44AAFFF20984746E70F
:10F1A0001C4611E70D2EBCD10D2B7FF443AE0F4B47
:10F1B0000C4A1B68D0211170EDB2C4F30746002B36
:10F1C0007FF4FEAEC4E7C4F30746EDB2240EFBE6BF
:10F1D000E0A0FF1FBCA0FF1FC0A0FF1FB0A0FF1F2B
:10F1E000CCA0FF1F90A2FF1F04A1FF1FDCA0FF1FE8
:10F1F00070B5124E33788BB1114D286840B14388F9
:10F20000C218147A6CB9FFF723FD33782C602BB148
:10F210000220FEF7DBFF28600028F0D14FF0FF301E
:10F2200070BD02880133934202D24380204670BDF4
:10F23000FFF70EFD002320462B6070BDA8A0FF1F26
:10F240001CA1FF1F70B50D4E33788BB10C4D286893
:10F2500040B1438803441C7A6CB9FFF7F9FC33785A
:10F260002C602BB10220FEF7B1FF28600028F0D1FE
:10F270004FF0FF3070BD204670BD00BFA8A0FF1F3B
:10F280001CA1FF1F38B5164D2868E0B101884488DD
:10F29000A14213DD03191B7A83B104F10803C218DC
:10F2A0000C1B002302E012F8011F21B10133A3421D
:10F2B000F9D1204638BD1C46204638BDFFF7C8FCB2
:10F2C0000020286038BD074B1B780BB9002038BDE3
:10F2D0000220FEF77BFF28600028D7D1F6E700BFA9
:10F2E0001CA1FF1FA8A0FF1F2DE9F04F3D4D0122DB
:10F2F00083B02A7071B3DFF8F8A0DFF8F880DFF888
:10F30000E89083460E46DAF80000002835D0364BE8
:10F3100001934488019BC4F14001B14228BF3146AA
:10F3200067180022BFB21A70761A478000F10802EF
:10F3300049B1013C224459441BF8014B02F8014FEA
:10F340005945F9D147883F2F09D8284B05221A7013
:10F35000002ED8D10020287003B0BDE8F08F4022E5
:10F36000224B02800146002401201C70FEF7A4FFFE
:10F37000CAF80040002EC6D1ECE798F800204AB346
:10F38000194B019344F2D95401270BE0013C17D0EB
:10F3900099F80020A2B92A7000F018FA2F7098F896
:10F3A0000020BAB10120FEF72FFF0528EED82F70FC
:10F3B000FFF72EFCCAF800000028AAD1013CE7D1D3
:10F3C0000199012200234FF0FF300A702B7003B027
:10F3D000BDE8F08F00234FF0FF302B7003B0BDE885
:10F3E000F08F00BF10A1FF1F18A1FF1F20A1FF1F5A
:10F3F00014A1FF1FA8A0FF1F00B583B002AB01211D
:10F4000003F8010D1846FFF76FFF03B05DF804FB2A
:10F4100038B50E4D0E4C2B68012020702BB158884A
:10F4200000232370C0F1400038BD0A4B1B7813B98C
:10F430000020207038BDFEF7E7FE0528F8D8FFF75A
:10F44000E7FB034628600028E9D1F1E714A1FF1F7C
:10F4500010A1FF1FA8A0FF1F0F4B1B78DBB110B539
:10F460000E4C2168B1B14B88A3B10D4800223F2B4F
:10F47000027007DC07330B4401F1470003F8012F4A
:10F480008342FBD140230B800120FEF715FF0023B0
:10F49000236010BD10BD7047A8A0FF1F14A1FF1F5F
:10F4A00020A1FF1F0D4B1B78BBB910B50C4C216878
:10F4B00003F0FF024B883F2B07DC07330B4401F1BD
:10F4C000470003F8012F8342FBD140230B8001202A
:10F4D000FEF7F2FE0023236010BD704710A1FF1F4E
:10F4E00014A1FF1F10B4EFF3108272B6437F33B93B
:10F4F000017F012907D003290FD00123437702B9E7
:10F5000062B610BC7047124C2168A1B11149436129
:10F510000B68836108605861EFE70F4C216881B187
:10F520000E4943610B688361086058610C4B4FF0D2
:10F5300080511960E1E7074B4161816120601860EB
:10F54000DBE7064B4161816120601860EEE700BF98
:10F5500034A1FF1F30A1FF1F24A1FF1F28A1FF1FFF
:10F5600004ED00E070B5EFF3108272B60C4C206829
:10F5700080B10C4E00254369236073B19D6102B9CF
:10F5800062B6457783689847EFF3108272B62068B9
:10F590000028F0D102B962B670BD3360EFE700BF5A
:10F5A00024A1FF1F28A1FF1FFFF7DCBF184A30B4BA
:10F5B0001468002C27D0036821688B420ED2CB1A26
:10F5C00000218460C1602360E06010600223037545
:10F5D00030BC704711688B42144608D3A2685B1A8E
:10F5E0000360002AF6D18260C460A060EEE7D268B2
:10F5F000C2608460E060C568CB1A0222A860236004
:10F60000027530BC70478460C4601060DEE700BFE4
:10F610002CA1FF1FF8B5224E34682CB32368002BB1
:10F620003AD1204F1D4604E03468ECB12368002B2A
:10F6300032D1A36803B1DD602069336003682575AA
:10F640001B68BB4221D1037F4560022BC46020D0E0
:10F65000FFF748FF6368002BE6D023602046FFF7E2
:10F66000A5FF3468002CE1D1EFF3108372B60E4A87
:10F6700000211068116003B962B628B18468FFF7F1
:10F6800095FF20460028F9D1F8BD22460021984771
:10F69000E0E783689847DDE7013B2360E4E700BFCC
:10F6A0002CA1FF1F35B600003CA1FF1F024A1368C2
:10F6B00001331360FFF7AEBF489FFF1FF8B572B16B
:10F6C00006460F4614460025336817F8011B1B68D1
:10F6D00030469847013C0544F6D12846F8BD15460A
:10F6E000FBE700BF00B5064A036812885B6883B079
:10F6F00001A9ADF804200222984703B05DF804FB8D
:10F70000C8440100F0B507468BB0002A33D0012A67
:10F7100008BF0A2251B3212400E0F4B2B1FBF2F594
:10F7200002FB1511C8B2092900F1300198BFC8B217
:10F730000AA988BF3730214488BFC0B201F8240C21
:10F74000661E2946002DE8D133B1013CE4B20AAB74
:10F7500023442D2203F8242C3B6801AA11195B686D
:10F760003846C4F1220298470BB0F0BD30228DF824
:10F7700025202124E8E70368C9B21B6898470BB02D
:10F78000F0BD00BF0029BABF49422D2300230A2241
:10F79000FFF7B8BF08B5F2F739FCF9F761FF00F0E1
:10F7A00015F8FAE7FFF74EBDFFF722BDFFF76ABD78
:10F7B000FFF752BEFFF72CBE08461146FFF794BD77
:10F7C0000846FFF719BE00BF704700BF38B5224C8E
:10F7D000237803B138BD01232370FFF753FD70BBBD
:10F7E00000F042F840BB00F0D5F810BBFEF72CFC4F
:10F7F000E0B900232370EFF30583002BEAD1EFF388
:10F80000108172B6154B1868E0B1154C2278CAB950
:10F8100045691D6001232370C5B1AA6101B962B6B3
:10F8200000254577836898472570D3E700F08EF967
:10F83000DFE700F089F9D9E700F084F9D3E7FFF7B3
:10F84000C3FFCDE70029C5D162B638BD054B1D60A9
:10F850000029E5D1E3E700BF40A1FF1F34A1FF1F4E
:10F8600038A1FF1F30A1FF1F054A064B10781B78F7
:10F87000C0B2DBB2984238BF4030C01A704700BFF8
:10F8800048A1FF1F49A1FF1FF0B4384B1A7912F0AD
:10F89000300F2CD072B6997D01F0FF0200293DD0C7
:10F8A00062B6334F334938780D78334E1C46C0B2B8
:10F8B000EDB2431C402BE17928BF0023AB4202F19B
:10F8C000FF32C9B21CBFF154184612F0FF02F0D14A
:10F8D0002A4B1B68C2B23A704BB1A84236BFC5F181
:10F8E0004005401B40192728C4BF01221A701F4938
:10F8F000CA78D2B2150616D452060DD51B4B1B7909
:10F900005B0609D51E4B1F491B6800220A7003B114
:10F910001A70164B3C22DA70F0BC70474022D9793D
:10F920005A7462B6E3E70B791C06E5D5164B174E01
:10F930001C783378E4B2DBB29C420ED0144D01E067
:10F94000A3420AD00133402B28BF00230879E85C8A
:10F95000C0B2C871087D0728F2D9DBB20349337001
:10F960000B79180644BF7C23CB70C5E700A0064086
:10F9700048A1FF1F49A1FF1F8CA1FF1F44A1FF1F2A
:10F98000D0A1FF1FCCA1FF1FD4A1FF1FCDA1FF1F3E
:10F990004CA1FF1F054A064B10781B78C0B2DBB2A2
:10F9A000984238BF4030C01A704700BF48A2FF1FBE
:10F9B000DDA1FF1FF0B4384B1A7912F0300F2CD0B4
:10F9C00072B6997D01F0FF0200293DD062B6334F37
:10F9D000334938780D78334E1C46C0B2EDB2431C23
:10F9E000402BE17928BF0023AB4202F1FF32C9B2BC
:10F9F0001CBFF154184612F0FF02F0D12A4B1B68CD
:10FA0000C2B23A704BB1A84236BFC5F14005401BA7
:10FA100040192728C4BF01221A701F49CA78D2B2E0
:10FA2000150616D452060DD51B4B1B795B0609D55E
:10FA30001E4B1F491B6800220A7003B11A70164B37
:10FA40003C22DA70F0BC70474022D9795A7462B611
:10FA5000E3E70B791C06E5D5164B174E1C78337877
:10FA6000E4B2DBB29C420ED0144D01E0A3420AD0B6
:10FA70000133282B28BF00230879E85CC0B2C87185
:10FA8000087D0728F2D9DBB2034933700B791806D9
:10FA900044BF7C23CB70C5E700B0064048A2FF1FDF
:10FAA000DDA1FF1F08A2FF1FD8A1FF1F4CA2FF1F4F
:10FAB000DCA1FF1F50A2FF1F49A2FF1FE0A1FF1FF3
:10FAC00070B584B072B6194B194D1A487022412690
:10FAD0000F2480211A702E701A4604701970137842
:10FAE0001B06FCD5144B186862B6144B144C984294
:10FAF00098BF00EB800001A998BF40000A22FDF7E3
:10FB000051FC01A92046002311F8012B01333AB121
:10FB10000A2B20F8022FF7D11623237004B070BDF2
:10FB20005B00DBB2237004B070BD00BF0000024078
:10FB30000700024006000240080002407F9698003D
:10FB4000E894FF1F704700BF704700BF704700BFB9
:10FB50002DE9F043DFF8EC808BB006460F4600F04D
:10FB600073F898F90030013304460D4637D030461B
:10FB7000394600F0DFF9002831D02BA3D3E9002368
:10FB80003046394600F026FE814668BB28A3D3E9FB
:10FB900000233046394600F0FFFD00B398F90030ED
:10FBA000254ACDF82090042400200021022BCDE925
:10FBB0000467CDE9026700940192CDE906012CD0DB
:10FBC000684600F0BDF940B3089B1BB101F0F4F9A1
:10FBD000089B0360DDE906010BB0BDE8F083204619
:10FBE00029460BB0BDE8F083134A98F90030019222
:10FBF00003210022CDE90467CDE902670091089254
:10FC00002BB90E4B4FF06042CDE90623D8E70C49E3
:10FC10000020022BCDE90601D2D101F0CDF922233B
:10FC20000360D1E7AFF30080EF39FAFE422E864041
:10FC300051302DD5104987C060450100FFFFEF47C7
:10FC40000000F07FFE94FF1F2DE9F04FB04F21F030
:10FC50000042BA4283B00C464FEAD17605460DD930
:10FC6000AC4FBA4225D9C1F31303034340F0EF80F0
:10FC70000EB10020014603B0BDE8F08FA64B9A42BA
:10FC800000F2CC80A54B9A4200F2DE808AA3D3E931
:10FC9000002300F05DF90022A14B00F09BFD00283D
:10FCA00000F005812846214600229D4B00F050F9C6
:10FCB000E1E783A3D3E9002300F08CFD002840F0A6
:10FCC000CB802846214680A3D3E9002300F064FDC1
:10FCD0000028CED1934B284603EBC60821467CA3CF
:10FCE000D3E9002300F0E6FAD8E9002300F030F968
:10FCF00000F07AFD804600F077FA77A3D3E900237D
:10FD000006460F4600F0D6FA02460B462846214624
:10FD100000F01CF972A3D3E90023CDE900013046BD
:10FD2000394600F0C7FA82468B4652465B46DDE90B
:10FD3000000100F00BF905460C462A4623462846EA
:10FD4000214600F0B7FA68A3D3E9002306460F4620
:10FD500000F0B0FA66A3D3E9002300F0F7F83246CA
:10FD60003B4600F0A7FA64A3D3E9002300F0F0F8C3
:10FD700032463B4600F09EFA61A3D3E9002300F02F
:10FD8000E5F832463B4600F095FA5FA3D3E900233D
:10FD900000F0DEF832463B4600F08CFA02460B4695
:10FDA0002846214600F0D2F806460F46284621464E
:10FDB00032463B46B8F1000F56D000F07BFA32468F
:10FDC00004460D463B4600204FF0804100F0BEF84F
:10FDD00002460B462046294600F096FB02460B469B
:10FDE0005046594600F0B2F8DDE9002300F0AEF8C5
:10FDF0000B4602464A49002000F0A8F86FF47F73D2
:10FE000098454FDA08F57A7801EB085100224FF057
:10FE1000B87300F04FFA03B0BDE8F08F424B9A423E
:10FE20003FF658AF414BF4002344D3E9002300F0E0
:10FE30008DF83F4BC6F101081C44CDE90001D4E91F
:10FE400000ABC6EB080870E74FF0000875E7024604
:10FE50000B4600F07DF80EE717A3D3E90023104608
:10FE6000194600F027FA06E700F024FA002280463F
:10FE700089464FF080433046394600F067F8024625
:10FE80000B464046494600F03FFB2A46234600F019
:10FE90005DF802460B460020214900F057F803B0F8
:10FEA000BDE8F08F01EB085103B0BDE8F08F80464C
:10FEB00043E700BFAFF300809C7500883CE4377EC9
:10FEC000EF39FAFE422E864051302DD5104987C0B9
:10FED000FE822B654715F73F0000E0FE422EE63F0D
:10FEE000763C7935EF39EA3DD0A4BE726937663E7B
:10FEF000F16BD2C541BDBB3E2CDE25AF6A56113F2A
:10FF000093BDBE166CC1663F3E5555555555C53F10
:10FF1000412E8640FFFFEF7F422ED63FFFFF2F3E50
:10FF20000000F03F68450100B1A2F03F88450100A4
:10FF30007845010041F0004101F58010C00F704785
:10FF40000020704781F0004102E000BF83F00043D1
:10FF500030B54FEA41044FEA430594EA050F08BF64
:10FF600090EA020F1FBF54EA000C55EA020C7FEA28
:10FF7000645C7FEA655C00F0E2804FEA5454D4EBA5
:10FF80005555B8BF6D420CDD2C4480EA020281EA6F
:10FF9000030382EA000083EA010180EA020281EAA7
:10FFA0000303362D88BF30BD11F0004F4FEA0131F9
:10FFB0004FF4801C4CEA113102D0404261EB410108
:10FFC00013F0004F4FEA03334CEA133302D052428E
:10FFD00063EB430394EA050F00F0A780A4F101044A
:10FFE000D5F1200E0DDB02FA0EFC22FA05F2801884
:10FFF00041F1000103FA0EF2801843FA05F359416A
:020000021000EC
:100000000EE0A5F120050EF1200E012A03FA0EFCE8
:1000100028BF4CF0020C43FA05F3C01851EBE37112
:1000200001F0004507D54FF0000EDCF1000C7EEB2F
:1000300000006EEB0101B1F5801F1BD3B1F5001F6D
:100040000CD349085FEA30004FEA3C0C04F101048C
:100050004FEA445212F5800F80F09A80BCF1004FB5
:1000600008BF5FEA500C50F1000041EB045141EA37
:10007000050130BD5FEA4C0C404141EB010111F438
:10008000801FA4F10104E9D191F0000F04BF0146E3
:100090000020B1FA81F308BF2033A3F10B03B3F1C1
:1000A00020020CDA0C3208DD02F1140CC2F10C0251
:1000B00001FA0CF021FA02F10CE002F11402D8BFAF
:1000C000C2F1200C01FA02F120FA0CFCDCBF41EA7B
:1000D0000C019040E41AA2BF01EB0451294330BD4A
:1000E0006FEA04041F3C1CDA0C340EDC04F1140427
:1000F000C4F1200220FA04F001FA02F340EA0300FE
:1001000021FA04F345EA030130BDC4F10C04C4F143
:10011000200220FA02F001FA04F340EA0300294623
:1001200030BD21FA04F0294630BD94F0000F83F46D
:10013000801306BF81F480110134013D4EE77FEA50
:10014000645C18BF7FEA655C29D094EA050F08BF9C
:1001500090EA020F05D054EA000C04BF194610467D
:1001600030BD91EA030F1EBF0021002030BD5FEAC1
:10017000545C05D14000494128BF41F0004130BDE9
:1001800014F580043CBF01F5801130BD01F000453D
:1001900045F0FE4141F470014FF0000030BD7FEAB0
:1001A000645C1ABF194610467FEA655C1CBF0B46AB
:1001B000024650EA013406BF52EA033591EA030FC2
:1001C00041F4002130BD00BF90F0000F04BF0021BA
:1001D000704730B54FF4806404F132044FF00005ED
:1001E0004FF0000150E700BF90F0000F04BF002166
:1001F000704730B54FF4806404F1320410F00045CC
:1002000048BF40424FF000013EE700BF42004FEAC6
:10021000E2014FEA31014FEA02701FBF12F07F4343
:1002200093F07F4F81F06051704792F0000F14BF40
:1002300093F07F4F704730B54FF4607401F0004584
:1002400021F0004120E700BF50EA010208BF7047DB
:1002500030B54FF000050AE050EA010208BF7047D0
:1002600030B511F0004502D5404261EB41014FF439
:10027000806404F132045FEA915C3FF4DCAE4FF03D
:1002800003025FEADC0C18BF03325FEADC0C18BF24
:10029000033202EBDC02C2F1200300FA03FC20FA75
:1002A00002F001FA03FE40EA0E0021FA02F11444C2
:1002B000C1E600BF70B54FF0FF0C4CF4E06C1CEAD7
:1002C00011541DBF1CEA135594EA0C0F95EA0C0F4C
:1002D00000F0DEF82C4481EA030621EA4C5123EABF
:1002E0004C5350EA013518BF52EA033541F48011EE
:1002F00043F4801338D0A0FB02CE4FF00005E1FBA1
:1003000002E506F00042E0FB03E54FF00006E1FBEA
:1003100003569CF0000F18BF4EF0010EA4F1FF042D
:10032000B6F5007F64F5407404D25FEA4E0E6D416D
:1003300046EB060642EAC62141EA55514FEAC5207E
:1003400040EA5E504FEACE2EB4F1FD0C88BFBCF5FA
:10035000E06F1ED8BEF1004F08BF5FEA500E50F1AB
:10036000000041EB045170BD06F0004646EA010171
:1003700040EA020081EA0301B4EB5C04C2BFD4EBA3
:100380000C0541EA045170BD41F480114FF0000E9C
:10039000013C00F3AB8014F1360FDEBF002001F00A
:1003A000004170BDC4F10004203C35DA0C341BDC84
:1003B00004F11404C4F1200500FA05F320FA04F056
:1003C00001FA05F240EA020001F0004221F000418A
:1003D00010EBD37021FA04F642EB06015EEA430EFD
:1003E00008BF20EAD37070BDC4F10C04C4F120052D
:1003F00000FA04F320FA05F001FA04F240EA0200E0
:1004000001F0004110EBD37041F100015EEA430EB0
:1004100008BF20EAD37070BDC4F1200500FA05F2D0
:100420004EEA020E20FA04F301FA05F243EA02034F
:1004300021FA04F001F0004121FA04F220EA02005E
:1004400000EBD3705EEA430E08BF20EAD37070BDA4
:1004500094F0000F0FD101F00046400041EB010184
:1004600011F4801F08BF013CF7D041EA060195F066
:10047000000F18BF704703F00046520043EB030320
:1004800013F4801F08BF013DF7D043EA060370470D
:1004900094EA0C0F0CEA135518BF95EA0C0F0CD018
:1004A00050EA410618BF52EA4306D1D181EA03015E
:1004B00001F000414FF0000070BD50EA410606BF58
:1004C0001046194652EA430619D094EA0C0F02D19D
:1004D00050EA013613D195EA0C0F05D152EA0336E2
:1004E0001CBF104619460AD181EA030101F0004100
:1004F00041F0FE4141F470014FF0000070BD41F049
:10050000FE4141F4780170BD70B54FF0FF0C4CF422
:10051000E06C1CEA11541DBF1CEA135594EA0C0F41
:1005200095EA0C0F00F0A7F8A4EB050481EA030E8E
:1005300052EA03354FEA013100F088804FEA033375
:100540004FF0805545EA131343EA12634FEA022243
:1005500045EA111545EA10654FEA00260EF0004104
:100560009D4208BF964244F1FD0404F5407402D256
:100570005B084FEA3202B61A65EB03055B084FEAE7
:1005800032024FF480104FF4002CB6EB020E75EBE4
:10059000030E22BFB61A754640EA0C005B084FEA0C
:1005A0003202B6EB020E75EB030E22BFB61A754689
:1005B00040EA5C005B084FEA3202B6EB020E75EBD4
:1005C000030E22BFB61A754640EA9C005B084FEA4C
:1005D0003202B6EB020E75EB030E22BFB61A754659
:1005E00040EADC0055EA060E18D04FEA051545EA48
:1005F00016754FEA06164FEAC30343EA52734FEAF1
:10060000C2025FEA1C1CC0D111F4801F0BD141EA69
:1006100000014FF000004FF0004CB6E711F4801FCE
:1006200004BF01430020B4F1FD0C88BFBCF5E06FAE
:100630003FF6AFAEB5EB030C04BFB6EB020C5FEABE
:10064000500C50F1000041EB045170BD0EF0004E13
:100650004EEA113114EB5C04C2BFD4EB0C0541EA45
:10066000045170BD41F480114FF0000E013C90E642
:1006700045EA060E8DE60CEA135594EA0C0F08BF06
:1006800095EA0C0F3FF43BAF94EA0C0F0AD150EA05
:1006900001347FF434AF95EA0C0F7FF425AF104698
:1006A00019462CE795EA0C0F06D152EA03353FF4C0
:1006B000FDAE1046194622E750EA410618BF52EA3D
:1006C00043067FF4C5AE50EA41047FF40DAF52EA11
:1006D00043057FF4EBAE12E74FF0FF3C06E000BFAE
:1006E0004FF0010C02E000BF4FF0010C4DF804CDBB
:1006F0004FEA410C7FEA6C5C4FEA430C18BF7FEA7B
:100700006C5C1BD001B050EA410C0CBF52EA430CA8
:1007100091EA030F02BF90EA020F0020704710F128
:10072000000F91EA030F58BF994208BF90422CBFB7
:10073000D8176FEAE37040F0010070474FEA410CB0
:100740007FEA6C5C02D150EA013C07D14FEA430CCE
:100750007FEA6C5CD6D152EA033CD3D05DF8040B3F
:10076000704700BF8446104662468C461946634671
:1007700000E000BF01B5FFF7B7FF002848BF10F148
:10078000000F01BD4DF808EDFFF7F4FF0CBF01208D
:1007900000205DF808FB00BF4DF808EDFFF7EAFF09
:1007A00034BF012000205DF808FB00BF4DF808EDC4
:1007B000FFF7E0FF94BF012000205DF808FB00BFB9
:1007C0004DF808EDFFF7CEFF94BF012000205DF843
:1007D00008FB00BF4DF808EDFFF7C4FF34BF012050
:1007E00000205DF808FB00BF4FEA410212F500123D
:1007F00015D211D56FF47873B3EB625212D94FEA68
:10080000C12343F0004343EA505311F0004F23FA51
:1008100002F018BF404270474FF00000704750EAA6
:10082000013005D111F0004008BF6FF00040704763
:100830004FF00000704700BF4FEA4102B2F1E043C1
:1008400024BFB3F5001CDCF1FE5C0DD901F0004CB7
:100850004FEAC0024CEA5070B2F1004F40EB830007
:1008600008BF20F00100704711F0804F21D113F133
:100870003872BCBF01F00040704741F480114FEA6C
:100880005252C2F11802C2F1200C10FA0CF320FAF5
:1008900002F018BF40F001004FEAC1234FEAD32312
:1008A00003FA0CFC40EA0C0023FA02F34FEA43037C
:1008B000CCE77FEA625307D150EA01331EBF4FF005
:1008C000FE4040F44000704701F0004040F0FE4020
:1008D00040F40000704700BF80F0004002E000BF1D
:1008E00081F0004142001FBF5FEA410392EA030F1B
:1008F0007FEA226C7FEA236C6AD04FEA1262D2EB65
:100900001363C1BFD218414048404140B8BF5B4269
:10091000192B88BF704710F0004F40F4000020F002
:100920007F4018BF404211F0004F41F4000121F018
:100930007F4118BF494292EA030F3FD0A2F1010262
:1009400041FA03FC10EB0C00C3F1200301FA03F1A0
:1009500000F0004302D5494260EB4000B0F5000FC3
:1009600013D3B0F1807F06D340084FEA310102F182
:100970000102FE2A51D2B1F1004F40EBC25008BF34
:1009800020F0010040EA03007047490040EB0000FE
:1009900010F4000FA2F10102EDD1B0FA80FCACF12D
:1009A000080CB2EB0C0200FA0CF0AABF00EBC2502C
:1009B00052421843BCBFD0401843704792F0000F1A
:1009C00081F4000106BF80F400000132013BB5E76D
:1009D0004FEA41037FEA226C18BF7FEA236C21D0E3
:1009E00092EA030F04D092F0000F08BF0846704748
:1009F00090EA010F1CBF0020704712F07F4F04D116
:100A0000400028BF40F00040704712F100723CBF28
:100A100000F50000704700F0004343F0FE4040F452
:100A2000000070477FEA226216BF08467FEA236310
:100A30000146420206BF5FEA412390EA010F40F4FB
:100A4000800070474FF0000304E000BF10F0004347
:100A500048BF40425FEA000C08BF704743F096432E
:100A600001464FF000001CE050EA010208BF704749
:100A70004FF000030AE000BF50EA010208BF7047D0
:100A800011F0004302D5404261EB41015FEA010CE5
:100A900002BF84460146002043F0B64308BFA3F1DD
:100AA0008053A3F50003BCFA8CF2083AA3EBC253BF
:100AB00010DB01FA02FC634400FA02FCC2F12002DE
:100AC000BCF1004F20FA02F243EB020008BF20F015
:100AD0000100704702F1200201FA02FCC2F120027B
:100AE00050EA4C0021FA02F243EB020008BF20EA70
:100AF000DC7070474FF0FF0C1CEAD0521EBF1CEA9E
:100B0000D15392EA0C0F93EA0C0F6FD01A4480EA8B
:100B1000010C400218BF5FEA41211ED04FF0006374
:100B200043EA501043EA5111A0FB01310CF00040A0
:100B3000B1F5000F3EBF490041EAD3715B0040EAC6
:100B4000010062F17F02FD2A1DD8B3F1004F40EB96
:100B5000C25008BF20F00100704790F0000F0CF069
:100B6000004C08BF49024CEA502040EA51207F3A2D
:100B7000C2BFD2F1FF0340EAC250704740F4000008
:100B80004FF00003013A5DDC12F1190FDCBF00F0F9
:100B900000407047C2F10002410021FA02F1C2F1A7
:100BA000200200FA02FC5FEA310040F1000053EA43
:100BB0004C0308BF20EADC70704792F0000F00F091
:100BC000004C02BF400010F4000F013AF9D040EA97
:100BD0000C0093F0000F01F0004C02BF490011F42B
:100BE000000F013BF9D041EA0C018FE70CEAD15329
:100BF00092EA0C0F18BF93EA0C0F0AD030F0004CA9
:100C000018BF31F0004CD8D180EA010000F000405C
:100C1000704790F0000F17BF90F0004F084691F01A
:100C2000000F91F0004F14D092EA0C0F01D1420254
:100C30000FD193EA0C0F03D14B0218BF084608D11D
:100C400080EA010000F0004040F0FE4040F4000067
:100C5000704740F0FE4040F4400070474FF0FF0CFA
:100C60001CEAD0521EBF1CEAD15392EA0C0F93EA41
:100C70000C0F69D0A2EB030280EA010C49024FEA93
:100C8000402037D04FF0805343EA111143EA10134C
:100C90000CF000408B4238BF5B0042F17D024FF404
:100CA000000C8B4224BF5B1A40EA0C00B3EB510FDF
:100CB00024BFA3EB510340EA5C00B3EB910F24BFC8
:100CC000A3EB910340EA9C00B3EBD10F24BFA3EB4D
:100CD000D10340EADC001B0118BF5FEA1C1CE0D115
:100CE000FD2A3FF650AF8B4240EBC25008BF20F0C8
:100CF000010070470CF0004C4CEA50207F32C2BF1C
:100D0000D2F1FF0340EAC250704740F400004FF0B8
:100D10000003013A37E792F0000F00F0004C02BFE9
:100D2000400010F4000F013AF9D040EA0C0093F0B3
:100D3000000F01F0004C02BF490011F4000F013B0D
:100D4000F9D041EA0C0195E70CEAD15392EA0C0F75
:100D500008D142027FF47DAF93EA0C0F7FF470AFAD
:100D6000084676E793EA0C0F04D14B023FF44CAFF0
:100D700008466EE730F0004C18BF31F0004CCAD185
:100D800030F000427FF45CAF31F000437FF43CAFC1
:100D90005FE700BF4FF0FF3C06E000BF4FF0010CE3
:100DA00002E000BF4FF0010C4DF804CD4FEA4002C5
:100DB0004FEA41037FEA226C18BF7FEA236C11D00F
:100DC00001B052EA530C18BF90EA010F58BFB2EBC2
:100DD000030088BFC81738BF6FEAE17018BF40F042
:100DE000010070477FEA226C02D15FEA402C05D1F6
:100DF0007FEA236CE4D15FEA412CE1D05DF8040B7B
:100E0000704700BF844608466146FFE70FB5FFF70D
:100E1000C9FF002848BF10F1000F0FBD4DF808EDC5
:100E2000FFF7F4FF0CBF012000205DF808FB00BFB6
:100E30004DF808EDFFF7EAFF34BF012000205DF810
:100E400008FB00BF4DF808EDFFF7E0FF94BF01205D
:100E500000205DF808FB00BF4DF808EDFFF7D2FF5A
:100E600094BF012000205DF808FB00BF4DF808ED9D
:100E7000FFF7C8FF34BF012000205DF808FB00BF6A
:100E80004FEA40024FEA41037FEA226C02D15FEA57
:100E9000402C08D17FEA236C02D15FEA412C02D1B9
:100EA0004FF0000070474FF0010070474FEA4002DA
:100EB000B2F1FE4F0FD34FF09E03B3EB12620DD988
:100EC0004FEA002343F0004310F0004F23FA02F0F2
:100ED00018BF404270474FF00000704712F1610F99
:100EE00001D1420205D110F0004008BF6FF0004070
:100EF00070474FF00000704742000ED2B2F1FE4F33
:100F00000BD34FF09E03B3EB126209D44FEA0023D8
:100F100043F0004323FA02F070474FF0000070479F
:100F200012F1610F01D1420202D14FF0FF30704740
:100F30004FF00000704700BF10B502FB01F100F058
:100F400071F80446D8B150F8042C22F00302043A98
:100F5000242A18D8132A14D900231B2A03604360BB
:100F600016D9242A8360C36011BF00F11002036107
:100F7000436100F118020023136053609360204620
:100F800010BD0246F7E7002100F068FB204610BDC7
:100F900000F10802EFE700BFF0B583B016461F4628
:100FA0000D460024FFF732F9009733462A46019494
:100FB00000F044FE03B0F0BD014B1868704700BF5D
:100FC0002899FF1F70B50F4E0F4D761BB61018BF36
:100FD000002405D0013455F8043B9847A642F9D1C6
:100FE0000A4E0B4D761B03F063FBB61018BF0024AE
:100FF00006D0013455F8043B9847A642F9D170BD9C
:1010000070BD00BFBC460100BC460100C8460100DF
:10101000BC460100024B0146186800F003B800BF4F
:101020002899FF1F2DE9F04F01F10B05162D83B014
:10103000064640F29F8035F0070500F1BF80A942C7
:1010400000F2BC8000F058FBB5F5FC7FC0F09C823C
:101050006B0A00F0BA80042B00F28381A80900F12A
:10106000390E4FEA4E033830C44F07EB8303A3F128
:1010700008015C68A14207D1ACE0002A80F2AC8094
:10108000E468A14200F0A680636823F003035A1BC2
:101090000F2AF2DDB9493C6901F1080E744500F0F0
:1010A000B381636823F003035A1B0F2A00F399816D
:1010B000002AC1F814E0C1F810E080F29E80B3F578
:1010C000007F80F06781DB0803F1010C01229B1097
:1010D00002FA03F34A6851F83C80C4F8088001EB37
:1010E000CC091A43A9F10803E3604A6041F83C4087
:1010F000C8F80C40831001249C40944200F28A807E
:10110000144206D120F003006400144200F10400F0
:10111000FAD007EBC009CC468046DCF80C108C45B1
:1011200007D173E1002A80F28181C9688C4500F003
:101130006D814B6823F003035A1B0F2AF2DD0C4626
:10114000D1F80CC054F8088F4B1945F001054D60DB
:1011500042F00101C8F80CC03046CCF808807B6131
:101160003B61C3F80CE0C3F808E059609A5000F006
:10117000C5FA1FE0102921D800F0BEFA1025062379
:1011800002207E4F07EB8303A3F108025C689442C0
:1011900000F045816368E168A56823F003032344F8
:1011A00030465A68E96042F001028D605A6000F0F2
:1011B000A5FA0834204603B0BDE8F08F00240C23C4
:1011C0002046336003B0BDE8F08F80234FF0400E1F
:1011D0003F2049E770465DE72344E1685A68A56807
:1011E00042F00102E96030468D605A6000F086FAF4
:1011F0000834204603B0BDE8F08F234430465A68D7
:1012000042F001025A6000F079FA0834204603B037
:10121000BDE8F08FBC68636823F00308A84504D3D9
:10122000C5EB08030F2B00F38C80554BDFF8609162
:101230001A68D9F8003001332A4404EB080A00F098
:10124000608102F580520F3222F47F6222F00F0299
:1012500011463046019200F043FCB0F1FF3F834657
:10126000019A00F05881824500F2FC80454B1968D4
:10127000DA451144196000F05381D9F80000DFF815
:1012800010E101301BBFCAEB0B0A5144CEF800B08D
:1012900019601BF0070100F01781C1F10800C1F5CA
:1012A0008051834408315A44C2F30B02C2EB010956
:1012B00049463046019300F013FC431C019B00F0AB
:1012C0003F81CBEB00024A4442F001021968C7F8A3
:1012D00008B04944BC42CBF804201960DFF8A49060
:1012E00016D0B8F10F0F40F2FD806268A8F10C0330
:1012F00023F00703E01802F001024FF0050E1A4335
:101300000F2B6260C0F804E0C0F808E000F21C8116
:101310001D4BBC681A68914288BF19601B4B1A6844
:101320009142626888BF196022F003029542A2EBE5
:10133000050301D80F2B04DC304600F0DFF9002450
:1013400038E7621943F0010345F001056560304656
:10135000BA60536000F0D2F90834204603B0BDE80B
:10136000F08F142B71D9542B00F2A480280B00F1BC
:101370006F0E4FEA4E036E3076E600BF2C99FF1FCA
:101380005CA2FF1F60A2FF1F58A2FF1F54A2FF1FF5
:10139000389DFF1F5A0A042A5ED9142A00F2B3802E
:1013A00002F15C0149005B3207EB810C57F8211018
:1013B000DFF8DC81ACF1080C8C4500F088804A68CD
:1013C00022F00302934202D289688C45F7D1D1F80A
:1013D0000CC07A68C4F80CC0A160CCF80840CC609E
:1013E00088E6631942F0010745F001056560304663
:1013F0004B610B61C3F80CE0C3F808E05F609A50E2
:10140000083400F07BF9D5E64A6873E608F1010874
:1014100018F0030F0CF1080C7FF47FAE30E0DC68AD
:10142000A34208BF02303FF435AEB3E60B440C468E
:101430005A68C96854F8085F42F001025A603046A1
:10144000E9608D6000F05AF9B4E603F15C0E03F137
:101450005B004FEA4E0307E69A0902F139014900A1
:101460003832A1E7BC424A4B3FF400AF9C68626847
:1014700022F003025AE759F80839994540F0828072
:1014800010F0030F00F1FF30F5D17B6823EA04036D
:101490007B6064009C423FF6BDAE002C3FF4BAAEC8
:1014A0001C4240467FF435AE64001C4200F104004B
:1014B000FAD02EE6B3F5AA7F18D8E80B00F1780E23
:1014C0004FEA4E037730CFE54FF48051EBE6012130
:1014D000D8F80430921001FA02F21A43C8F8042036
:1014E000614677E70123CBF8043025E740F25452F8
:1014F000934220D8A80C00F17D0E4FEA4E037C30B9
:10150000B2E51032A4E6542A26D81A0B02F16F0174
:1015100049006E3248E7BC68626822F0030205E7C2
:10152000CAF30B0000287FF4A8AE4244BB6842F027
:1015300001025A60ECE6FE234FF07F0E7E2093E519
:1015400001224FF00009C1E604F10801304600F025
:101550004DFCD9F80010DBE6B2F5AA7F05D8DA0B0E
:1015600002F17801490077321EE740F254518A4275
:1015700005D89A0C02F17D0149007C3214E7FE2166
:101580007E2211E77B6884E7E808431C5B00F8E5EE
:101590002C99FF1F8842F0B50DD98B1898420AD2BA
:1015A0008118002A51D09A1A13F8014D01F8014D03
:1015B0009342F9D1F0BD0F2A48D941EA00039B07B5
:1015C00046D100F1100401F11003154653F8106CD8
:1015D00044F8106C53F80C6C44F80C6C53F8086C1D
:1015E00044F8086C103D53F8046C44F8046C0F2D5B
:1015F00003F1100304F11004E8D8A2F1100323F062
:101600000F0302F00F0E1033BEF1030F1944034411
:1016100021D91E1F0D467446043C55F8047B46F83C
:10162000047F032CF8D8AEF1040424F0030404343E
:101630002344214402F0030262B1013B0A4411F841
:10164000014B03F8014F8A42F9D1F0BD0346F3E79D
:101650000346F2E7F0BD7246EEE700BF70B48407C0
:1016600046D0541E002A41D0CDB2034602E0621E8D
:10167000E4B3144603F8015B9A07F8D1032C2ED982
:10168000CDB245EA05250F2C45EA054519D903F1E8
:1016900010022646103E0F2E42F8105C42F80C5CF9
:1016A00042F8085C42F8045C02F11002F2D8A4F19E
:1016B000100222F00F0204F00F041032032C134426
:1016C0000DD91E462246043A032A46F8045BFAD88E
:1016D000221F22F003020432134404F003042CB14D
:1016E000C9B21C4403F8011BA342FBD170BC704774
:1016F00014460346C2E700BF704700BF704700BFF3
:101700002DE9F04F174683B0002900F0C1800E4646
:10171000814607F10B05FFF7EFFF56F804EC162D95
:101720002EF00304A6F1080840D810221546AF4257
:1017300041D8944275DAC94B996808EB0400884295
:10174000416800F0D98021F0010303445B68DB07A6
:101750007DD51EF0010F35D039464846FFF762FCB3
:101760000746E0B156F8043C23F001034344A0F1DE
:1017700008029A4200F04481221F242A00F231819B
:10178000132A00F204810346324611681960516839
:10179000596092689A603146484600F027FB4846F7
:1017A000FFF7ACFF384603B0BDE8F08F25F0070522
:1017B000002D2A46BBDA0C230020C9F8003003B004
:1017C000BDE8F08F56F8083CC3EB080ADAF804309D
:1017D00023F0030C04EB0C039342BDDB5746DAF80D
:1017E0000C1057F8080F221F242AC160886000F2ED
:1017F0001781132A40F212813168CAF80810716803
:10180000CAF80C101B2A00F22B8108360AF11002CC
:101810003168116071685160B16891603E461C4644
:10182000D046631B0F2B1DD8D8F8043003F00103FA
:1018300023434444C8F80430636843F00103636001
:101840004846FFF75BFF304603B0BDE8F08F21F05C
:1018500003012144914221DBC36882680C46D360B6
:101860009A60DEE7D8F8042008EB050102F00102D7
:10187000154343F001020B44C8F804504A605A680B
:1018800042F0010208315A60484600F0AFFAD7E74B
:10189000114603B0BDE8F04FFFF7C4BB1EF0010FC7
:1018A0007FF45AAF56F8083CC3EB080ADAF8043064
:1018B00023F0030C01EB0C0E96458BDBC3688268AA
:1018C0005746D3609A6057F8081FDAF80C30CB609F
:1018D000221F242A996000F29980132A62D9336862
:1018E000CAF808307368CAF80C301B2A00F2A080CE
:1018F00008360AF1100356E021F0030BA34405F16A
:101900001000834559DA1EF0010F7FF425AF56F819
:10191000081CC1EB080ADAF8041021F0030CE344B8
:1019200058453FF757AF5746DAF80C1057F8080FED
:10193000221F242AC160886000F2B480132A40F27A
:10194000A5803168CAF808107168CAF80C101B2A03
:1019500000F2AF8008360AF1100231681160716838
:101960005160B16891600AEB0501C5EB0B0242F0D2
:10197000010299604A60DAF8043003F001031D4364
:101980004846CAF80450FFF7B9FE38465CE73368AA
:101990000360736843601B2A27D800F1080306F12F
:1019A0000802F2E63B4632681A6072685A60B26812
:1019B0009A603E467446D04633E708EB0501C5EB16
:1019C0000B0B4BF0010299604A6056F8043C03F09F
:1019D00001031D43484646F8045CFFF78FFE30467E
:1019E00032E73146FFF7D6FDD5E6B3688360F3688A
:1019F000C360242A28D000F1100306F11002C4E6C7
:101A000050F8043C23F003031C440AE731463846EF
:101A10007446D046FFF7BEFD3E4602E73A46F7E67B
:101A2000314638461C46D046FFF7B4FD3E46F8E640
:101A3000B368CAF81030F368CAF81430242A1BD0EF
:101A400010360AF11803AEE7336903617369436125
:101A500006F1180200F1180397E600BF2C99FF1F4A
:101A6000B168CAF81010F168CAF81410242A0FD00F
:101A700010360AF11802CBE63369CAF818307369D8
:101A8000CAF81C3018360AF120038CE73A4664E79E
:101A90003269CAF818207269CAF81C2018360AF18F
:101AA0002002B5E6314638460193FFF773FD019BEE
:101AB00059E7B168CAF81010F168CAF81410242A5E
:101AC00003D010360AF1180247E73269CAF8182025
:101AD0007269CAF81C2018360AF120023DE700BFDF
:101AE00038B5074C0023054608462360FBF724FC65
:101AF000431C00D038BD2368002BFBD02B6038BDC1
:101B0000BCA3FF1FFFFFFFFFFFFFFFFFFFFFFFFF64
:101B1000FFFFFFFFFFFFFFFFFFFFFFFFFFFFFFFFD5
:101B2000FFFFFFFFFFFFFFFFFFFFFFFFFFFFFFFFC5
:101B3000FFFFFFFFFFFFFFFFFFFFFFFFFFFFFFFFB5
:101B400090F800F06DE9024520F007016FF0000CFD
:101B500010F0070491F820F040F049804FF00004A5
:101B60006FF00700D1E9002391F840F000F1080080
:101B700082FA4CF2A4FA8CF283FA4CF3A2FA8CF3B8
:101B80004BBBD1E9022382FA4CF200F10800A4FA1F
:101B90008CF283FA4CF3A2FA8CF3E3B9D1E9042373
:101BA00082FA4CF200F10800A4FA8CF283FA4CF3AA
:101BB000A2FA8CF37BB9D1E9062301F1200182FA64
:101BC0004CF200F10800A4FA8CF283FA4CF3A2FA6A
:101BD0008CF3002BC6D0002A04BF04301A4612BA78
:101BE000B2FA82F2FDE8024500EBD2007047D1E97B
:101BF000002304F00305C4F100004FEAC50514F00A
:101C0000040F91F840F00CFA05F562EA05021CBFDA
